:0200000480007A
:10000000971500009385059B732510FC6B10B500B8
:10001000EF00101A130510006B0005001785010092
:100020001305459B17860100130646AF3306A6400D
:1000300093050000EF10C00B17150000130505AE67
:10004000EF108006EF009023EF0080006F10000794
:1000500037650180130101FF130585AD23261100CB
:1000600023248100EF009035EF00401513040500B4
:10007000EF00C0213304A400EF00C02D3304A4001E
:10008000EF0080403304A400EF00005F3304A400BD
:10009000EF00C04E3304A400EF0040733304A4000B
:1000A0006312040237650180130585AEEF0010313D
:1000B0008320C10013050400032481001301010102
:1000C0006780000037650180130545AFEF00102FF2
:1000D0006FF01FFE9307000063880700371500804C
:1000E000130585B16F00507C67800000F32730CC8A
:1000F00037870180939627001307C7A53307D700DA
:10010000938617042320D70093B717006B8007004E
:100110006780000003A705001315250083A745008D
:100120003307A700032707003385A7002320E50036
:1001300067800000130101FE232E1100232C810093
:10014000232A910023282101232631012324410160
:100150006352B006930405001389150413041004B8
:1001600093090000376A018003A604009306040087
:1001700013050AB09305F4FB63068600EF00102414
:10018000938919001304140093844400E31E24FD92
:100190008320C1010324810183244101032901013A
:1001A000032A8100138509008329C100130101027C
:1001B00067800000930900006FF09FFD37650180A4
:1001C000130101FE130545B2232C8100232A91005F
:1001D000232821012326310123244101B7840180F2
:1001E000232E1100EF00901D9387C49E1307100467
:1001F00023A0E7001307200423A2E700130730041D
:1002000023A4E7001307400423A6E70013075004C4
:1002100023A8E7001307600423AAE700130770046C
:1002200023ACE7001307800423AEE7009384C49E49
:100230001304200413090000376A01809309900415
:1002400003A644009306040013050AB09305F4FBCB
:1002500063068600EF0090161309190013041400BA
:1002600093844400E31E34FD8320C10103248101F3
:10027000832441018329C100032A81001305090059
:100280000329010113010102678000003765018025
:10029000130101FC130585B3232C8102232A91024B
:1002A000232821032326310323244103232E110273
:1002B000EF00D010930710042320F10093072004CF
:1002C0002322F100930730042324F1009307400414
:1002D0002326F100930750042328F10093076004BC
:1002E000232AF10093077004232CF1009307800464
:1002F000232EF100930401001304200413090000CD
:10030000376A01809309900403A644009306040011
:1003100013050AB09305F4FB63068600EF00100A8C
:10032000130919001304140093844400E31E34FDE0
:100330008320C10303248103832441038329C10251
:10034000032A810213050900032901031301010493
:100350006780000037650180130101FF1305C5B4F4
:100360002324810023261100EF005005B7C7FFFEAC
:100370001307100423A6E7001307200423A8E700AF
:100380001307300423AAE7001307500423AEE70045
:100390001307600423A0E7021307700423A2E702F7
:1003A000130640041307800423ACC70023A4E7020C
:1003B0009307400413040000630EF60037650180C4
:1003C0009306400493053000130505B0EF00007F4D
:1003D00013041400B7C7FFFE03A6C7019307500418
:1003E000630EF600376501809306500493054000C4
:1003F000130505B0EF00807C13041400B7C7FFFE9F
:1004000003A6070293076004630EF60037650180B8
:100410009306600493055000130505B0EF00007AC1
:1004200013041400B7C7FFFE03A647029307700426
:10043000630EF60037650180930670049305600033
:10044000130505B0EF00807713041400B7C7FFFE53
:1004500003A6870293078004630EF60037650180C8
:100460009306800493057000130505B0EF00007536
:10047000130414008320C100130504000324810029
:10048000130101016780000037650180130101FF3E
:10049000130505B623261100232481002322910091
:1004A000EF00C071930740006B800700F32700CC7A
:1004B000378401801304C4A4139727003307E40092
:1004C000938717042320F700930710006B80070021
:1004D000032604009307100493040000630EF60043
:1004E000376501809306100493050000130505B0DD
:1004F000EF00C06C9304100003264400930720040F
:10050000630EF60037650180930620049305100002
:10051000130505B0EF00806A93841400032684005D
:1005200093073004630EF6003765018093063004AC
:1005300093052000130505B0EF0040689384140074
:100540000326C40093074004630EF600376501805C
:100550009306400493053000130505B0EF000066D4
:10056000938414008320C1000324810013850400B8
:100570008324410013010101678000003765018079
:10058000130101FF130545B7232611002324810021
:1005900023229100EF008062B7070080130740001C
:1005A0009387C70E6B10F700F32730CC3784018098
:1005B0001304C4A513972700938617043307E40098
:1005C0002320D70093B717006B8007000326040091
:1005D0009307100493040000630EF6003765018052
:1005E0009306100493050000130505B0EF00005DAD
:1005F000930410000326440093072004630EF600C2
:10060000376501809306200493051000130505B09B
:10061000EF00C05A9384140003268400930730042B
:10062000630EF600376501809306300493052000C1
:10063000130505B0EF008058938414000326C4000E
:1006400093074004630EF60037650180930640046B
:1006500093053000130505B0EF0040569384140055
:100660008320C100032481001385040083244100FA
:10067000130101016780000037650180130101FF4C
:10068000130545B82326110023248100232291005D
:10069000EF00C052930740006B800700F32700CCA7
:1006A00013B727006B20070013071000637AF70EBB
:1006B00013B737006B200700378401801307200031
:1006C0001304C49D6388E70C93972700B307F400D5
:1006D0001307400423A0E7006B3000006B300000DC
:1006E000930710006B800700032604009307100493
:1006F00093040000630EF600376501809306100432
:1007000093050000130505B0EF00404B9304100063
:100710000326440093072004630EF600376501802A
:100720009306200493051000130505B0EF0000495F
:10073000938414000326840093073004630EF600AC
:10074000376501809306300493052000130505B03A
:10075000EF00C046938414000326C40093074004AE
:10076000630EF60037650180930640049305300060
:10077000130505B0EF008044938414008320C1006A
:100780000324810013850400832441001301010127
:1007900067800000930730042324F4006FF0DFF338
:1007A00013C717006B200700378401801304C49D12
:1007B00063980700930710042320F4006FF0DFF123
:1007C000930720042322F4006FF01FF1130101FEB0
:1007D000232C8100232A910037840180B784018073
:1007E000376501809384C4A21304C4A093058000DC
:1007F000130505BA232E110023282101232491007B
:1008000023268100EF00803B9307200423A2F400FD
:100810009307300423A4F4009307400423A6F400B4
:100820009307500423A8F4009307600423AAF4005C
:10083000B70500809307700423ACF4001306810011
:100840009307800413091004938545111305800054
:1008500023A0240123AEF400EF00C04703260400C8
:1008600093040000630E260137650180930610048F
:1008700093050000130505B0EF0040349304100009
:100880000326440093072004630EF60037650180B9
:100890009306200493051000130505B0EF00003205
:1008A000938414000326840093073004630EF6003B
:1008B000376501809306300493052000130505B0C9
:1008C000EF00C02F938414000326C4009307400454
:1008D000630EF600376501809306400493053000EF
:1008E000130505B0EF00802D938414000326040146
:1008F00093075004630EF600376501809306500499
:1009000093054000130505B0EF00402B93841400BD
:100910000326440193076004630EF60037650180E7
:100920009306600493055000130505B0EF000029FD
:10093000938414000326840193077004630EF60069
:10094000376501809306700493056000130505B0B8
:10095000EF00C026938414000326C401930780048B
:10096000630EF600376501809306800493057000DE
:10097000130505B0EF008024938414008320C10187
:10098000032481010329010113850400832441010B
:100990001301010267800000630605009301050052
:1009A00073000000EF00004F130500006B0005000E
:1009B000732500FC6B00050097710100938101E530
:1009C00017F1FF7E1301016493050040732610CCDC
:1009D000B385C5023301B140F32630CC63860600EF
:1009E000130500006B000500678000001305F0FF91
:1009F000678000001305F0FF67800000130500000A
:100A00006780000013050000678000001305F0FFF9
:100A1000678000001305000067800000130101FFDC
:100A20002320210123261100232481002322910069
:100A300013090600635EC00013840500B384C5007B
:100A40000345040013041400EF00C012E31A94FEDF
:100A50008320C10003248100832441001305090081
:100A60000329010013010101678000001305F0FF55
:100A700067800000732540F167800000130101FFCB
:100A800023248100232021013774018037790180DC
:100A900093070400130909003309F94023261100C4
:100AA0002322910013592940630009021304040012
:100AB000930400008327040093841400130444006B
:100AC000E7800700E31899FE3774018037790180C9
:100AD00093070400130949003309F94013592940C9
:100AE0006300090213040400930400008327040038
:100AF0009384140013044400E7800700E31899FE70
:100B00008320C100032481008324410003290100C4
:100B10001301010167800000130101FF23248100FC
:100B2000B77701803774018013044400938747002E
:100B3000B3878740232291002326110093D42740B6
:100B4000638004029387C7FF3384870083270400F0
:100B50009384F4FF1304C4FFE7800700E39804FEC6
:100B60008320C1000324810083244100130101017B
:100B700067800000F32220CC93F2F203130300FC01
:100B8000B38262002380A20067800000130101FF8E
:100B900023248100138405000325040083A5450058
:100BA00023261100EF0080628320C1002324A400CB
:100BB000032481001301010167800000130101FC7F
:100BC00013030500371500802322B102232AF10206
:100BD0001305C5B89307410293054100232E110068
:100BE0002324C1022326D1022328E102232C01035E
:100BF000232E11032320F100232261002324F1007E
:100C0000EF00C0218320C1010325C10013010104AD
:100C100067800000130101FE232E1100232C8100A8
:100C2000232A91002328210123263101F32700FCE8
:100C30006B800700F32650CCF32930CC732700CC0F
:100C4000732600FCB787018093962600938747A9F7
:100C5000B387D70083A4070003A4040183A6C400BC
:100C600033A98900930704003309D900338436037C
:100C700063D4F900938709003304F40083A6840049
:100C80003304C402B307E9023304D4003304F4008C
:100C900033098900635E240183A7040083A544000F
:100CA0001305040013041400E7800700E31689FE0F
:100CB00093B919006B8009008320C10103248101CD
:100CC00083244101032901018329C1001301010289
:100CD00067800000130101FC232E1102232C8102E6
:100CE000232A91022328210323263103F32620FC03
:100CF000732810FC732400FCF32750CC1307F00179
:100D00006344F70CB30804031307100063D4A8006E
:100D10003347150363C8E60C63D8E70A9386F6FFEA
:100D20003343E502930803006396F6003365E5025A
:100D3000B3086500B3C4880233E9880263CA040BB0
:100D40009306100033C704036306070093060700E9
:100D500033E70403B7890180938949A9232EE10071
:100D60001307C1002326B1002328C100232CD10082
:100D70003303F30293972700B387F90023A0E7001A
:100D8000232A6100634C90066300090433848402C3
:100D9000232A81006B000900F32750CC732520CC57
:100DA00093972700B389F90083A7090083A68700DA
:100DB00003A7070083A547003305D500E700070018
:100DC000930710006B8007008320C1030324810375
:100DD00083244103032901038329C1021301010470
:100DE0006780000013870600E3CAE7F26FF0DFFDBB
:100DF00013070000930610006FF0DFF5138704005F
:100E00006354980013070800B7170080938747C101
:100E10006B10F700EFF01FE06FF01FF7130181FE7A
:100E2000232A1100232841012326310123242101F3
:100E30002322910023208100130A050093890500D5
:100E4000732900FCF32400CC13040000B302944087
:100E5000B33250006BA00200639802001305040037
:100E600093850900E7000A006B30000013041400AA
:100E7000E34E24FD83204101032A01018329C1009F
:100E8000032981008324410003240100130181010F
:100E900067800000F32750CC3707FF00B387E700D7
:100EA00093978700732700B023A0E700732710B043
:100EB00023A2E700732720B023A4E700732730B0F4
:100EC00023A6E700732740B023A8E700732750B09C
:100ED00023AAE700732760B023ACE700732770B044
:100EE00023AEE700732780B023A0E702732790B0FA
:100EF00023A2E7027327A0B023A4E7027327B0B0B0
:100F000023A6E7027327C0B023A8E7027327D0B057
:100F100023AAE7027327E0B023ACE7027327F0B0FF
:100F200023AEE702732700B123A0E704732710B1B3
:100F300023A2E704732720B123A4E704732730B169
:100F400023A6E704732740B123A8E704732750B111
:100F500023AAE704732760B123ACE704732770B1B9
:100F600023AEE704732780B123A0E706732790B16F
:100F700023A2E7067327A0B123A4E7067327B0B125
:100F800023A6E7067327C0B123A8E7067327D0B1CD
:100F900023AAE7067327E0B123ACE7067327F0B175
:100FA00023AEE706732700B823A0E708732710B81D
:100FB00023A2E708732720B823A4E708732730B8D3
:100FC00023A6E708732740B823A8E708732750B87B
:100FD00023AAE708732760B823ACE708732770B823
:100FE00023AEE708732780B823A0E70A732790B8D9
:100FF00023A2E70A7327A0B823A4E70A7327B0B88F
:1010000023A6E70A7327C0B823A8E70A7327D0B836
:1010100023AAE70A7327E0B823ACE70A7327F0B8DE
:1010200023AEE70A732700B923A0E70C732710B992
:1010300023A2E70C732720B923A4E70C732730B948
:1010400023A6E70C732740B923A8E70C732750B9F0
:1010500023AAE70C732760B923ACE70C732770B998
:1010600023AEE70C732780B923A0E70E732790B94E
:1010700023A2E70E7327A0B923A4E70E7327B0B904
:1010800023A6E70E7327C0B923A8E70E7327D0B9AC
:1010900023AAE70E7327E0B923ACE70E7327F0B954
:1010A00023AEE70E6780000093050500930600005D
:1010B00013060000130500006F004014130101FF28
:1010C000930500002324810023261100130405004A
:1010D000EF00801CB787018003A5079C8327C50309
:1010E00063840700E780070013050400EFF0DF8A40
:1010F0001303F00013070500637EC3029377F70024
:101100006390070A63920508937606FF1376F6004C
:10111000B386E6002320B7002322B7002324B700BC
:101120002326B70013070701E366D7FE6314060002
:1011300067800000B306C340939626009702000024
:10114000B38656006780C6002307B700A306B70022
:101150002306B700A305B7002305B700A304B70013
:101160002304B700A303B7002303B700A302B7000B
:101170002302B700A301B7002301B700A300B70003
:101180002300B7006780000093F5F50F9396850064
:10119000B3E5D50093960501B3E5D5006FF0DFF612
:1011A0009396270097020000B386560093820000B2
:1011B000E78006FA93800200938707FF3307F74022
:1011C0003306F600E378C3F66FF0DFF3B7870180EC
:1011D00083A7479C938605001306050083A5870017
:1011E000138507006F00801D938705008325850008
:1011F00093060600138607006F00401CB787018026
:1012000003A7079C83278714638C070403A7470061
:101210001308F001634EE806131827006306050261
:10122000338307012324C30883A8871813061000FB
:101230003316E600B3E8C80023A417192324D310FB
:10124000930620006304D5021307170023A2E700CA
:10125000B387070123A4B7001305000067800000CF
:101260009307C7142324F7146FF05FFA83A6C718F7
:101270001307170023A2E70033E6C60023A6C7180A
:10128000B387070123A4B70013050000678000009F
:101290001305F0FF67800000130101FDB78701808F
:1012A000232C410103AA079C23202103232611029A
:1012B00003298A142324810223229102232E31013F
:1012C000232A51012328610123267101232481014E
:1012D00063000904130B0500938B0500930A1000AB
:1012E0009309F0FF832449001384F4FF634204024E
:1012F00093942400B304990063840B0483A74410DF
:10130000638077051304F4FF9384C4FFE31634FF6E
:101310008320C102032481028324410203290102A4
:101320008329C101032A8101832A4101032B010181
:10133000832BC100032C810013010103678000008F
:101340008327490083A644009387F7FF638E8704B1
:1013500023A20400E38806FA8327891833978A00BA
:10136000032C4900B377F70063920702E780060079
:101370000327490083278A1463148701E304F9F8DB
:10138000E38807F8138907006FF0DFF58327C91892
:1013900083A544083377F700631C070013050B008F
:1013A000E78006006FF0DFFC232289006FF09FFAD0
:1013B00013850500E78006006FF09FFB130101E134
:1013C0002326111E232A511D2328611D2320A11D20
:1013D000938A0500130D06002326D1002324811EC5
:1013E0002322911E2320211F232E311D232C411D3A
:1013F0002326711D2324811D2322911D232EB11B21
:10140000130B0500EF60404D83270500138507008F
:101410002320F104EF80404B232EA1022328010E4C
:10142000232A010E232C010E232E010E63060B002E
:1014300083278B03E38A072A8396CA0093970601C2
:101440001397260193D70701634A0702B7270000C5
:1014500003A64A06B3E7F60093970701B7E6FFFF36
:1014600093D707419386F6FFB376D6002396FA000A
:101470009397070123A2DA0693D7070193F6870013
:101480006380062E83A60A01638C062C93F7A701BE
:101490009306A0006388D72EB7670180938787BF24
:1014A000232AF10083470D00930BC110B769018017
:1014B0002322710F2326010E2324010E232801006D
:1014C000232C010023220104232C010223240104E4
:1014D000232601042322010093880B00938949D716
:1014E0006382072213040D00930650026388D740DD
:1014F0008347140013041400E39A07FEB304A441C5
:101500006302A4218326C10E8327810E23A0A80194
:10151000B38696009387170023A298002326D10E46
:101520002324F10E930670009388880063C0F63E72
:101530000327410083470400330797002322E1007B
:101540006382071C83441400A303010C13041400DA
:101550001303F0FF130A000013090000130CA00589
:10156000930C9000930DA00213041400938704FEC3
:101570006364FC040327410193972700B387E700C6
:1015800083A7070067800700130A0000938704FD04
:101590008344040093162A00338A4601131A1A0062
:1015A000338A4701938704FD13041400E3F2FCFE21
:1015B000938704FEE370FCFC6386041423069114F5
:1015C000A303010C130C1000930C1000130DC11495
:1015D000930D00001303000023260102232A0102B9
:1015E00023280102937F290063840F00130C2C0031
:1015F000137F49088327C10E63180F0033088A41FF
:10160000635400016F00D07C8346710C638A06022C
:101610008326810E1306710C23A0C8009387170040
:10162000130610009386160023A2C8002326F10E8D
:101630002324D10E13067000938888006342D6627B
:10164000638C0F028326810E1306810C23A0C80031
:1016500093872700130620009386160023A2C80054
:101660002326F10E2324D10E1306700093888800E0
:101670006354D6006F10C00593060008E30ADF46E6
:1016800033039341E340605493760910E3960632A6
:101690000327810EB387970123A0A8011307170022
:1016A00023A298012326F10E2324E10E9306700055
:1016B00063C4E666938888001379490063060900CD
:1016C000B3048A41634A906663548A01130A0C008A
:1016D00003274100330747012322E100E392075A21
:1016E0002324010E63880D0093850D0013050B0064
:1016F000EF30401D93880B00130D040083470D004D
:10170000E39207DE8327C10E638407006F10D03891
:1017100083D7CA0093F70704638407006F2040292A
:101720008320C11E0324811E032541008324411E02
:101730000329011E8329C11D032A811D832A411DFE
:10174000032B011D832BC11C032C811C832C411CEA
:10175000032D011C832DC11B1301011F6780000095
:1017600093850A0013050B00EF20D00663040500E3
:101770006F20002483D7CA009306A00093F7A70127
:10178000E39CD7D08397EA00E3C807D08326C10043
:1017900013060D0093850A0013050B00EF208077D8
:1017A0002322A1006FF0DFF713050B00232E110198
:1017B00023246100EF604012832745001385070052
:1017C0002326F104EF8040109307050013050B005A
:1017D000938407002324F104EF6000108327850021
:1017E000032381008328C101232CF10263840400B8
:1017F0006F100018834404006FF01FD78344040067
:10180000136909026FF05FD6136909019377090222
:10181000638807608327C1009387770093F787FF6A
:1018200003A7470083AD0700938787002326F100B5
:10183000930C0700634007621307F0FF130C0900C5
:101840006300E37633E79D01137CF9F7631A0774AD
:10185000631E037413090C0013030000930C0000B3
:10186000130D011B138C0C0063D46C00130C0300CC
:101870008347710C23260102232A01022328010237
:10188000930D0000E38007D6130C1C006FF09FD56A
:101890001369090193770902638C07548327C100F8
:1018A00013877700137787FF832D0700832C47006A
:1018B000930787002326F100137CF9BF130700006C
:1018C000A303010C9306F0FF630AD35AB3E69D010C
:1018D0001379FCF7E39A064EE3120308E31E07F6BA
:1018E000937C1C00130D011BE38E0CF69307000381
:1018F000A307F11A130DF11A6FF0DFF6B304A44138
:10190000E312A4C1834704006FF09FC31306410E86
:1019100093850A0013050B00EFA0D049E31A05DEFA
:1019200093880B006FF0DFC0937789006394070002
:101930006F10C0080327C100832707001307470063
:101940002326E10083A5070003A6470083A687009E
:1019500083A7C7002328B10E232AC10E232CD10E42
:10196000232EF10E1305010F232E110123246100F4
:10197000EF50D06F2326A10C930720000323810092
:101980008328C1016314F5006F100048930710000D
:101990006314F5006F10C05C930710066394F400A5
:1019A0006F204018930710046394F4006F10101018
:1019B00093FCF4FD9307F0FF232891076314F300D1
:1019C0006F204017930770046394FC006F2000178A
:1019D000032EC10F23242107832E010F032F410F54
:1019E000832F810F9367091063540E006F204039D5
:1019F000232E010613890700930D0000930760044E
:101A00006394FC006F109062930750042324110329
:101A10006384FC006F101059930C1300130C010B1E
:101A20001308C10D93860C009307010D1307C10C19
:101A30001306200093050C0013050B0023226102FE
:101A40002328D10B2320D103232AE10B232EE101EC
:101A5000232CF10B2328F101232EC10B2324C101D8
:101A6000EF409034032E8100832F0101032FC10129
:101A7000832E01020323410283288102330895014A
:101A8000130D0500930C010A93850C0013050C003F
:101A9000232E010123281101232461002328D10BC7
:101AA000232AE10B232CF10B232EC10B2320010A47
:101AB0002322010A2324010A2326010AEF00C1463A
:101AC0000328C10103238100832801019307080033
:101AD000630205028327C10D63FE0701130600039D
:101AE00093861700232ED10C2380C7008327C10DB6
:101AF000E3E807FF0327C10CB387A7412328F100C0
:101B00002328E10203270107930770046314F700F9
:101B10006F10903A03270107930760046314F700DE
:101B20006F10D06383270103032701079305100477
:101B30009387F7FF2326F10C93F6F40F13060000AA
:101B40006318B7009386F60093F6F60F130610009D
:101B5000230AD10C9306B00263DA070003270103BE
:101B6000930710009306D002B387E740A30AD10C75
:101B70009306900063C4F6006F2040211308310ED5
:101B8000130508001306A000130E3006B3E6C702C3
:101B900093050500138307001305F5FF93860603DD
:101BA000A38FD5FEB3C7C702E3426EFE9387070338
:101BB00013F6F70FA30FC5FE9387E5FF63E4070154
:101BC0006F20C0329306610D6F00800003C60700CE
:101BD0002380C6009387170093861600E39807FFBB
:101BE0009307510EB387B7401307610DB307F70092
:101BF0009306410DB387D7402322F1040327010147
:101C00008326410493071000B30CD70063C4E70098
:101C10006F2080258327C103B38CFC0083278106B6
:101C200013CCFCFF135CFC4113F9F7BF13690910D7
:101C300033FC8C0123260102232A010223280102FE
:101C40008327C107639407006F10502E9307D002BB
:101C5000A303F10C13030000130C1C006FF09F98FA
:101C60001306410E93850A0013050B002320610221
:101C7000232EE1012324F101EFA0D013E31C050082
:101C80008327C10E03230102032FC101832F81008B
:101C900093880B006FF0DF9A832601040327C103AA
:101CA0001306700023A0D8008326810EB307F70027
:101CB00023A2E800938616002326F10E2324D10EDA
:101CC000938888006354D6021306410E93850A0058
:101CD00013050B00EFA0100E631E057A8325C10CBF
:101CE0008327C10E8326810E93880B0063D40500E1
:101CF0006F10904D032701019386160023A0A801C1
:101D0000B307F70023A2E8002326F10E2324D10E07
:101D100013077000E350D79A1306410E93850A000B
:101D200013050B00EFA01009631605768327C10E7B
:101D300093880B006FF05F98930600010327810ED4
:101D400063C496006F109047B7660180938E46D6A5
:101D500013090001930C70006F00C000938404FF0E
:101D6000635A9904938707011307170023A0D8012A
:101D700023A228012326F10E2324E10E9388880054
:101D8000E3DEECFC1306410E93850A0013050B00FD
:101D90002324D101EFA01002631E056E938404FF7B
:101DA0008327C10E0327810E832E810093880B00A9
:101DB000E34A99FAB38797001307170023A0D801C5
:101DC00023A298002326F10E2324E10E930670002F
:101DD000E3DCE68E1306410E93850A0013050B0023
:101DE000EFA0407D6318056A8327C10E6FF0DF8D79
:101DF0008326C1009377090113874600E39C0740BF
:101E000093770904639407006F1000108327C100C3
:101E1000930C00002326E10083DD07006FF0DFA9AB
:101E20008326C1009377090113874600E39E073696
:101E300093770904639407006F1080108327C10013
:101E40002326E100839D070093DCFD4113870C00EE
:101E5000E354079E3337B001B3079041B38CE7409A
:101E60001307D002A303E10C9306F0FFB30DB041BA
:101E7000130C090013071000E31AD3A493061000F3
:101E80006300D712930620006306D72E130D011BA3
:101E90001396DC0193F67D0093DD3D0093860603E7
:101EA000B36DB60193DC3C00A30FDDFE33E69D016C
:101EB00093050D00130DFDFFE31C06FC93771C003A
:101EC0006384072E930700036380F62E9385E5FF56
:101ED000A30FFDFE9307011BB38CB74013090C0041
:101EE000138D05006FF01F9813050B00EF201005F0
:101EF0006FF08FD40327C100A303010C130C100053
:101F000083270700130747002326E1002306F11467
:101F1000930C1000130DC1146FF08FEB8327C100D9
:101F2000A303010C03AD070093864700E3040D40B3
:101F30009307F0FFE306F376130603009305000012
:101F400013050D00232ED100232611012324610047
:101F5000EF608034032381008328C1008326C10100
:101F6000930D0500631405006F109018B30CA54184
:101F70008347710C13CCFCFF135CFC412326D1007A
:101F800023260102232A01022328010233FC8C01AB
:101F9000930D000013030000E398078E6FF08FE4A9
:101FA000E3920C4813079000E36EB747938D0D033F
:101FB000A307B11B13090C00930C1000130DF11AA9
:101FC0006FF05F8A83440400136949006FF0CFD932
:101FD0009307B00283440400A303F10C6FF0CFD841
:101FE00083440400136909086FF00FD88344040088
:101FF000930614006394B4016F10106C938704FD72
:10200000138406001303000063E2FCD6834404003B
:102010009316230033836600131313003303F30076
:10202000938704FD13041400E3F2FCFE6FF00FD459
:102030008327C1008344040003AA07009387470055
:102040002326F10063520AD2330A40411369490042
:102050006FF08FD183440400136919006FF0CFD063
:102060008347710C83440400639007D093070002F8
:10207000A303F10C6FF04FCF136C090193770C029F
:10208000E38C07088327C10013877700137787FF46
:1020900093078700832D0700832C47002326F10038
:1020A000130710006FF0DF81834404001369890077
:1020B0006FF08FCB8327C1003787FFFF134707835C
:1020C00083AD07002314E10C938747003767018035
:1020D0002326F100930747BC930C0000136C2900E2
:1020E000232CF10013072000930480076FF04FFDAD
:1020F0008326C1009377090203A706009386460052
:102100002326D100E39A070493770901E392075845
:1021100093770904638407006F10C01013790920B6
:10212000E308095683274100130D04002300F7003C
:102130006FF0CFDC834404009307C006E38CF41AED
:10214000136909016FF04FC28344040093078006AE
:10215000E38AF418136909046FF00FC193061000A5
:102160006314D7006F10901193062000130C090020
:10217000E31ED7D0130D011B8327810193F6FD00C9
:1021800093DD4D00B386D70003C606009396CC01BD
:10219000B3EDB60193DC4C00A30FCDFEB3E69D0179
:1021A000130DFDFFE39A06FC9307011BB38CA741B7
:1021B00013090C006FF00FEB9306500663D6962EB2
:1021C0008326010F9305010A1305010B2328D10A69
:1021D0008326410F232EF10023241101232AD10A43
:1021E0008326810F2320010A2322010A232CD10AEE
:1021F0008326C10F2324010A2326010A232ED10A94
:10220000EFF09052832881008327C101631A054EA5
:102210000327810EB7660180938646BF23A0D800AE
:1022200093871700930610001307170023A2D80006
:102230002326F10E2324E10E930670009388880074
:10224000E3C0E6380327C10C83260101635ED76E25
:10225000032701048326C1039388880023ACE8FE8A
:102260000327810EB387D70023AED8FE13071700CC
:102270002326F10E2324E10E93067000E3CCE6083A
:10228000032701019304F7FF635890C293060001EE
:102290000327810EE3D69634930C0001130D7000D2
:1022A0006F00C000938404FFE3DC9C329387070136
:1022B0001307170023A0380123A298012326F10E4B
:1022C0002324E10E93888800E35EEDFC1306410EA3
:1022D00093850A0013050B00EFA0C02D631C051A9F
:1022E0008327C10E0327810E93880B006FF09FFB9D
:1022F00033088A41635600B9130600018326810E14
:10230000635C0607130E0001930E70006F00C0009F
:10231000130808FF63520E07938707019386160080
:1023200023A0380123A2C8012326F10E2324D10EB5
:1023300093888800E3DEDEFC1306410E93850A00D5
:1023400013050B00232E010123246100EFA080263A
:10235000631205140328C101130E00018327C10E67
:10236000130808FF8326810E0323810093880B0046
:10237000930E7000E3420EFBB387070193861600AD
:1023800023A0380123A208012326F10E2324D10E15
:1023900013067000938888006354D6AE1306410E6E
:1023A00093850A0013050B0023246100EFA0802011
:1023B0006312050E8327C10E0323810093880B004F
:1023C0006FF00FAC130600018326810E635866067A
:1023D00013080001130E70006F00C000130303FF09
:1023E000635E6804938707019386160023A0380173
:1023F00023A208012326F10E2324D10E93888800FE
:10240000E35EDEFC1306410E93850A0013050B0004
:1024100023246100EFA0001A631E05060323810038
:10242000130800018327C10E130303FF8326810EC7
:1024300093880B00130E7000E34668FAB3876700B9
:102440009386160023A0380123A268002326F10EEC
:102450002324D10E13067000938888006356D6A2F9
:102460001306410E93850A0013050B00EFA080149C
:10247000631205028327C10E93880B006FF0CFA073
:102480001306410E93850A0013050B00EFA080127E
:10249000630805A4638E0DA693850D0013050B003C
:1024A000EF2040426FF0CFA60326810E03270101E3
:1024B0009306100023A0A801938717009304160029
:1024C000938C880063DCE63A9306100023A2D800C0
:1024D0002326F10E2324910E9306700063C096709C
:1024E0000327C1038326010493841400B387E70004
:1024F00023A0DC0023A2EC002326F10E2324910E5E
:1025000093067000938C8C0063CC966E8326010F2B
:10251000138814009305010A2328D10A8326410F4A
:102520001305010B232EF100232AD10A8326810FE4
:10253000232401012320010A232CD10A8326C10F61
:102540002322010A2324010A232ED10A2326010A69
:10255000EFF0901D832701010328810093888C00F0
:102560009386F7FF130608008327C101630C053229
:1025700013071D00B387D70023A0EC0023A2DC00C3
:102580002326F10E2324010F130770006344074D27
:1025900013870C0113862400938C0800930807000E
:1025A000832641041307410D23A0EC00B387F600F6
:1025B00023A2DC002326F10E2324C10E1307700092
:1025C000635CC78E6FF04FF5130C09006FF01F8B23
:1025D00037670180130600018326810E930E47D6CC
:1025E000130E000193027000634806016F0040085B
:1025F000130808FF635E0E07938707019386160092
:1026000023A0D80123A2C8012326F10E2324D10E32
:1026100093888800E3DED2FC1306410E93850A00FE
:1026200013050B002324D10323220103232061027D
:10263000232EE1012324F101EF90D077E31C05E480
:1026400003284102130E00018327C10E130808FF5F
:102650008326810E832E810203230102032FC101F1
:10266000832F810093880B0093027000E3460EF9DC
:10267000B38707019386160023A0D80123A208017F
:102680002326F10E2324D10E1306700093888800B0
:102690006344D6006FE05FF71306410E93850A008E
:1026A00013050B0023206102232EE1012324F101F5
:1026B000EF905070E31005DE8327C10E0323010263
:1026C000032FC101832F810093880B006FE0DFF39C
:1026D0001306410E93850A0013050B00232E61009B
:1026E0002324E101EF90106DE31605DA8327C10E74
:1026F0000323C101032F810093880B006FE0DFF7F4
:102700008325C10C635CB0600327010383260101AC
:102710009304070063C8E630635690028326810E57
:10272000B387970023A0A8019386160023A29800E0
:102730002326F10E2324D10E1306700093888800FF
:10274000E34ED62893C6F4FF0327010393D6F64140
:10275000B3F4D400B3049740634E903E03270103C3
:1027600093760940B304ED00E39E06048325C10C73
:102770000327010163C6E50093761900E384062868
:10278000832601040327C1031306700023A0D80089
:102790008326810EB387E70023A2E8009386160004
:1027A0002326F10E2324D10E938888006354D6008B
:1027B0006F10C010832601013307DD003386B64059
:1027C00033079740930C06006354C700930C07002F
:1027D000635890030327810EB387970123A09800C5
:1027E0001307170023A298012326F10E2324E10EDC
:1027F000930670009388880063D4E6006F10401839
:1028000013C7FCFF1357F74133F7EC00B304E6405E
:10281000634490006FE05FEA930600010327810E96
:1028200063D0965C930C0001130D70006F00C00024
:10283000938404FF63D69C5A9387070113071700FC
:1028400023A0380123A298012326F10E2324E10EB0
:1028500093888800E35EEDFC1306410E93850A0021
:1028600013050B00EF901055E31605C28327C10E28
:102870000327810E93880B006FF09FFB937519005F
:10288000E39405C423A2D8002326F10E2324910E3D
:10289000130770006340971C1306260093880801F5
:1028A0006FF01FD0E35ED0CE130700016344D70062
:1028B0006F10C05C130D70006F000001938606FF5F
:1028C0006358D716138814009387070123A03C018F
:1028D00023A2EC002326F10E2324010F9304080009
:1028E000938C8C00E35C0DFD1306410E93850A006A
:1028F00013050B002324D100EF90D04BE31C05B847
:102900008327C10E8324810E83268100938C0B00C4
:10291000130700016FF09FFA8326C10093770C0123
:10292000138746006398070693770C04638E075A53
:102930008327C100930C00002326E10083DD0700FC
:10294000130710006FE0DFF7137719006314070017
:102950006FE09FD66FF0DF8F83264100130D0400D8
:1029600093D7F6412320D7002322F7006FE01FD929
:102970008327810383440400639407006FE0DFBE74
:1029800083C70700639407006FE01FBE1369094007
:102990006FE09FBD2326E10083AD0600930C00008D
:1029A000130710006FE0DFF183AD06002326E1007E
:1029B00093DCFD4113870C006FE0DFE78327C10044
:1029C0001305010B232E11019387770093F787FFDF
:1029D00083A5070003A6470093878700232461008F
:1029E0002326F100EF20511A8327010B8328C10110
:1029F000032381002328F10E8327410B232AF10EA4
:102A00008327810B232CF10E8327C10B232EF10E7C
:102A10006FE05FF583AD0600930C00002326E10014
:102A20006FE09FE993840600E34A90CE6FF09FD158
:102A30001386140013878C00B387D70023A2DC0011
:102A400023A03C012326F10E2324C10E930670001F
:102A500063D6C6741306410E93850A0013050B0056
:102A6000EF905035E31805A20326810E8327C10E8F
:102A70009308411113061600938C0B006FF05FB2A0
:102A8000130C09006FF08FDFB7670180938747BC95
:102A9000232CF10093770902638207128327C10078
:102AA00013877700137787FF832D0700832C470058
:102AB000930787002326F10013771900630E0700A0
:102AC00033E79D01630A0700130700032304E10CA9
:102AD000A304910C13692900137CF9BF130720008C
:102AE0006FE01FDE834414001369092013041400EF
:102AF0006FE09FA7834414001369090213041400B4
:102B00006FE09FA6B7670180938787BD232CF100F4
:102B10006FF05FF81306410E93850A0013050B0052
:102B2000EF905029E31805968327C10E93880B0078
:102B30006FF00FF593076000930C030063E0676C80
:102B400037670180138C0C002326D100130DC7BEFC
:102B50006FE01FA8130600018326810E6352964280
:102B6000930C0001130870006F00C000938404FFF1
:102B700063D89C40938707019386160023A03801F1
:102B800023A298012326F10E2324D10E93888800D6
:102B9000E35ED8FC1306410E93850A0013050B0073
:102BA000EF905021E318058E8327C10E8326810EF6
:102BB00093880B00130870006FF05FFB8326C10041
:102BC0009377090113874600638E071C83AD0600C7
:102BD000930C00002326E1006FF01FEE1306410E58
:102BE00093850A0013050B00EF90D01CE314058AAF
:102BF0008327C10E8324810E938C0B006FF05F8EB0
:102C00001306410E93850A0013050B00EF90901AEE
:102C1000E31205888327C10E8324810E938C0B0059
:102C20006FF0DF8E13790C4023280100130D011B78
:102C30006F0040031306A0009306000013850D00EB
:102C400093850C00232E110123246100EFD0102363
:102C5000032381008328C101E3840C2E930D05001A
:102C6000938C05001306A0009306000013850D0049
:102C700093850C00232E110123246100EFD05063B3
:102C80008327010113050503A30FADFE93871700EA
:102C90002328F100032381008328C101130DFDFFC8
:102CA000E30A09F80327810383460700E394D7F872
:102CB0001307F00FE380E7F863960C00930790008A
:102CC00063F4B7CF832781048325C104232E110128
:102CD000330DFD401386070013050D00232461000A
:102CE000EF605047832781031306A000930600007E
:102CF00003CE170013850D0093850C00333EC001F1
:102D0000B387C701232CF102EFD0501703238100B2
:102D10008328C101232801006FF05FF48326810E10
:102D200037660180130646BF23A0C80093871700AB
:102D3000130610009386160023A2C8002326F10E66
:102D40002324D10E13067000938888006340D64672
:102D5000638405006FE05FF4032701019376190097
:102D6000B3E6E600639406006FE01F958326010436
:102D70000327C1031306700023A0D8008326810E09
:102D8000B307F70023A2E800938616002326F10E6E
:102D90002324D10E6354D6006FE01FF3938888007C
:102DA0006FE05FF593770904638E07168327C100F0
:102DB000930C00002326E10083DD07006FF0DFCFD6
:102DC0001306410E93850A0013050B00EF90807ED9
:102DD000631205EC8327C10E93880B006FF08FC63A
:102DE00023A0380123A29800B38797001307170088
:102DF0002326F10E2324E10E9306700063C4E6003F
:102E00006FE05F8B6FE05FF18327010F9305010A8D
:102E10001305010B2328F10A8327410F23241101F5
:102E20002320010A232AF10A8327810F2322010A82
:102E30002324010A232CF10A8327C10F2326010A28
:102E4000232EF10AEFF0C03583288100E34C0528DA
:102E50008347710C13077004635C973637670180F2
:102E6000130D87BB23260102232A01022328010216
:102E70001379F9F7130C3000930D0000930C300018
:102E800013030000638407006FE01FA06FE08FF55D
:102E900083274100130D04002320F7006FE01F86F5
:102EA00013050D00232411012326D100EF60D0214A
:102EB0008347710C134CF5FF135CFC412326010280
:102EC000232A01022328010283288100930C050094
:102ED000337C8501930D0000130300006384070019
:102EE0006FE09F9A6FE00FF093770C2063840738B0
:102EF0008327C100930C00002326E10083CD070047
:102F0000130710006FE0DF9B93770920638A073473
:102F10008327C100930C00002326E10083CD070026
:102F20006FE09F9993770920638207328327C1005E
:102F3000930C00002326E10083CD07006FF0DFB77C
:102F4000937709206388072E8327C1002326E10099
:102F5000838D070093DCFD4113870C006FE09F8D8C
:102F60008327C10F63C407328347710C13077004B2
:102F7000E356971A37670180130D07BC6FF09FEE79
:102F8000B38797009386160023A0380123A29800E8
:102F90002326F10E2324D10E130670009388880097
:102FA000635ED6FA1306410E93850A0013050B00E3
:102FB000EF904060631005CE8327C10E93880B000D
:102FC0006FF0CFF903270101130E70001308000101
:102FD0003307ED002324E10003274103630E070AB2
:102FE0000327C102631E070A032781031307F7FFA4
:102FF000232CE102032741031307F7FF232AE102F1
:103000008326C104032781049388880023ACD8FE5B
:103010008326810EB387E70023AEE8FE9386160071
:103020002326F10E2324D10E634EDE1003278103E5
:103030008346070003278100938C060033069740E0
:103040006354D600930C0600635890038326810EC8
:10305000B387970123A098009386160023A29801B6
:103060002326F10E2324D10E6342DE1003278103B1
:10307000938888008346070013C6FCFF1356F64169
:10308000B3FCCC00B38C964163449003B384D4006A
:1030900003274103E31607F40327C1026304076013
:1030A0000327C1021307F7FF2326E1026FF05FF544
:1030B0008326810E634898016F00C005938C0CFF36
:1030C000635A9805938707019386160023A0380159
:1030D00023A208012326F10E2324D10E9388880011
:1030E000E35EDEFC1306410E93850A0013050B0018
:1030F000EF90404C631005BA13080001938C0CFF4D
:103100008327C10E8326810E93880B00130E700057
:10311000E34A98FBB38797019386160023A03801F2
:1031200023A298012326F10E2324D10E6340DE64EE
:10313000032781039388880083460700B384D40063
:103140006FF01FF51306410E93850A0013050B005F
:10315000EF904046631005B48327C10E93880B009F
:1031600013080001130E70006FF05FEC1306410EA0
:1031700093850A0013050B00EF90C043631C05B054
:103180008327810393880B001308000183C607007F
:10319000130E70008327C10E6FF01FEE130616008A
:1031A00093088700930C07006FF08FBF1306410E42
:1031B00093850A0013050B00EF90C03F631C05AC1C
:1031C0008325C10C8327C10E93880B006FF05FB875
:1031D00037670180130D47BB6FF0DFC81306410E40
:1031E00093850A0013050B00EF90C03C631405AAF9
:1031F0008327C10E93880B006FF0CFD4930C60002F
:103200006FF01F94832601013307DD003386B6403B
:1032100033039740930C06006354C3DE930C030002
:103220006FF00FDE83274100130D04002310F70019
:103230006FE0CFCC8327C1002326E10083AD0700D8
:1032400093DCFD4113870C006FE0CFDE8327C100C4
:10325000930C00002326E10083AD07006FF0DF85AB
:103260008327C100930C00002326E10083AD0700F3
:103270006FE08FE48327C100930C00002326E10058
:1032800083AD0700130710006FE08FE39307D002B0
:10329000A303F10C6FF09FCD1306410E93850A0036
:1032A00013050B00EF9000316FE08FC6930700030A
:1032B0002304F10C9307800513672900A304F10C84
:1032C0002324E10693073006930D0000130DC1146B
:1032D000E3C46702032EC10F93FCF4FD232891077A
:1032E000232E0106832E010F032F410F832F810F01
:1032F0001369291063420E4693071006E38AF416F9
:10330000930710046384F4006FE04FEF130C010B7C
:1033100013050C0023261103232461022328D10B5B
:10332000232AE10B232CF10B232EC10BEF20412884
:103330001306C10CEF6040191386050093050500C4
:1033400013050C00EF204104930701099385070042
:103350002324F1008327010B930C010A13060108B3
:103360002328F1088327410B13850C002326C1066F
:10337000232AF1088327810B232001082322010837
:10338000232CF1088327C10B23240108232EF108E5
:10339000B707FC3F2326F108EFE050750328010A28
:1033A000032E410A832E810A032FC10A93850C0044
:1033B00013050C002328010B23220103232AC10B30
:1033C0002320C103232CD10B232ED101232EE10B6B
:1033D0002328E1012320010A2322010A2324010AD0
:1033E0002326010AEFE05034032F0101832EC1018F
:1033F000032E010203284102032381028328C10214
:1034000063160500930710002326F10CB7670180AF
:10341000938787BD2322F1069306F3FF93070D00E0
:103420006F00C00893850C0013050C002320C10613
:10343000232EF105232C5104232A71042328F1049F
:103440002328710A23267102232A510A23245102B8
:10345000232CF10B2322F103232EC10A2320C102C6
:103460002320010A2322010A2324010A2326010A18
:10347000EFE0902B8326C101032F0102832E41022E
:10348000032E81020328C102032301038328410381
:10349000832701058323410583228105832FC105ED
:1034A000032601069386F6FF630E051003268100AE
:1034B00093850C002328F10413050C00B707034083
:1034C000232A1103232861022326D102232EF10887
:1034D0002326E10B2320010B2322C10B2324D10B34
:1034E00023280108232A0108232C0108EFE010609B
:1034F000832E010B032E410B0328810B0326C10BE6
:1035000013050C002324D1032322C103232001032C
:10351000232EC100EF109137930505002328A10049
:1035200013050C00EF1051510326C101832E8102B7
:10353000032E4102232EC1080326010B032801029A
:10354000832581002320C1080326410B13850C002D
:103550002328D1092322C1080326810B232AC1096C
:10356000232C01092324C1080326C10B2326C108EB
:103570000326C106EF000105032741068327010149
:103580008326C1028323010A3306F7008345060020
:10359000832701058322410A832F810A0326C10A5A
:1035A000232CF1062380B700232AD1061307F0FF4E
:1035B000232ED1000323010383284103938717009F
:1035C000E392E6E6B706FE3F93850C0013050C0078
:1035D0002320F102232E1101232461002328710AE4
:1035E00023287102232A510A23265102232CF10B8E
:1035F0002324F103232EC10A2322C1022320010A1E
:103600002322010A2324010A2326D10AEFE0902471
:10361000032381008328C101832701026344A0465C
:10362000832301038322C102832F810203264102E7
:10363000B706FE3F93850C0013050C002328710A82
:10364000232A510A232CF10B232EC10A2320010A1D
:103650002322010A2324010A2326D10AEFE0D00CF9
:10366000032381008328C101832701026318050019
:10367000032701019376170063960640032741074D
:103680001306000393061700B386D70063540700A0
:103690006FE04FC693871700A38FC7FEE39CF6FE2B
:1036A0006FE04FC503270101B306ED0063F0968C70
:1036B000938406006FF08F8B032701039307D0FFDD
:1036C0006344F700635AE3009384E4FF93F7F4FD47
:1036D0002328F1066FE00FC58327010103270103AB
:1036E0006344F72483278106930C070093F71700A0
:1036F000638607008327C103B30CF7008327810685
:1037000093F707406386070083270103634AF04C61
:1037100013CCFCFF135CFC4133FC8C01930470065A
:1037200023260102232A01026FE08FD18347710C07
:1037300013030000638407006FE00F956FD09FEACA
:103740009307900063ECB7D16FE01FA623242107F5
:10375000930D000013890200B707008033CEC70124
:103760009307D002232EF1066FF01FB91306410E06
:1037700093850A0013050B00EF80D06363040500F6
:103780006FE05FD18327810393880B00130800014A
:1037900083C60700130E70008327C10EB384D400C4
:1037A0006FF01F8F130C010B9307010D930603009D
:1037B0001308C10D1307C10C1306200093050C005C
:1037C00013050B00232261022328D10B2320D103F0
:1037D000232AE10B232EE101232CF10B2328F101F5
:1037E000232EC10B2324C101EF20105C930770042A
:1037F000032E8100832F0101032FC101832E0102BB
:103800000323410283288102130D05006394FC0801
:103810008327810693F717006396072C130770041C
:103820008327C10D2328E1066FE0CFAC130C010BF9
:10383000930603001308C10D9307010D1307C10C74
:103840001306300093050C0013050B00232411030D
:10385000232261022328D10B2320D103232AE10B49
:10386000232EE101232CF10B2328F101232EC10B80
:103870002324C101EF205053032E8100832F010127
:10388000032FC101832E01020323410283288102F9
:10389000130D05009307600433086D00639AFC2440
:1038A00083460D00930700036380F654930C010ACE
:1038B0008327C10C3308F8006FE00F9D1306410EFB
:1038C00093850A0013050B00EF80D04E63040500BA
:1038D0006FE05FBC8325C10C8327C10E93880B006A
:1038E0006FE05FED9307D002A303F10C6FF08FD66A
:1038F0008347710C2326D10023260102232A0102CB
:1039000023280102130C0300930C0300130300008F
:10391000638407006FD05FF76FD0DFCC376701801B
:10392000130DC7BB6FF00FD4832701010327C10319
:1039300093047006B38CE70083270103635AF048B1
:103940008327810693F70740639E072813CCFCFF6B
:10395000135CFC4133FC8C016FF09FDC83278106F4
:103960000327010393F71700B3E76700635CE05098
:1039700063960744832C0103930460066FF05FFC99
:103980001306410E93850A0013050B00EF80904249
:10399000630405006FE01FB08324C10C03270101FD
:1039A0008327C10E93880B00330697406FE05FE5D5
:1039B0009307F0FF2322F1006FD09FD6B7660180F6
:1039C000938E46D66FE00FBF130600FFB304B040DE
:1039D00063D2C506930C0001130870006F00C0008D
:1039E000938404FF63D89C04938707019386160091
:1039F00023A0380123A298012326F10E2324D10EFF
:103A000093888800E35ED8FC1306410E93850A0074
:103A100013050B00EF80103A630405006FE09FA7C9
:103A20008327C10E8326810E93880B001308700034
:103A30006FF01FFBB38797009386160023A0380111
:103A400023A298002326F10E2324D10E1306700022
:103A50006356D6B41306410E93850A0013050B0076
:103A6000EF805035630405006FE0DFA28327C10EAD
:103A70008326810E93880B006FE0CFA7130C0900FB
:103A80006FE0CFD20327810793860700232EE10C36
:103A90000327410603C6F7FF8345F7006310B6020C
:103AA00013050003A38FA6FE8326C10D1386F6FF20
:103AB000232EC10C03C6F6FFE386C5FE9305160050
:103AC0001305900393F5F50F6306A600A38FB6FECA
:103AD0006FE04F82032741068345A700A38FB6FE00
:103AE0006FE04F819307700433086D002328F106BF
:103AF000930C010A6FD05FF99305130013050B00B7
:103B00002328110123246100EF30907D03238100DD
:103B100083280101130D05006302053C930D050088
:103B20006FF04FFB930700032304F10C930780070A
:103B30006FF08FF8130360006FD09FE963140300E8
:103B400013031000032EC10F832E010F032F410F0B
:103B5000832F810F93620910E34A0EBE130C010BF1
:103B6000930603001308C10D9307010D1307C10C41
:103B70001306200093050C0013050B0023265102A9
:103B800023241103232261022328D10B2320D103F4
:103B9000232AE10B232EE101232CF10B2328F10131
:103BA000232EC10B2324C101EF2010208322C10248
:103BB00023242107032E8100832F0101032FC1013C
:103BC000832E01020323410283288102130D050085
:103BD00013890200232E0106930D00006FF05FC3CE
:103BE00093047006832781039306F00F23260102B6
:103BF00083C70700232A01026388D7040327010330
:103C000063D4E704B307F740032781032328F102B5
:103C100083471700638E070003264103130717002D
:103C2000232CE10213061600232AC1026FF0DFFCE9
:103C30000327C102832781031307170083C70700E7
:103C40002326E1026FF05FFB0327C10283274103B4
:103C5000B387E70003278104B387E702B38C97019A
:103C600013CCFCFF135CFC4133FC8C016FD05FFD77
:103C7000130C010B13050C002326110323246102EE
:103C80002328D10B232AE10B232CF10B232EC10B6C
:103C9000EF1011121306C10CEF501003138605002C
:103CA0009305050013050C00EF10016E9307010941
:103CB000938507002324F1008327010B930C010A4D
:103CC000130601082328F1088327410B13850C00F4
:103CD0002326C106232AF1088327810B232001080C
:103CE00023220108232CF1088327C10B2324010878
:103CF000232EF108B707FC3F2326F108EFE0005F11
:103D00000328010A032E410A832E810A032FC10AC8
:103D100093850C0013050C002328010B23220103BB
:103D2000232AC10B2320C103232CD10B232ED10125
:103D3000232EE10B2328E1012320010A2322010A7B
:103D40002324010A2326010AEFE0001E032F0101AC
:103D5000832EC101032E01020328410203238102A5
:103D60008328C10263160500930710002326F10C77
:103D7000B7670180938747BC2322F1066FF0CFE934
:103D8000930D0000138907006FF01F9D9306610DCE
:103D90006318060093060003230BD10C9306710DE4
:103DA0001307011B938707033386E6402380F60041
:103DB0009307D60D2322F1046FD05FE48327C1035C
:103DC00093046006B30CF700B38C6C006FF05FB720
:103DD000B38CFC40938C1C0013CCFCFF135CFC41A7
:103DE00033FC8C016FF0DF93930C010A93850C0078
:103DF00013050C002326010323241103232261024F
:103E00002328D10B2320D103232AE10B232EE10108
:103E1000232CF10B2328F101232EC10B2324C101F4
:103E20002320010A2322010A2324010A2326010A4E
:103E3000EFE0800F032E8100832F0101032FC101CA
:103E4000832E010203234102832881020328C10239
:103E5000E30005A693071000B38767402326F10C03
:103E60003308F8006FD05FC28327810693F71700ED
:103E7000639407006FD09FDA6FD0DFD913870800F3
:103E80006FE09FBB639A0700130C10009304600659
:103E9000930C10006FF0DF888327C1039304600642
:103EA000938C1700B38C6C0013CCFCFF135CFC41AB
:103EB00033FC8C016FF0DF868327C10003A307006A
:103EC00093874700635403001303F0FF83441400F7
:103ED0002326F100138406006FD00FE983D7CA00B0
:103EE00093E707042396FA006FD09F829307200080
:103EF0002322F1046FD09FD03787018093070500FC
:103F00000325479C9306060013860500938507004A
:103F10006FD0CFCA83D7C50003AE450603D3E500F3
:103F200083A8C50103A84502130101B893F7D7FF81
:103F300013070040232C8146231AF1001384050047
:103F40009307010793058100232A914623282147DF
:103F5000232E1146130905002326C107231B6100E8
:103F600023221103232601032324F100232CF10033
:103F70002328E100232EE10023200102EFD00FC40B
:103F800093040500635C05028357410193F707041E
:103F9000638807008357C40093E707042316F400DF
:103FA0008320C14703248147032901471385040067
:103FB0008324414713010148678000009305810075
:103FC00013050900EF00C03CE30005FC9304F0FF7B
:103FD0006FF09FFBB787018083A7479C130101FF08
:103FE000232481002322910023261100930405003D
:103FF000138405006386070003A787036300070E89
:104000000317C400931707019376870093D707011E
:1040100063800604832604016380060613F61700F6
:10402000630406080326440123240400130500004A
:104030003306C040232CC400638606088320C100D9
:1040400003248100832441001301010167800000E3
:1040500093F607016384060C93F7470063960708FD
:104060008326040113678700931707012316E400D2
:1040700093D70701E39406FA13F607289305002067
:10408000E30EB6F89305040013850400EF305013D7
:104090000317C400832604019317070193D7070170
:1040A00013F61700E31006F813F627009305000037
:1040B00063140600832544012324B4001305000083
:1040C000E39E06F693F70708E38A07F613670704EB
:1040D0002316E4001305F0FF6FF05FF61385070069
:1040E000EF00C0656FF0DFF183250403638E0500E8
:1040F000930704046388F50013850400EF00807CB7
:104100000317C40023280402832604011377B7FD94
:10411000232204002320D4006FF0DFF493079000E3
:1041200023A0F400136707042316E4001305F0FF2F
:104130006FF0DFF08397C500130101FE232C81008F
:1041400023263101232E1100232A91002328210147
:1041500093F687001384050093090500639A0610FF
:10416000371700001307078083A64500B3E7E70071
:104170002396F5006354D01803278402630A070CC2
:1041800083A409009396070123A009001396370121
:104190008325C40193D606016348061693061000D2
:1041A0001306000013850900E70007009307F0FFDE
:1041B000630CF5188356C400032784028325C401C9
:1041C00093F64600638E060083264400832704038B
:1041D0003305D540638607008327C4033305F540C4
:1041E000130605009306000013850900E700070089
:1041F0009307F0FF631EF51003A709008317C4009F
:10420000630807169306D0016306D7009306600182
:104210006314D70C8326040137F7FFFF1307F77FDA
:10422000B3F7E7002316F400232204002320D40070
:104230008325040323A09900638C050093070404DD
:104240006386F50013850900EF00C0672328040288
:10425000130500008320C10103248101832441014F
:10426000032901018329C1001301010267800000B5
:1042700003A90501E30E09FC83A4050013970701B8
:10428000135707011377370023A02501B384244176
:10429000930700006314070083A745012324F4005B
:1042A000634890006FF0DFFA3309A900E35290FAF7
:1042B000832744028325C401938604001306090062
:1042C00013850900E7800700B384A440E34EA0FCF7
:1042D0008357C4001305F0FF93E707048320C1014F
:1042E0002316F400032481018324410103290101E1
:1042F0008329C100130101026780000003A7C503E1
:10430000E34CE0E66FF0DFF4032504056FF05FEBAC
:104310008357C40037F7FFFF1307F77FB3F7E700B2
:10432000832604019397070193D707412316F400CE
:10433000232204002320D40013973701E35A07EE09
:104340002328A4046FF0DFEE83A70900E38407E6C7
:104350001307D0016388E702130760016384E70253
:104360008357C40093E707042316F4006FF09FEE11
:1043700037F7FFFF1307F77F83260401B3F7E70042
:104380006FF0DFFA23A09900130500006FF09FEC97
:10439000130101FE232C8100232E110013040500BC
:1043A0006306050083278503638007028397C500A2
:1043B000639607028320C1010324810113050000D5
:1043C00013010102678000002326B100EF000037CF
:1043D0008325C1008397C500E38E07FC1305040005
:1043E000032481018320C101130101026FF09FD4D6
:1043F0009305050063080500B787018003A5479C66
:104400006FF01FF9B787018003A5079CB7450080AF
:10441000938505396F009006130500006780000042
:10442000B7E50080938505A96F005005130101FED3
:10443000B7470080232E1100232C8100232A9100EE
:104440002328210123263101232441012322510164
:10445000232061010324450093870742232EF502A0
:104460001307C52E930730002324E52E2322F52EB3
:104470002320052E93074000130905002326F4008E
:104480001306800093050000232204062320040065
:10449000232204002324040023280400232A0400E8
:1044A000232C04001305C405EFC09FC4379B008074
:1044B00083248900B79A0080379A0080B7A90080CA
:1044C000130BCB6B938A0A72130A8A7A9389098138
:1044D000B707010023206403232254032324440349
:1044E00023263403232E84009387970023A6F40009
:1044F000130680009305000023A2040623A00400F5
:1045000023A2040023A4040023A8040023AA040077
:1045100023AC04001385C405EFC09FBD0324C9006C
:10452000B707020023A0640323A2540323A4440377
:1045300023A6340323AE9400938727012326F40097
:104540002322040623200400232204002324040041
:1045500023280400232A0400232C04001305C40587
:104560001306800093050000EFC09FB88320C101AF
:1045700023206403232254032324440323263403E7
:10458000232E84000324810193071000232CF902B9
:1045900083244101032901018329C100032A8100E9
:1045A000832A4100032B01001301010267800000F0
:1045B0001305000067800000130101FF2322910012
:1045C000130680069384F5FFB384C40223202101DF
:1045D00013890500232481002326110093854407B5
:1045E000EF30005013040500630005021305C500F9
:1045F00023200400232224012324A40013868406FC
:1046000093050000EFC0DFAE8320C1001305040056
:1046100003248100832441000329010013010101C7
:1046200067800000130101FEB78701802328210164
:1046300003A9079C23263101232E11008327890318
:10464000232C8100232A9100930905006386070A21
:104650001309092E9304F0FF8327490003248900DE
:104660009387F7FF63D807006F00000813048406E0
:10467000638C97060317C4009387F7FFE31807FEC0
:10468000B707FFFF938717002322040623200400A7
:1046900023220400232404002326F40023280400FA
:1046A000232A0400232C0400130680009305000035
:1046B0001305C405EFC0DFA323280402232A040244
:1046C00023220404232404048320C10113050400CD
:1046D0000324810183244101032901018329C100AD
:1046E000130101026780000003240900630C040029
:1046F000130904006FF05FF613050900EFF01FD3F4
:104700006FF01FF59305400013850900EFF0DFEA15
:104710002320A90013040500E31C05FC9307C00037
:1047200023A0F9006FF05FFAB787018003A5079C0B
:10473000B7E50080938505A96F0040548327850362
:1047400063840700678000006FF05FCE6780000021
:10475000678000006780000067800000B7870180E5
:1047600003A5479CB7450080938585416F00C046EF
:10477000B787018003A5479CB74500809385055BFB
:104780006F008045130101FE23263101B7790180B6
:10479000232C8100232A9100232821012324410175
:1047A000232E1100138A050013090500938909437C
:1047B000EF30D03B03A78900B71700001384F7FE42
:1047C000832447003304444193F4C4FF330494002A
:1047D0001354C4001304F4FF1314C400634EF40014
:1047E0009305000013050900EF40D05883A7890006
:1047F000B38797006308F50213050900EF305037BF
:104800008320C10103248101832441010329010183
:104810008329C100032A810013050000130101024E
:1048200067800000B305804013050900EF409054F5
:104830009307F0FF630AF504B78701809387C7A643
:1048400003A7070083A68900B384844093E414007F
:10485000330487401305090023A2960023A0870094
:10486000EF3010318320C1010324810183244101F1
:10487000032901018329C100032A810013051000C7
:104880001301010267800000930500001305090071
:10489000EF40504E03A789009306F000B307E540B0
:1048A000E3DCF6F4B786018083A6869C93E71700C5
:1048B0002322F7003305D540B786018023A6A6A69C
:1048C0006FF09FF3638A0512130101FF2324810017
:1048D0002322910013840500930405002326110070
:1048E000EF30D0280328C4FF130784FFB775018079
:1048F0009377E8FF3306F700938505438326460048
:1049000003A5850093F6C6FF630AC51A2322D600C5
:10491000137818003305D6006310080A032384FFB8
:1049200003284500377501803307674083288700D7
:1049300013058543B3876700137818006380A814B4
:104940000323C70023A66800232413016304081E61
:1049500093E617002322D7002320F6009306F01FCA
:1049600063E8F60A93F687FF9386860003A5450061
:10497000B386D50003A6060013D85700930710008E
:10498000B3970701B3E7A700138586FF2326A70087
:104990002324C70023A2F50023A0E6002326E60077
:1049A000032481008320C100138504008324410077
:1049B000130101016F30D01B03254500137515004D
:1049C000631E050237750180B387D7001305854341
:1049D0008326860093E817003308F7006388A6163D
:1049E0000326C60023A6C6002324D60023221701CF
:1049F0002320F8006FF09FF66780000093E6170011
:104A0000232ED4FE2320F6009306F01FE3FCF6F4D9
:104A100093D6970013064000636CD60E93D66700BA
:104A2000138896031386860313183800338805010C
:104A300083260800130888FF6308D81203A64600DF
:104A40001376C6FF63F6C70083A68600E318D8FE78
:104A500003A8C600232607012324D70003248100CE
:104A60008320C1002324E80013850400832441002F
:104A700023A6E600130101016F30900F631608149E
:104A80008325C60003268600B387F6000324810031
:104A90002326B60023A4C50093E617008320C10097
:104AA0002322D700138504003307F7008324410035
:104AB0002320F700130101016F30900B13781800C9
:104AC000B387D70063100802032584FF3307A7408C
:104AD0008326C70003268700B387A7002326D600B6
:104AE00023A4C600B786018013E6170083A6C69CE0
:104AF0002322C70023A4E500E3E4D7EAB7870180B7
:104B000083A5879D13850400EFF0DFC76FF05FE991
:104B1000130640016374D602130640056364D6068B
:104B200093D6C7001388F6061386E60613183800D6
:104B30006FF0DFEFB387D7006FF09FE91388C605EA
:104B40001386B605131838006FF05FEE23AAE50050
:104B500023A8E5002326A7002324A700232217016A
:104B60002320F8006FF0DFE303A54500135626402D
:104B7000930710003396C7003366A60023A2C50032
:104B80006FF05FED13064015636CD60093D6F70007
:104B90001388860713867607131838006FF01FE90D
:104BA00013064055636CD60093D627011388D607A9
:104BB0001386C607131838006FF05FE71308803FAD
:104BC0001306E0076FF09FE693E617002322D70055
:104BD0002320F6006FF0DFDC130101FE2328210102
:104BE0002326310123244101232251012320610185
:104BF000232E1100232C8100232A9100138B050002
:104C0000930A052E130A0000930910001309F0FF00
:104C100083A44A0003A48A009384F4FF63C60402B9
:104C20008357C4009384F4FF63FCF9008317E40006
:104C30001305040063862701E7000B00336AAA000E
:104C400013048406E39E24FD83AA0A00E3920AFC6F
:104C50008320C1010324810183244101032901012F
:104C60008329C100832A4100032B010013050A0098
:104C7000032A81001301010267800000130101FD76
:104C800023202103232E3101232C4101232A51010A
:104C90002328610123267101232611022324810286
:104CA00023229102930A0500938B0500130B052E16
:104CB000130A0000930910001309F0FF83244B002E
:104CC00003248B009384F4FF63C804028357C40059
:104CD0009384F4FF63FEF9008317E4009305040056
:104CE00013850A0063862701E7800B00336AAA0058
:104CF00013048406E39C24FD032B0B00E3100BFC40
:104D00008320C1020324810283244102032901027A
:104D10008329C101832A4101032B0101832BC10097
:104D200013050A00032A81011301010367800000B3
:104D300093064500930700001305A5013788FFFF80
:104D40006F00C001939717002390E6009397070127
:104D50009386260093D70701630ED50203D706007A
:104D6000137617006304060093E717001357170024
:104D700013F62700B3650701E30606FC93971700B7
:104D80002390B600939707019386260093D70701D7
:104D9000E316D5FC67800000930685011307000029
:104DA000130525006F00C001131717002390F600AC
:104DB000131707019386E6FF135707016304D50411
:104DC00083D70600139607011356064193971700E1
:104DD00063540600136717009397070193D70701E1
:104DE0001376270093E51700E30006FC131717005E
:104DF0002390B600131707019386E6FF13570701A8
:104E0000E310D5FC67800000130101FE370E01009E
:104E1000231D0100231E0100938585019307C10115
:104E200013088100130EFEFF03D705009387E7FFE9
:104E30009385E5FF63180702239F07FEE39607FFAC
:104E4000130646009306E10103D707009387270066
:104E500013062600231FE6FEE398D7FE1301010286
:104E6000678000003307A70283D8270003D3070019
:104E7000B376C701B38616011357070193D806010D
:104E80003307670033071701935807012391D700B1
:104E90002390E700239F17FFE39807F96FF05FFA6D
:104EA00013072501835705001305250063980700A4
:104EB000E31AE5FE130500006780000013051000EB
:104EC00067800000130101FF232291008354250114
:104ED000232481002326110093C7F4FF13971701A1
:104EE0001304050063160700EFF09FFB631805002D
:104EF000B787FFFFB3C4F400231994008320C100D7
:104F00000324810083244100130101016780000014
:104F1000130101FF232481000354250123261100DE
:104F20009347F4FF13971701631A0700EFF05FF739
:104F30009307050013050000639407001355F40060
:104F40008320C10003248100130101016780000058
:104F500083572501130101FD2324810293D7F70014
:104F6000232291022326110223202103232E310123
:104F7000B307F0402390F5008357250137870000E1
:104F80001307F7FFB377F7002391F50093040500AB
:104F9000130405016382E7049387650023920500EB
:104FA0001305E5FF035704001304E4FF938727006C
:104FB000239FE7FEE31885FE239C05008320C102A2
:104FC0000324810283244102032901028329C101B0
:104FD0001301010367800000035725011389450071
:104FE00033F7E700631CF7022326B100EFF05FEB15
:104FF0008325C100630405029387650023920500A1
:105000001385C4FF035704001304E4FF93872700AC
:10501000239FE7FEE31885FE6FF05FFA9389A501F1
:1050200013092900231F09FEE39C29FF8320C102E5
:105030000324810283244102032901028329C1013F
:10504000130101036780000083572501130101FB51
:105050002324810493C7F7FF2322910423261104FC
:1050600013971701930405001384050063160700C6
:10507000EFF01FE3631205088357240193C7F7FF7E
:105080001397170163040706930581001385040035
:10509000EFF01FEC9305410213050400EFF05FEB06
:1050A0008355810003554102630CB5049307A100A9
:1050B000130761021306010283D6070093872700B6
:1050C000639A0608835607001307270063940608AF
:1050D000E394C7FE130500008320C1040324810468
:1050E00083244104130101056780000013050400B7
:1050F000EFF01FDBE30A05F81305E0FF6FF0DFFDBB
:10510000133515000356A100835661023305A040F4
:105110001307A10093076102137525001305F5FF1E
:105120009305C1039387270013072700631ED6004A
:10513000E382B7FA0356070083D607001307270058
:1051400093872700E306D6FEE3E8C6F83305A040C0
:105150006FF09FF813051000E38005F81305F0FFCA
:105160006FF09FF7130101FF23261100EFF05FD3CB
:105170008320C10013351500130101016780000071
:10518000130101FE232C8100232A9100232E1100FC
:1051900023282101232631019384050013040500EF
:1051A00063C4050A9307F000138605001305450044
:1051B000930684019305F00063D4970293070500DA
:1051C00003D7270093872700239FE7FEE39AD7FEA4
:1051D000231C0400130606FFE3C2C5FE93F4F4008B
:1051E0009307700063D89702130784019305240086
:1051F00093070000835607001307E7FF1396860006
:10520000B3E7C7002311F70093D78600E314B7FE76
:10521000938484FF638A04009384F4FF13050400DD
:10522000EFF09FB7E39A04FE130500008320C1014D
:105230000324810183244101032901018329C10041
:105240001301010267800000930710FF3309B0408B
:1052500063DCF51293058501930900009306450070
:105260001306F0000357840193870500B3E9E900B2
:1052700003D7E7FF9387E7FF2391E700E39AD7FE81
:1052800023120400130909FFE34E26FD930700FFD4
:10529000130710FFB38797401309000063C4E40AA3
:1052A0003309F9009307700063D627059399090124
:1052B00093D90941834784019305A401B3E9F90017
:1052C0009399090193D909019307000003D60600B9
:1052D000938626001357860033E7E700931786006E
:1052E00093970701239FE6FE93D70701E390B6FE4D
:1052F000130989FF630C0906835784011309F9FF19
:105300001305040093F71700B3E93701EFF05FA22C
:10531000E31409FE9397090193D7074163900704AB
:1053200013950901135505018320C101032481014F
:1053300083244101032901018329C10013010102D2
:105340006780000013F907FF330920413309F90092
:1053500093077000E3D027FB6FF05FF5930910000F
:1053600013950901135505016FF01FFC1385090002
:105370006398090013150501135505016FF01FEB24
:10538000130510006FF01FFF930790FF93090000B3
:10539000E3D4F5F6930644006FF0DFF18357450040
:1053A000130101FF232291002326110023248100F1
:1053B0002320210193040500639C070C035765001B
:1053C000130400009317070193D7074163C4070A2A
:1053D0009306A5011306000A631807029387640069
:1053E0006F00800003D7070093872700239EE7FE06
:1053F000E39AF6FE239C040013040401630CC40624
:1054000003D76400E30C07FC937707F0639007046D
:10541000138584019385240093070000130705007A
:10542000835607001307E7FF13968600B3E7C7000C
:105430002311F70093D78600E394E5FE03D76400B9
:1054400013048400937707F0E38807FC1309000A2C
:105450006F00400113041400EFF01F94634C8900A7
:1054600003D764001317070113570741138504007E
:10547000E35207FE8320C1001305040003248100CA
:10548000832441000329010013010101678000000A
:1054900013F707F013040000631007041309F0F674
:1054A0006F0040011304F4FFEFF09F88E30424FD34
:1054B00083D7440013850400E39607FE8320C100D0
:1054C0001305040003248100832441000329010003
:1054D0001301010167800000930645009305A501B3
:1054E000130700006F00800083D7060013D68700E3
:1054F0003367C700939787002390E600139707014F
:105500009386260013570701E390B6FE83D7440025
:10551000130480FF6FF09FF8130101FE232C81001C
:10552000232A91002328210123263101232441012C
:10553000232251011389060093840700232E1100B2
:105540001304050093890500130A0600930A070057
:10555000EFF0DFE4930700093309A94063DCA716E5
:10556000B78700009387E7FF63DA271F63840A1C6D
:1055700003A5440083A70400630AF5061387A4016A
:105580009387440313072700231F07FEE31CF7FE3E
:1055900093078003630CF53263D0A71693070004CA
:1055A000630CF52E930710076318F534B787004096
:1055B0009387F7FF1307A00023AAF400B787FFFF24
:1055C00023A4E400239CF40023A6E4009307A00096
:1055D000378700009387870093971700B387F400FD
:1055E0002395E70023A0A4006358201B83A5840013
:1055F00083D744011308F008139615003306C4003E
:1056000003570600B376F700634AA8021308B000F8
:105610006346B802930706009305840103D7270069
:105620006304070093E61600239107009387270081
:10563000E396F5FE0357060083D7440193C7F7FFAF
:10564000B3F7E7002310F60083D7640133F7D700E0
:10565000630007046384D71A138624039306840126
:105660009384C401130700008357060083D5060006
:105670009386E6FF1306E6FFB387B700B387E7001C
:1056800013D707012391F60013771700E31E96FC4A
:105690006358201983574400639E0712B7870000A0
:1056A000231C04009387E7FF63C827092311240103
:1056B0008320C101032481018324410103290101C5
:1056C0008329C100032A8100832A410013010102BA
:1056D000678000006354090E930700F7635CF908C4
:1056E000930724001304A40193872700239F07FE38
:1056F000E39C87FE6FF0DFFB930780016308F516DC
:1057000093075003631AF51E37170000B70700040C
:10571000930660009387F77F1307078023AAF4009E
:1057200023A4D400239CE40023A6D40093076000A4
:105730006FF05FEA231C0400B787FFFF93C7F7FFF2
:105740002311F400930744001304840123900700FD
:1057500093872700E31CF4FE6FF09FF59307240066
:105760001304A40193872700239F07FEE39C87FE71
:105770006FF01FF49305090013050400EFF05FA01C
:105780006304050093091000638C0A0C03A5440010
:1057900083A70400E314F5DE930700096304F50A08
:1057A000835784011305040093F71700B3E9F90048
:1057B000EFF00FD803A544006FF05FE3E3800AEE3B
:1057C00003A5440083A70400E31AF5DAE34020E3CD
:1057D0006FF09FFC13050400EFF08FD5B787000032
:1057E00013091900231C04009387E7FFE3C627F57C
:1057F000E35E09EA231104006FF09FEB6394090C48
:1058000083A7C40003D7840193971700B307F4005C
:1058100083D70700B3F7E700E39007E4E34C20E702
:10582000930700096306F50013050400EFF0CFD6D7
:1058300083574400E39007FA231C0400E34C09FA61
:105840006FF0DFE603A6840083D744011316160029
:105850003306C40003570600B3F6E7006FF01FDEFF
:10586000231C0400231104006FF09FE4B70780009D
:105870009387F70F1307400023AAF4009307001043
:1058800023A4E400239CF40023A6E4009307400033
:10589000130700106FF01FD49307700023A4F400C7
:1058A000B70701809387F7FF23AAF400930710003E
:1058B000239CF4009307600023A6F4001307100054
:1058C0006FF05FD1E30A0AD86FF09FDCB707800062
:1058D0009387F70F1307600023AAF40093070010C3
:1058E00023A4E400239CF40023A6E40093076000B3
:1058F000130700106FF01FCE9307C00023A4F4001D
:10590000B70701809387F7FF23AAF40093071000DD
:10591000239CF4009307B00023A6F40013071000A3
:105920006FF05FCB130101FD23229102232E310181
:105930009384050083592500232611022324810224
:1059400023202103232C410113090600232A51019E
:10595000232861012326710123248101232291013F
:105960002320A101130A0500EFF05FA303D4240054
:105970009307050013850400B389F940930A49038E
:10598000EFF0DFA13304A4401307E90493870A0072
:1059900093872700239F07FEE39CE7FE634A3409B1
:1059A000930B4A00138B44009389F9FF930CAA01CF
:1059B000138C240013070B0093870B0003D60700FA
:1059C000835607009387270013072700631AD60A18
:1059D000E39697FF13068A0113878401930600005C
:1059E00083570700835506001307E7FFB387D740A7
:1059F000B387B74093D607012311F70093F616003B
:105A00001306E6FFE31EECFC130D100013850A00DD
:105A1000EFF08FB88357C9041304F4FF1385040013
:105A2000336DFD002316A905EFF00FB7E31434F929
:105A300093060400032481028320C1028329C1014B
:105A4000032A8101832A4101032B0101832BC10019
:105A5000032C8100832C4100032D010093070900D2
:105A60001385040003290102832441021307000067
:105A70001306000093050000130101036FF0DFA976
:105A8000130D0000E3E4C6F86FF0DFF403570500E0
:105A9000835725006306070037870000B3E7E70058
:105AA0002399F50003572500B78700009387F7FF78
:105AB0006304F702930765009385050113058501CB
:105AC00003D70700938727009385E5FF2391E5001F
:105AD000E398A7FE67800000930765001305A50102
:105AE00003D7070093872700631A0702E39AA7FEEC
:105AF000138725019387050093872700239F07FEBF
:105B0000E31CF7FE83D72501378700001307F7FF53
:105B1000B3E7E7002399F5006780000013870501CC
:105B20009387050093872700239F07FEE31CF7FE5A
:105B3000B7C7FF7F23A8F50067800000130101F7B6
:105B400023286107035B2501B78700009387F7FFD0
:105B5000232C410733FA6701131A0A012324810811
:105B60002322910823202109232E310723261108FF
:105B7000232A510723267107232481072322910713
:105B8000135A0A0193040500138905001304060043
:105B9000938906006312FA10EFF08FB0631A05289C
:105BA000835A2901B3775A016382472B1385040076
:105BB000EFF04FDB630E052EB76501809385C5DAE4
:105BC00013050900EFF04FC863060536835A290113
:105BD000B78700009387F7FFB3FA5701939A0A013A
:105BE00093DA0A016394FA2C13050900EFF08FD7BA
:105BF0006310053283D72401B3F7FA006398570B7B
:105C000013850400EFF00FD6631805001305090093
:105C1000EFF04FD5630C050813850400EFF04FAF8C
:105C20009304050013050900EFF08FAEB384A44080
:105C3000B33490009394F4002319940013072401C3
:105C40009307040093872700239F07FEE31CF7FEBA
:105C500083572401378700001307F7FFB3E7E700F6
:105C60002319F4008320C1080324810883244108F8
:105C7000032901088329C107032A8107832A4107D1
:105C8000032B0107832BC106032C8106832C4106BD
:105C9000130101096780000083DA250133F75701FA
:105CA0001317070113570701630AF704138504004C
:105CB0009305C100EFF0CFA91305090093058102F8
:105CC000EFF00FA98354E1000359A102639C04047F
:105CD00093070101930641026388D72003D7070089
:105CE00093872700E30A07FE1305C100EFF00FEBCF
:105CF0000357A102B304A0406F0000031385050001
:105D0000EFF00F9AE30605EC1307490183570900EA
:105D10001309290013042400231FF4FEE318E9FEED
:105D20006FF05FF413070900930A09009307C1029B
:105D300093060104631207026382F61C03D707006F
:105D400093872700E30A07FE13058102EFF00FE5B2
:105D50000357A102B30AA94083578102138C890318
:105D6000239BE902239AF9021387E90493070C00A5
:105D70002390070093872700E31CF7FE138AC904CA
:105D8000930B000013094102930C0101130B6104F2
:105D9000035509001309E9FF6318050C03D7C9046B
:105DA00093070A00B3EBEB0003D7E7FF9387E7FF06
:105DB0002391E700E39A87FF239C0902E31A99FDE8
:105DC00013874903930781029305210403560700B3
:105DD0009387270013072700239FC7FEE398F5FE4C
:105DE000B7C6FFFFB38454019386260093850B004A
:105DF000130581029387090013070004B386D400BA
:105E000013060000EFF04FF1035781028357C100E2
:105E10009305040013058102B387E740B337F00010
:105E2000B307F0402314F102EFF05FC66FF09FE379
:105E30001387440183D704009384240013042400AF
:105E4000231FF4FEE398E4FE6FF0DFE11305090081
:105E5000EFF00F85E31A05EA13850400EFF08FB029
:105E6000E30805D66FF05FD5130641049305810260
:105E7000EFE09FF993050A00130600001307C10520
:105E800003D80500835707009385E5FF1307E7FF55
:105E9000B3870701B387C70013D607012391F50025
:105EA00013761600E31E67FD6FF05FEF03DB24013E
:105EB000B78700009387F7FF33FB6701131B0B01C4
:105EC000135B0B01E314FBDE13850400EFF08FA9D5
:105ED000E31405D48357290193C7F7FF13971701DC
:105EE000E31607DC6FF09FD29307440113042400EC
:105EF000231F04FEE39C87FE6FF0DFD69307440167
:105F000013042400231F04FEE31CF4FE6FF09FD54E
:105F1000B76501809385C5DA13850400EFF0CF9251
:105F2000630A050083D72401B3F7FA00E38E57F91B
:105F30006FF05FFA130704019307040093872700AB
:105F4000239F07FEE39CE7FEB7C7FF7F2328F400EB
:105F50006FF05FD183572501130101F52324810AD6
:105F600093C7F7FF2322910A2320210B232E310907
:105F70002326110A232C4109232A510923286109C8
:105F80002326710923248109232291092320A109B1
:105F9000232EB107139717011309050093890500F4
:105FA000130406009384060063160700EFE05FEF1A
:105FB0006318053883D7290193C7F7FF1397170193
:105FC000630E0708376A01809305CADA13050900D2
:105FD000EFF08F8763040510035A290103D72901C5
:105FE000B78700009387F7FF33FA4701B3FAE7005A
:105FF000631AFA0813050900EFF0CF96630805103D
:1060000063984A0113850900EFF0CF956310050EE0
:106010009307440113042400231F04FEE31CF4FE31
:106020008320C10A0324810A8324410A0329010A27
:106030008329C109032A8109832A4109032B010904
:10604000832BC108032C8108832C4108032D0108F0
:10605000832DC1071301010B678000001385090020
:10606000EFE01FE4E30005F61387490183D7090039
:106070009389290013042400231FF4FEE398E9FE0A
:106080006FF01FFA6386FA08130509009305C10132
:10609000EFE01FEC9305810313850900EFE05FEB50
:1060A000835BA1030359E10163920B0C9307C103C6
:1060B000930D0105638EFD3403D7070093872700F6
:1060C000E30A07FE13058103EFF04FADB307A040CD
:1060D0000356E1012326F1006F00C0099305CADAD7
:1060E00013850900EFE05FF6E31805EE13070401DE
:1060F0009307040093872700239F07FEE39CE7FE96
:10610000B7C7FF7F2328F4006FF09FF1E39E4AF7A3
:1061100013850900EFF00F85E30805F61305090064
:10612000EFE01FDF9304050013850900EFE05FDE59
:10613000B387A440B337F0009397F7002319F40016
:10614000130724019307040093872700239F07FE6A
:10615000E39CE7FE83572401378700001307F7FF0E
:10616000B3E7E7002319F4006FF09FEB23267101DA
:10617000130609002324210193070102930641031A
:10618000631206026380F62A03D70700938727006D
:10619000E30A07FE1305C101EFF04FA0B307A940C2
:1061A0002324F10003278103138D840393070D003B
:1061B00023AAE4021389E40493872700239F07FEA0
:1061C000E31CF9FE13058103EFE09FB6035C210297
:1061D000370A0100930D0105931A0C01B38A8A4115
:1061E000130BA103130AFAFF930CE106930961054F
:1061F0008357C1030357E103930B0A0093970701E9
:10620000B387E70063E8FA00B3D78703939B0701DE
:1062100093DB0B01130641059305C10113850B00A8
:10622000EFE09FBE1307C1039307810583D50700E5
:106230000356070093872700130727006390C512B2
:10624000E39697FF930700009305C10613860D00A0
:106250000357060003D805001306E6FF3307F7408F
:1062600033070741935707012311E60093F71700FF
:106270009385E5FFE31E66FD23107D019307C103AF
:1062800003D7270093872700239FE7FEE39AB7FFF2
:1062900023180104130D2D00E31CA9F5930500003C
:1062A0009307C1039306210503D7070093872700AF
:1062B000B3E5E500E39AD7FE9397050193D707412D
:1062C00063840700930510009395050193D505019C
:1062D000138744039307810303560700938727001E
:1062E00013072700239FC7FEE398F6FE8327C1000C
:1062F00003278100B74600009386F6FFB38BE74083
:10630000130581039387040013070004B386DB00A1
:1063100013060000EFF04FA0035781038357C1011C
:106320009305040013058103B387E740B337F000FA
:10633000B307F040231CF102EFF04FF56FF05FCE92
:106340001307490183570900130929001304240086
:10635000231FF4FEE318E9FE6FF09FCCE374B6EE62
:106360009387FBFF9398070193D8080193070000D8
:10637000930541031306C1060357060003D8050021
:106380001306E6FF3307F74033070741935707012A
:106390002311E60093F717009385E5FFE31E36FD12
:1063A0001307C1039307810583D507000356070030
:1063B00093872700130727006398C500E39697FF8C
:1063C000938B08006FF01FE8E37CB6FE9387EBFF2A
:1063D000939B070193DB0B01130600009305410318
:1063E0001307C1068357070003D805001307E7FF0B
:1063F000B387C740B387074113D607012311F700BE
:10640000137616009385E5FFE31E37FD6FF09FE3DB
:106410009307440113042400231F04FEE39C87FE1A
:106420006FF01FC00357C101835781036304F70056
:10643000378600002319C4001307240193070400C2
:1064400093872700239F07FEE31CF7FE8357240151
:10645000378700001307F7FFB3E7E7002319F400BD
:106460006FF01FBC130101FD2324810223261102BA
:1064700013840500930741001307E1019387270068
:10648000239F07FEE39CE7FE0356E50093170601F2
:1064900093D7074163CA0706B78700009387F7FFC2
:1064A000231201003376F600630CF6069307E5002D
:1064B0002313C1001307A10083D6E7FF9387E7FFEB
:1064C00013072700231FD7FEE318F5FE6312060209
:1064D000231401009305040013054100EFF00FDBC6
:1064E0008320C1020324810213010103678000009D
:1064F000930710009305F0FF130541002314F100EA
:10650000EFE01FC86FF01FFD9307F0FF2312F100AB
:10651000B78700009387F7FF3376F600E318F6F8A5
:10652000930705009306E50003D70700938727002C
:10653000631C0704E39AD7FE130744019307040082
:1065400093872700239F07FEE31CF7FE1307240110
:106550009307040093872700239F07FEE31CF7FEA1
:1065600083572401378700001307F7FFB3E7E700DD
:106570002319F4008317E500E3D407F6130504009C
:10658000EFE05F946FF0DFF5130704019307040059
:1065900093872700239F07FEE31CF7FEB7C7FF7F03
:1065A0002328F4006FF0DFF383A8C500130101E195
:1065B00083AE050003AE450003A38500232E11031F
:1065C000832505049308F0FF232011179308000981
:1065D0002324811E232C411D2326111E2322911EBC
:1065E0002320211F232E311D232A511D2328611D05
:1065F0002326711D2324811D2322911D2320A11DEB
:10660000232EB11B2328D103232AC103232C61028B
:10661000232211172324C1002328D100232AE100BB
:10662000232E0101130A050013840700638005026D
:106630000327450493071000B397E70023A2E50062
:1066400023A4F500EF10905D23200A0493090106AE
:106650009385090013050103EFF0DFE013850900BE
:10666000EFE01F8B032781003335A0002320A40017
:1066700093073000E302F714930740012326F1004B
:10668000E31E0760835721070327411693C7F7FFCF
:10669000232CE100139717016318070013850900E5
:1066A000EFE01F80E3160540930700092322F1164F
:1066B0001307C107938709001306410783D6070014
:1066C0009387270013072700231FD7FEE398C7FEF1
:1066D0000356E108232201009317060193D70741CF
:1066E00063DE070013161601B707010013561601E3
:1066F0009387F7FF2317C1082322F100B76A0180AF
:106700009387CADA938B47019306000093078109A8
:1067100013870B00930DC10A6F008000835607009A
:1067200093872700239FD7FE13072700E398B7FF1F
:1067300063020616B78700009387F7FFE30CF6584D
:106740008317C108E3DE075C9305C10713850B00BF
:10675000EFE09F8F630C0514E34C050C8357E108B1
:10676000E39207668317C10893040000130901161A
:1067700063C80702B76701809387C7DA138487115C
:106780001306C107930609009305060013050400CC
:10679000EFF0CFBA8317C1089384F4FFE3D207FE6A
:1067A0001304010D130B810E130704009307C10797
:1067B0001306010983D607009387270013072700D4
:1067C000231FD7FEE398C7FE9306000093078109B5
:1067D00013870B006F008000835607009387270004
:1067E000239FD7FE13072700E398B7FFB767018001
:1067F0001387C7DA9387C7DA37FDFFFF930C870249
:10680000930DC712138C87116F00C000938D4D013B
:10681000938C4C019305040013850B00EFE0DF829D
:10682000930705009305040013850D006356F004DB
:10683000EFE09F819307050093060900130604000B
:106840009305040013850C0063C00702EFF00FAF3F
:1068500013068109930609009305060013850C00B1
:10686000EFF0CFADB384A4019357FD01338DA701A1
:10687000135D1D40E39C8CF9130681099306090002
:1068800093850B0013050600EFF0CFEC930C41123B
:106890006F0000039307C1079306E10803D70700C1
:1068A00093872700E31207EAE39AD7FE93040000D8
:1068B000930C4112130901161304010D130B810EE1
:1068C0009305040013058109EFE08FE813078109A0
:1068D0009307040083D60700938727001307270038
:1068E000231FD7FEE39867FF930504001305C10734
:1068F0002318010AEFE0CFE59307C107035704000F
:106900001304240093872700239FE7FEE31864FF06
:1069100013058109130609009305C107231A01080D
:10692000EFF04F800355C11A6314051C130D410984
:106930001304E107930B610B9385CADA1305C107B2
:10694000EFE08FF06306051A1307000093060D00B1
:106950006F00C001131717002390F60013170701EB
:106960009386E6FF135707016384860483D70600E6
:1069700013960701135606419397170063540600B8
:10698000136717009397070193D707011376270022
:1069900093E51700E30006FC131717002390B600D9
:1069A000131707019386E6FF13570701E39086FC50
:1069B0001307410B9307C10783D60700938727006E
:1069C00013072700231FD7FEE398A7FF2316010C08
:1069D000130700009306C10C6F00C00113171700C6
:1069E0002390F600131707019386E6FF135707015C
:1069F0006384760583D70600139607011356064174
:106A000093971700635406001367170093970701C5
:106A100093D707011376270093E51700E30006FCE0
:106A2000131717002390B600131707019386E6FF8C
:106A300013570701E39076FD130700009306C10C7E
:106A40006F00C001131717002390F60013170701FA
:106A50009386E6FF135707016384760583D7060004
:106A600013960701135606419397170063540600C7
:106A7000136717009397070193D707011376270031
:106A800093E51700E30006FC131717002390B600E8
:106A9000131707019386E6FF13570701E39076FD6E
:106AA0001306000093060D001307C10C83D50600E2
:106AB000835707009386E6FF1307E7FFB387B70006
:106AC000B387C70013D607012391F600137616008B
:106AD000E31E77FD13058109130609009305C1071D
:106AE000EFE05FE40355C11A9384F4FFE30605E485
:106AF000832741008326810013073000B337F0005D
:106B0000B307F04093F7D700938707022302F112EF
:106B10008327C1006394E600B38797001307A002A0
:106B2000138407006354F7001304A0021307A000A6
:106B30006308E54C130505031307E002A302A11245
:106B40002303E112E3CE071E930771122322F10003
:106B5000930B0000130D410B130B4109130CE107BC
:106B6000930D610B1306000093050B006F00C0012D
:106B7000131616002390F500131606019385E5FF02
:106B8000135606016384850583D705001395070115
:106B900013550541939717006354050013661600BB
:106BA0009397070193D707011375260093E8170001
:106BB000E30005FC131616002390150113160601B9
:106BC0009385E5FF13560601E39085FD13060D003E
:106BD0009307C10783D50700938727001306260074
:106BE000231FB6FEE39867FF2316010C130600006F
:106BF0009305C10C6F00C001131616002390F50019
:106C0000131606019385E5FF135606016384B50547
:106C100083D7050013950701135505419397170076
:106C200063540500136616009397070193D7070175
:106C30001375260093E81700E30005FC13161600F1
:106C400023901501131606019385E5FF13560601DF
:106C5000E390B5FD130600009305C10C6F00C00161
:106C6000131616002390F500131606019385E5FF11
:106C7000135606016384B50583D7050013950701F4
:106C800013550541939717006354050013661600CA
:106C90009397070193D707011375260093E8170010
:106CA000E30005FC131616002390150113160601C8
:106CB0009385E5FF13560601E390B5FD130500002B
:106CC00093050B001306C10C83D8050083570600FB
:106CD0009385E5FF1306E6FFB3871701B387A70087
:106CE00013D507012391F50013751500E31EB6FDBA
:106CF000130609009305C10713058109EFE09FC240
:106D00008357C11A03274100938507033306770190
:106D10002300B600938B1B00E35674E51345F4FF84
:106D20001355F5413375A4001309150033092701E4
:106D3000B30BA70013074000635EF704130750006E
:106D4000E386E7028347E9FF1307E9FF93F7F707B5
:106D5000634A047A9306E002130680039305000356
:106D6000638ED7006358F67A8347F7FF2300B70096
:106D70001307F7FF93F7F7076FF09FFE8347F7FFBF
:106D800093068003E3FAF60293071003938414003A
:106D9000A30FF7FEB765018013860400938585DA9B
:106DA00013850B00EF20D0098357210703278101AA
:106DB0002328911693C7F7FF2322E1161397170193
:106DC000631E070013850900EFE0CFB963100522A9
:106DD00013850900EFE0CF8C631A0520832641015B
:106DE000034741129387140023A0F60093870C00F9
:106DF000630A07029306E002630CD71C03C717005F
:106E000093871700E31A07FE9306500463E6FC001D
:106E10006F0040016388970103C7F7FF9387F7FF6F
:106E2000E31AD7FE2380070093870C009306000225
:106E30001306D00203C707006304D7006316C70018
:106E4000938717006FF01FFF13840C006F00C000C2
:106E500003C70700138406002300E4009306140010
:106E600093871700E31607FE83268100930720000F
:106E70000347F4FF6386F6128327C1009386070059
:106E800063D4970093860400930700036316F70208
:106E9000B307944163D2F602130600036F0080002B
:106EA00063DCE6008347E4FFA30F04FE1304F4FF52
:106EB00033079441E386C7FE032781009307300020
:106EC0006302F70A8327010123220A0493869700AD
:106ED0009307700163F2D70C13071000930740006B
:106EE00093971700138647019305070013071700B0
:106EF000E3F8C6FE2322BA0413050A00EF10804708
:106F00002320AA0493850C0093040500EF20D010E1
:106F10008327C101638807003304944133848400CC
:106F200023A087008320C11E0324811E0329011E84
:106F30008329C11D032A811D832A411D032B011DA5
:106F4000832BC11C032C811C832C411C032D011C91
:106F5000832DC11B138504008324411E1301011FCF
:106F6000678000008327C100B384970063CE04527A
:106F7000832741010327010183A70700B307F70017
:106F80002328F1008327010123220A049386370076
:106F900093077001E3E2D7F4930500006FF0DFF58B
:106FA00093070003E310F7F2B30794419306100030
:106FB000E3C4F6EE6FF01FF1032C010123268101DB
:106FC0009307A00263D087ED2326F1006FF08FEBCB
:106FD00003C70700E30A07E203C7170093871700F8
:106FE000A38FE7FEE31A07FE6FF01FE203274101BC
:106FF000B72700009387F7702320F7006FF0DFE2D8
:1070000013071003A302E1121307E0022303E112A6
:1070100093841400635EF02A93070003A303F11224
:10702000930781121304F4FF2322F1006FF05FB283
:10703000130D410B13070D009307C1071306010938
:1070400083D607009387270013072700231FD7FE47
:10705000E398C7FEB74700009387E7082313F10CB6
:10706000B76701809387C7DA138B870CB787000057
:107070009387F7FF2322F102B7C7FFFF938727000B
:10708000130E000193040000930C41121309011622
:107090001304010D130CA10A2324F1029306090025
:1070A0001306810993050D0013050B002320C1036E
:1070B000EFE05FEA032E01021307C1049307810981
:1070C00083D607009387270013072700231FD7FEC7
:1070D000E398B7FF832741028355E10533F6F500B6
:1070E000832781023305F600635AA03C130600098A
:1070F0003306A640130704009307C10483D6070094
:107100009387270013072700231FD7FEE39837FF35
:107110006358C0069307F0001307040063DCC7023E
:10712000130606FF93564600138716001317170021
:107130003307E4009307040093872700239F07FE8B
:10714000E39CE7FE130600083306A640939646002C
:107150003306D640B76701809387C7DA1316160047
:107160003386C7008356062383570700B3F7D7003B
:107170002310F7009395050193D5054163C20516C9
:10718000930781091307040003D6070083560700FD
:1071900093872700130727006314D602E316FCFE2B
:1071A00013070D009307810983D6070093872700F3
:1071B00013072700231FD7FEE398B7FFB384C4014A
:1071C000B76701809387C7DA130B4B019387C71208
:1071D000135E1E00E314FBEC8357610C0357E108B8
:1071E0001306810CB387E70037C7FFFF130727F7A4
:1071F000B387E7002313F10C1307C10793070D00B2
:1072000083D607009387270013072700231FD7FE85
:10721000E398C7FE13070000930781096F00800001
:1072200003D70B0093872700239FE7FE938B2B0048
:10723000E398B7FFB76701801387C7DA9387C7DA88
:10724000B71D0000130B8702938B87116F0000019D
:1072500093DD1D0063047B2B130B4B0193050D0085
:1072600013850B00EFD05FDE1307050093050D00BB
:1072700013050B006344E028EFD01FDDE34AA0FCB8
:107280009306090013060D0093050D0013050B006E
:10729000EFE05FCC13068109930609009305060011
:1072A00013050B00EFE09F89B384B4016FF05FFA20
:1072B000930C4112B7650180938545D813850C0066
:1072C000B7240000EF20C0379384F4706FF0DFAD77
:1072D000930B7112E39007AC232271016FF05F876B
:1072E0009307C104130704006F00C0009306E10573
:1072F000E388F6E803D60700835607009387270044
:1073000013072700E304D6FE8357210E032741020B
:10731000B377F7006394E702130504002320C10349
:10732000EFD01FB8032E0102E31C05E4130504008F
:10733000EFD05FE3032E0102E31405E49305C10ED1
:1073400013850B002320C103EFD09FC0930581104C
:1073500013050400EFD0DFBF0356C10E0355A11083
:10736000835EE10E1346F6FF13160601135606015F
:107370002316C10EB385AE40032E0102930605000D
:10738000635EB00693860C00130781109307011209
:10739000835507001307270093862600239FB6FE18
:1073A000E318F7FE231E0112130781109306C10E86
:1073B0006F00800003D6060013072700231FC7FEB7
:1073C00093862600E318F7FE231001121307C10E5F
:1073D00093870C00130FC11383D6070093872700F0
:1073E00013072700231FD7FEE398E7FF8356A1105A
:1073F000B305D54123120110138506006380052EC5
:107400002326D1029307F0F663CEF5061305C10ECD
:107410002320C103EFD0DFD6032E01028326C10251
:107420009305050093070112130641100355C10E81
:10743000035781106300E5301305000003D70700F0
:10744000835E06009387E7FF3307A7403307D741E2
:10745000135507012391E7001307A11013751500B9
:107460001306E6FFE39CE7FC1306100093070900F0
:1074700013070004130581102320C103EFE0CF8917
:10748000032E010293050400130581102320C1037C
:10749000EFE0CFDF032E01026FF09FCE83270101C3
:1074A000138CF7FF6FF09FB1832741012302011274
:1074B00013840C0023A007006FF0DFAC93070400D7
:1074C0001307410E93872700239F07FEE39CE7FEE7
:1074D0006FF05FCA83274100930C4112638A07064D
:1074E000B76501809385C5D813850C00B7240000CB
:1074F000EF2000159384F4706FF01F8B130B810E37
:107500006FF00FBC93071003230FF9FE9384140050
:107510006FF05F88938717002300F7006FF09F8755
:10752000930C4112B7650180938545DA13850C00F1
:10753000B7240000EF20C0109384F4706FF0DF8652
:107540008357C11A930B6112130971126FF08FFEEA
:10755000B7650180938585D913850C00B724000099
:10756000EF20000E9384F4706FF01F84930581095F
:107570001305C107EFE08FD19385CADA130581099E
:10758000EFD09FAC631005FCE34604808347E9FF1E
:10759000138727FD133717001347F7FF3387EB00D7
:1075A0000347070013771700630607FE1307E9FF79
:1075B00093F7F7076FF00FFA93871700A30FF7FE03
:1075C0006FF04FFD1304010D930504001305C1076F
:1075D000374D0000EFD0DF9793040000130B810EAE
:1075E0001309C10C930C210D130DEDFF130C50FD6D
:1075F0008357810E93F777006398070C1307410BAD
:107600009307040083D607009387270013072700FA
:10761000231FD7FEE39867FF1305410B2316010CC8
:10762000EFD00FF11305410BEFD08FF013060000E0
:107630009306090013070B0083D506008357070044
:107640009386E6FF1307E7FFB387B700B387C7004A
:1076500013D607012391F60013761600E31E97FD5B
:107660008357610B0357810B93873700231BF10A64
:10767000630007021305410BEFD08FEB8357610BBB
:107680000357810B93871700231BF10AE31407FEAE
:107690008357C10C639A07028357610B6366FD022F
:1076A000130704009307410B83D607009387270035
:1076B00013072700231FD7FEE39827FF2314010E8B
:1076C0009384F4FFE39684F39305C1071305040044
:1076D000EFE0CFBB130901166FF00F8D1307C11038
:1076E0009307010F83DE07000356070093872700E7
:1076F000130727006398CE0213066110E394C7FEB8
:107700000357C10E835781106302F70693070400E5
:107710001307410E93872700239F07FEE39CE7FE94
:107720006FF01FA66366D60D930701121306411072
:107730006FF0DFCF13050000130FE10E83DE0700AB
:10774000035706009387E7FF1306E6FF3307D701C9
:107750003307A700135507012391E70013751500A0
:10776000E31EE6FD130600006FF05FD013870600EE
:10777000639206068317E11063CE07049306011295
:107780006F0000022390F60013171700131707016C
:107790009386E6FF9307A11013570701E384F6CE03
:1077A00083D70600139607011356064193971700D7
:1077B00063540600136717009397070193D70701D7
:1077C0001376270093E51700E30E06FA2390B60020
:1077D0006FF09FFB1306C110930701126312070895
:1077E0006382C70803570600130626006FF01FFFC9
:1077F00013860C001307811093070112035507002D
:107800001307270013062600231FA6FEE318F7FE22
:10781000231E0112130581101307C10E1306411018
:10782000835E07001307270013052500231FD5FFDC
:10783000E318C7FE231001121305C10E13870C00B5
:10784000130FC113835E07001307270013052500DC
:10785000231FD5FFE318E7FF231201106FF01FBDB0
:10786000138516002315A1106FF0DFC103278500D3
:107870008327C5000326050083264500130101FC6C
:1078800013050100930541012324E1002326F100A3
:10789000232E11022320C1002322D100EFE09FBC40
:1078A000835761021305000093C7F7FF1397170171
:1078B000631A070013054101EFD08FDE1335150061
:1078C000130515008320C103130101046780000024
:1078D0001305050F67800000378501801305859229
:1078E000678000003785018013058592678000005E
:1078F000130101F923248106138405008395E50013
:107900002322910623202107232611069304060033
:107910001389060063CA050413068100EF60404F17
:10792000634405040327C100B7F700008320C106A4
:10793000B3F7E70037E7FFFFB387E70003248106CB
:1079400093B717002320F9009307004023A0F40009
:10795000371500008324410603290106130505801D
:1079600013010107678000008357C400232009002A
:1079700093F70708638407028320C1060324810666
:107980009307000423A0F400032901068324410681
:107990001305000013010107678000008320C10662
:1079A000032481069307004023A0F4000329010665
:1079B00083244106130500001301010767800000BE
:1079C00083D7C500130101FE232C8100232E110053
:1079D000232A91002328210193F72700138405000F
:1079E000638807029387350423A0F50023A8F500D8
:1079F0009307100023AAF5008320C101032481010D
:107A00008324410103290101130101026780000061
:107A10009306C1001306810093040500EFF05FEDAB
:107A2000832581001309050013850400EF00400B36
:107A30008317C40063080504374700801307074213
:107A400023AEE402032781008326C10093E70708E1
:107A50002316F4002320A4002328A400232AE400F2
:107A600063980604B3E727018320C1012316F400BD
:107A7000032481018324410103290101130101022F
:107A80006780000013F70720E31807F693F7C7FF96
:107A900093E72700130734042316F400930710001C
:107AA0002320E4002328E400232AF4006FF0DFF40D
:107AB0008315E40013850400EF609006631605004B
:107AC0008317C4006FF01FFA0357C4001377C7FF72
:107AD000136717009317070193D707416FF09FF8BB
:107AE000130101FD232E31012326110223248102DB
:107AF0002322910223202103232C4101232A510117
:107B0000232861012326710123248101232291016D
:107B10009387B50013076001930905006366F706B4
:107B20009307000163E6B71EEF00500493040001C1
:107B30001306200093078001377901801309094358
:107B4000B307F90003A44700138787FF630AE42003
:107B5000832744008326C4000326840093F7C7FFCD
:107B6000B307F40003A747002326D60023A4C600CA
:107B7000136717001385090023A2E700EF00407F79
:107B8000130584006F00801993F487FF63C2071800
:107B900063E0B418EF00807D9307701F63F697468B
:107BA00093D794006386071A13074000636CF73C71
:107BB00093D76400138697031385870393163600C3
:107BC0003779018013090943B306D90003A446009D
:107BD000938686FF638686029305F0006F0000019E
:107BE000635C07320324C400638C8600832744004F
:107BF00093F7C7FF33879740E3D4E5FE13060500EC
:107C0000032409019308890063081417032544001D
:107C10009306F0001375C5FFB307954063CCF6409B
:107C2000232A19012328190163D6073E9307F01F61
:107C300063EAA72E937785FF938787008325490002
:107C4000B307F90083A6070013555500130710006A
:107C50003317A7003367B700938587FF2326B40047
:107C60002324D4002322E90023A0870023A6860032
:107C70009357264093051000B395F5006368B7103D
:107C8000B3F7E50063940702939515001376C6FFDA
:107C9000B3F7E50013064600639A070093951500B5
:107CA000B3F7E50013064600E38A07FE1308F00069
:107CB0001313360033036900130503008327C5003F
:107CC000130E06006302F52E03A747001384070076
:107CD00083A7C7001377C7FFB30697406342D82E28
:107CE000E3C206FE3307E400832647000326840030
:107CF0001385090093E616002322D7002326F600F9
:107D000023A4C700EF00C066130584006F000001C4
:107D10009307C00023A0F900130500008320C102CF
:107D20000324810283244102032901028329C10122
:107D3000032A8101832A4101032B0101832BC10006
:107D4000032C8100832C4100130101036780000094
:107D500093060020130600041305F0036FF05FE69E
:107D600003A4C70013062600E39487DE0324090159
:107D700093088900E31C14E9032749009357264020
:107D800093051000B395F500E37CB7EE032489005A
:107D9000832A440013FBCAFF63689B00B3079B4020
:107DA0001307F0006346F714B7870180B78C018092
:107DB00083AA879D03A78C9C9307F0FF330A640175
:107DC000B38A5401630AF734B71700009387F700AA
:107DD000B38AFA00B7F7FFFFB3FAFA0093850A00F7
:107DE00013850900EF1000799307F0FF930B05004E
:107DF000630CF52863684529378C0180130CCCA6E9
:107E000083250C00B385BA002320BC0093870500AE
:107E10006304AA3A83A68C9C1307F0FF638CE63AAE
:107E2000338A4B41B307FA002320FC0093FC7B000C
:107E300063860C30B7170000B38B9B419385870096
:107E4000938B8B00B3859541B38A5B019387F7FFD2
:107E5000B385554133FAF50093050A0013850900EF
:107E6000EF1040719307F0FF6300F53C3305754157
:107E7000B30A450183250C002324790193EA1A00F3
:107E8000B305BA002320BC0023A25B01630824359C
:107E90009306F00063F866350327440093074BFF11
:107EA00093F787FF137717003367F7002322E40067
:107EB000130650003307F4002322C7002324C70011
:107EC00063EEF63683AA4B0013840B00B78701805C
:107ED00003A7479D6374B70023AAB79CB7870180A7
:107EE00003A7079D6376B71A23A8B79C6F00401AB3
:107EF00013E714002322E400B30494002324990020
:107F000093E717001385090023A2F400EF00404611
:107F1000130584006FF09FE08326C40003268400CD
:107F20006FF01FC493579500130740006372F71456
:107F300013074001636AF7229386C7059385B70547
:107F400093963600B306D90083A70600938686FF72
:107F50006388F61C03A747001377C7FF6376E50025
:107F600083A78700E398F6FE83A6C700032749008E
:107F70002326D4002324F40023A4860023A687000C
:107F80006FF01FCF130740016376F7121307400508
:107F9000636AF71E93D7C4001386F7061385E706B6
:107FA000931636006FF0DFC1130E1E0093773E006C
:107FB00013058500638E07108327C5006FF09FD0DF
:107FC0000326840093E514002322B4002326F60040
:107FD00023A4C700B3049400232A990023289900FE
:107FE00093E7160023A6140123A4140123A2F4008E
:107FF0003307E400138509002320D700EF00403742
:10800000130584006FF09FD113D63400938784004A
:108010006FF09FB23307A400832747001385090040
:1080200093E717002322F700EF0080341305840044
:108030006FF0DFCE13E714002322E400B3049400B2
:10804000232A99002328990013E7170023A6140177
:1080500023A4140123A2E4003305A4002320F50087
:1080600013850900EF00C030130584006FF01FCBAB
:1080700093576500938697039385870393963600FD
:108080006FF05FEC630E241103248900832A4400FF
:1080900093FACAFFB3879A4063E69A001307F00089
:1080A000E348F7E413850900EF00802C1305000076
:1080B0006FF0DFC61386C7051385B7059316360024
:1080C0006FF01FB0832783001306F6FF6392671CCF
:1080D00093773600130383FFE39607FE03274900D7
:1080E00093C7F5FFB3F7E7002322F9009395150036
:1080F000E3EEB7C8E38C05C833F7F500631A070051
:108100009395150033F7F500130E4E00E30A07FEB2
:1081100013060E006FF0DFB9938A0A016FF01FCCCF
:108120000325490093D52540130710003317B700E6
:108130003367A7002322E9006FF09FE3B3855B015B
:10814000B305B0409395450113DA450193050A0044
:1081500013850900EF1000429307F0FFE318F5D0F4
:10816000130A00006FF01FD1130740056362F70880
:108170009357C5009386F7069385E70693963600D6
:108180006FF05FDC130740156362F70893D7F400C4
:108190001386870713857707931636006FF05FA263
:1081A000378C0180130CCCA683270C00B387FA0010
:1081B0002320FC006FF01FC613174A01E31C07C4FD
:1081C00003248900B30A5B0193EA1A0023225401B5
:1081D0006FF0DFCF23A47C9D6FF05FC513840B008D
:1081E0006FF0DFCE9307100023A2FB006FF09FEB30
:1081F000130740156362F7069357F50093868707C8
:1082000093857707939636006FF0DFD313074055B9
:108210006362F70693D724011386D7071385C70730
:10822000931636006FF0DF99938C8CFFB38A9A0116
:10823000B38A7A41130A00006FF0DFC3930584000C
:1082400013850900EFC00FE80324890083250C0083
:10825000832A44006FF09FC7130740556364F702F9
:10826000935725019386D7079385C70793963600C2
:108270006FF05FCD9306803F1306F0071305E0070C
:108280006FF01F949306803F9305E0076FF09FCB3C
:10829000832749006FF09FE59377350093F6F50F3C
:1082A000638A07029307F6FF630E06021306F0FFC8
:1082B0006F0080011305150013773500630E07006A
:1082C0009387F7FF6380C70203470500E314D7FED7
:1082D0006780000093070600130730006366F7020B
:1082E000639607001305000067800000B307F500E0
:1082F0006F00C00013051500E386A7FE03470500C5
:10830000E31AD7FE678000003707010093988500C5
:108310001307F7FFB3F8E80093F5F50FB3E5B800DE
:1083200093980501B3E8B8003708FFFEB785808051
:108330001308F8EF938505081303300003270500A1
:1083400033C7E800330607011347F7FF3377E6002A
:108350003377B700E31C07F89387C7FF1305450081
:10836000E36EF3FCE39407F86FF0DFF7678000003B
:10837000678000008327C504130101FF23248100C7
:10838000232291002326110023202101130405003C
:1083900093840500638E070213952400B387A7001A
:1083A00003A50700630605040327050023A0E700D3
:1083B00023280500232605008320C1000324810013
:1083C000832441000329010013010101678000009B
:1083D0001306100293054000EF50805A2326A40490
:1083E00093070500E31A05FA130500006FF0DFFCA0
:1083F00013091000331999001306590013162600AB
:108400009305100013050400EF508057E30E05FCA0
:1084100023229500232425016FF09FF96380050234
:1084200003A745008327C50413172700B387E70078
:1084300003A7070023A0E50023A0B7006780000082
:10844000130101FE232A910083A4050137030100D3
:10845000232C81002328210123263101232E110002
:1084600023244101138905009309050013840600A4
:1084700013884501930800001303F3FF83270800C6
:108480001308480093881800B3F66700B386C60245
:1084900093D70701B387C702B386860013DE0601B0
:1084A00033F76600B386C701939706013387E70069
:1084B000232EE8FE13D40601E3C298FC63020402F3
:1084C0008327890063D0F40493874400939727009F
:1084D000B307F90023A2870093841400232899008E
:1084E0008320C10103248101832441018329C10028
:1084F000032A810013050900032901011301010268
:1085000067800000832549001385090093851500C5
:10851000EFF05FE6130A0500630C0504032609016A
:108520009305C9001305C50013062600131626007F
:10853000EF50107D0327490083A7C90413172700B4
:10854000B387E70003A707002320E90023A0270142
:108550009387440013090A0093972700B307F90093
:1085600023A2870093841400232899006FF05FF7FB
:10857000B766018037650180938606001306000008
:108580009305500B13054501EF50C038130101FE50
:10859000232C8100232A9100232821012326310145
:1085A000232441011388860093079000232E110095
:1085B000232251013348F80293890600130905006C
:1085C00013840500130A06009304070063D8D70C30
:1085D00093071000930500009397170093851500EB
:1085E000E3CC07FF13050900EFF0DFD89305050082
:1085F000630A050A930710002328F500232A950033
:108600009307900063D64709930A940093840A0065
:108610003304440183C604001306A00013050900B7
:10862000938606FDEFF0DFE19384140093050500C7
:10863000E39284FE13048AFF33848A0063563A036C
:10864000B3894941B3093401834604001306A000ED
:1086500013050900938606FDEFF09FDE1304140056
:1086600093050500E39289FE8320C1010324810163
:1086700083244101032901018329C100032A8100C8
:10868000832A410013850500130101026780000061
:108690001304A400130A90006FF05FFA9305000022
:1086A0006FF05FF4B766018037650180938606003E
:1086B000130600009305E00C13054501EF508025DB
:1086C0003707FFFF3377E500930705001305000028
:1086D000631607009397070113050001370700FF92
:1086E00033F7E700631607001305850093978700AB
:1086F000370700F033F7E70063160700130545005E
:1087000093974700370700C033F7E7006316070069
:10871000130525009397270063C8070013971700D8
:10872000130515006354070067800000130500025D
:1087300067800000832705001307050093F6770084
:108740006384060293F6170013050000639E060675
:1087500093F627006380060893D717002320F700BD
:1087600013051000678000009396070193D6060159
:10877000130500006396060093D707011305000157
:1087800093F6F70F639606001305850093D78700CD
:1087900093F6F700639606001305450093D747004C
:1087A00093F63700639606001305250093D727003C
:1087B00093F61700639C060093D717001305150066
:1087C0006396070013050002678000002320F7006E
:1087D0006780000093D727002320F70013052000AF
:1087E00067800000130101FF23248100138405002A
:1087F0009305100023261100EFF0DFB76300050298
:108800008320C100232A8500032481001307100060
:108810002328E5001301010167800000B76601808D
:108820003765018093860600130600009305001447
:1088300013054501EF50000E130101FE232821010D
:108840002326310103A9050183290601232A91006A
:1088500023244101232E1100232C8100138A0500BB
:1088600093040600634C39011387090093840500C3
:1088700093090900130A06001309070083A784005F
:1088800083A5440033842901B3A78700B385F5008D
:10889000EFF05FAE630C051A130345019318240033
:1088A000B3081301930703006378130123A00700A3
:1088B00093874700E3EC17FF13084A01131E2900B2
:1088C000938E440193952900330EC801B385BE00F1
:1088D000637CC80B93875401130F400063FEF514AB
:1088E000370601001306F6FF6F0000011308480069
:1088F00013034300637AC809832F0800B3F4CF0041
:108900006394040C93DF0F01E3820FFE032703003F
:108910009302030093860E00930407009303000064
:1089200083A7060093D904013377C700B3F7C700C4
:10893000B387F70383A442009382420093864600E4
:1089400033F9C400B3873701B387770093930701E6
:1089500033E7E30023AEE2FE03D7E6FF93D7070138
:108960003307F703330727013307F7009353070152
:10897000E3E8B6FAB307E30123A0E70013084800D1
:1089800013034300E36AC8F7634880006F00800167
:108990001304F4FF6308040083A7C8FF9388C8FF8B
:1089A000E38807FE8320C101232885000324810179
:1089B00083244101032901018329C100032A810085
:1089C00013010102678000009303030093820E00ED
:1089D0001309000003A7020083AF03009383430041
:1089E000B376C700B38696029357070133F7CF00DB
:1089F00093DF0F0193824200B3879702B386E600AC
:108A0000B386260113D70601B3F6C600B387F70174
:108A1000B387E70013970701B366D70023AED3FEF1
:108A200013D90701E3E8B2FAB307E30123A0270152
:108A3000832F08006FF01FED338F9540130FBFFE9B
:108A4000137FCFFF130F4F006FF09FE9B7660180D0
:108A50003765018093860600130600009305D01544
:108A600013054501EF40106B130101FE232C81001B
:108A70002326310123244101232E1100232A9100B2
:108A8000232821019377360013040600930905007B
:108A9000138A05006394070C1354244013090A0039
:108AA0006308040683A48904638E040C937714007E
:108AB00013090A006390070213541440630A040464
:108AC00003A50400630805069304050093771400CA
:108AD000E38407FE1386040093050900138509004B
:108AE000EFF09FD5630809060327490083A7C9044F
:108AF0001354144013172700B387E70003A7070098
:108B00002320E90023A0270113090500E31A04FA32
:108B10008320C10103248101832441018329C100F1
:108B2000032A810013050900032901011301010231
:108B300067800000138604009385040013850900F4
:108B4000EFF09FCF23A0A40023200500930405008D
:108B50006FF0DFF7130905006FF01FF69387F7FF3B
:108B6000376701801307070793972700B307F700BC
:108B700003A6070093060000EFF09F8C130A050080
:108B80006FF09FF19305102713850900EFF09FC543
:108B900023A4A90493040500232005006FF01FF10E
:108BA000130101FE2324410103AA050183A78500C7
:108BB0002326310193595640338A4901232C8100E1
:108BC000232A91002328210123225101232E110061
:108BD00013091A00938405001304060083A54500B9
:108BE000930A050063D82701939717009385150012
:108BF000E3CC27FF13850A00EFF0CFF7630C0510D5
:108C0000130845016354300393895900939929004F
:108C100033073501930708009387470023AE07FE0B
:108C2000E39CE7FE9389C9FE3308380103A70401DA
:108C3000938744011373F401131627003386C7008A
:108C40006304030A93050002B38565409308080096
:108C50009306000003A70700938848009387470006
:108C6000331767003367D70023AEE8FE03A7C7FFBB
:108C7000B356B700E3E0C7FE1387540193074000E3
:108C8000636AE600B30796409387B7FE93F7C7FF82
:108C9000938747003308F8002320D8006384060038
:108CA000130A090003A7440083A7CA048320C10153
:108CB00013172700B387E70003A707002328450100
:108CC0000324810123A0E40023A0970003290101CC
:108CD000832441018329C100032A8100832A4100A2
:108CE000130101026780000003A707009387470074
:108CF00013084800232EE8FEE3F6C7FA03A707008F
:108D00009387470013084800232EE8FEE3EEC7FCD4
:108D10006FF05FF9B76601803765018093860600C2
:108D2000130600009305901D13054501EF40903E8A
:108D30000327050183A70501130805003305F74044
:108D40006314F7049397270013084801938545019E
:108D50003307F800B387F5006F0080006376E80200
:108D60008326C7FF03A6C7FF1307C7FF9387C7FF65
:108D7000E386C6FEB3B6C6003305D0401375E5FFE3
:108D800013051500678000006780000083A70501B8
:108D900003270601130101FF2324810023229100F0
:108DA00023202101232611009384050013040600CB
:108DB0003389E7406394E71A9316270093854501AA
:108DC00013074601B387D5003307D7006F00800033
:108DD00063FCF51803A6C7FF8326C7FF9387C7FF69
:108DE0001307C7FFE306D6FE6360D61683A54400CB
:108DF000EFF04FD86302051A03AE04018322040189
:108E0000938F4401931E2E00130844019392220075
:108E100093034501B708010023262501B38EDF0126
:108E2000B3025800138F030013830F009307000051
:108E30009388F8FF0327030083250800130F4F00D2
:108E4000B3761701B386F600B3F71501B386F64083
:108E500093D5050193570701B387B74013D7064150
:108E6000B387E70013970701B3F61601B366D7007F
:108E700013084800232EDFFE1303430093D7074156
:108E8000E36A58FAB38582409385B5FE1304540112
:108E900093D525001307000063E482001397250093
:108EA0003387E3001308400063E6820093851500D2
:108EB00013982500B38F0F01B383030163FEDF0511
:108EC000B70801001388030093850F009388F8FF0B
:108ED00003A7050013084800938545003376170162
:108EE0003306F6009356064193570701B387D70020
:108EF0009396070133761601B3E6C600232ED8FEFB
:108F000093D70741E3E6D5FD1387FEFFB30FF74183
:108F100013F7CFFF3387E300639A06008327C7FF69
:108F2000130EFEFF1307C7FFE38A07FE8320C1006D
:108F3000032481002328C501832441000329010063
:108F400013010101678000009387040013091000DA
:108F500093040400138407006FF05FE9E34609FE01
:108F6000130900006FF09FE893050000EFF08FC039
:108F7000630205048320C1000324810093071000CD
:108F80002328F500232A050083244100032901003A
:108F90001301010167800000B76601803765018019
:108FA000938606001306000093050024130545016F
:108FB000EF405016B7660180376501809386060042
:108FC000130600009305202313054501EF4090147C
:108FD000B707F07FB3F5B700B707C0FCB385F5005E
:108FE0006358B000930700001385070067800000F6
:108FF000B305B04093D545419307300163C8B7002E
:10900000B7070800B3D5B7406FF0DFFD1387C5FE83
:109010009306E0019305000093071000E3C6E6FC09
:10902000B7070080B3D7E70013850700678000000B
:10903000130101FE232A910083240501232C8100C2
:109040001304450193942400B304940023282101C0
:1090500003A9C4FF2326310123244101130509007C
:1090600093890500232E1100EFF08FE5130700020E
:10907000B307A74023A0F9009307A000138AC4FFF9
:1090800063D0A708130555FF6370440583A784FFC9
:1090900063000504B306A74033D7D7003319A900EE
:1090A0003369E900138684FF3707F03F3367E9002F
:1090B000B397A7006372C40203A644FFB356D60059
:1090C000B3E7D7006F004001930700006314050663
:1090D0003707F03F3367E9008320C1010324810192
:1090E00083244101032901018329C100032A81004E
:1090F0001385070093050700130101026780000034
:109100009306B000B386A640B707F03F3357D900A7
:109110003367F700930700006376440183A784FF59
:10912000B3D7D700130555013315A900B367F50070
:109130006FF09FFA3315A9003707F03F3367E5005A
:10914000930700006FF05FF9130101FD232C41012B
:10915000138A050093051000232291022320210386
:10916000232E31012326110223248102232A5101B7
:10917000930406009389060013090700EFF08F9F00
:10918000630A051093D74401370710001306F7FF51
:1091900093965701130405003376960093FAF77FF0
:1091A000638406003366E6002326C10063080A08CC
:1091B0001305810023244101EFF0CFD70327C1001D
:1091C000930705006302050C032681009306000245
:1091D000B386A640B316D700B3E6C6003357A70040
:1091E000232AD4002326E100B334E0009384140042
:1091F000232CE4002328940063840A06938ADABCB3
:10920000B38AFA001305500323A05901B307F540B0
:109210002320F9008320C1021305040003248102E6
:1092200083244102032901028329C101032A810108
:10923000832A410113010103678000001305C10067
:10924000EFF04FCF930710002328F4008327C100CD
:1092500093041000232AF40093070502E3900AFA0E
:10926000139724003307E400032507019387E7BC25
:1092700023A0F900EFF0CFC493945400B384A4402A
:10928000232099006FF01FF983268100232AD40040
:109290006FF09FF5B7660180376501809386060001
:1092A000130600009305A03013054501EF408066CA
:1092B000130101FD2320210313890500930581007B
:1092C000232611022324810223229102232E31011D
:1092D00093090500EFF0DFD5930405001384050022
:1092E000130509009305C100EFF09FD483270901FE
:1092F00003A709018326C1003307F74083278100B4
:1093000013175700B387D740B307F700930605003C
:10931000635EF0029397470133848700138606004B
:10932000138504009386050093050400EF705039FF
:109330008320C10203248102832441020329010204
:109340008329C101130101036780000013974701BE
:10935000B385E5406FF09FFC130101FF232021013D
:1093600023261100232481002322910093077001FA
:109370001309050063DAA704378701808327879ADA
:109380008325C79A378701800324079B8324479B43
:10939000138507001306040093860400EF80403E07
:1093A0001309F9FF93070500E31409FE8320C100A8
:1093B0000324810083244100032901001385070051
:1093C0001301010167800000B767018013193500A0
:1093D0009387070733892701832709018320C10069
:1093E00003248100832549018324410003290100CE
:1093F0001385070013010101678000008326060121
:109400009385F5FF93D55540938515009307460145
:109410009396260093952500B386D700B305B50033
:1094200063F8D7021307050003A8070093874700D6
:1094300013074700232E07FFE3E8D7FEB387C64094
:109440009387B7FE93F7C7FF938747003305F5006F
:109450006378B50013054500232E05FEE36CB5FEC9
:10946000678000000327050113D655409306450188
:109470006352C70293172700B387F60063F2F6041E
:1094800003A7C7FF9387C7FFE30A07FE1305100072
:109490006780000093172600B387F600E350E6FECE
:1094A00093F5F501E38C05FC03A6070013051000F6
:1094B0003357B600B315B700E302B6FC678000006F
:1094C0001305000067800000130101FF23229100B3
:1094D000B7040080232481002326110093C4F4FFE5
:1094E0001304060023200600B3F6B4003706F07F0D
:1094F000938705001307050063D0C606B3E8A600EE
:10950000638C080433F6C500138805009308000037
:1095100063120602B787018083A6C79B03A6879BB9
:10952000EF8000261307050013880500B3F6B4008A
:109530009308A0FC93D64641B70710809387F7FFA6
:10954000938626C03378F800B3861601B707E03F4C
:10955000B367F8002320D4008320C10003248100D6
:1095600083244100130507009385070013010101BF
:1095700067800000130101FF232481002322910052
:1095800013040500B784018013850500232611000C
:1095900023AA04B0EF700FC89307F0FF630CF50027
:1095A0008320C100032481008324410013010101B1
:1095B0006780000083A744B1E38407FE8320C100D5
:1095C0002320F400032481008324410013010101BE
:1095D00067800000130101F6930EC108232AF108E9
:1095E00037030080B707FFFF138E05001343F3FF17
:1095F0002326D108938787209305810093860E0048
:10960000232E1106232AF1002328E108232C010927
:10961000232E11092324C101232CC101232E610013
:10962000232861002322D101EF00403D83278100E0
:10963000238007008320C1071301010A678000000F
:10964000130E050037850180130101F60325459CA3
:10965000930E8108232AF10837030080B707FFFF24
:109660001343F3FF2324C1082326D10893878720BF
:109670001386050093860E0093058100232E1106A4
:10968000232AF1002328E108232C0109232E1109A4
:109690002324C101232CC101232E61002328610052
:1096A0002322D101EF00803583278100238007002A
:1096B0008320C1071301010A67800000130101FF25
:1096C00023248100138405008395E50023261100DF
:1096D000EF50C00663400502832704058320C100C4
:1096E000B387A7002328F404032481001301010198
:1096F000678000008357C40037F7FFFF1307F7FFA9
:10970000B3F7E7008320C1002316F400032481008F
:10971000130101016780000013050000678000004D
:109720008397C500130101FE232C8100232A910099
:109730002328210123263101232E110013F70710BE
:1097400013840500930405008395E50013090600C2
:1097500093890600631E070237F7FFFF1307F7FF21
:10976000B3F7E7002316F400032481018320C1012D
:1097700093860900130609008329C100032901010A
:109780001385040083244101130101026F40C011BD
:109790009306200013060000EF4090488317C40092
:1097A0008315E4006FF05FFB130101FF23248100A8
:1097B000138405008395E50023261100EF405046F1
:1097C0009307F0FF6304F5028357C40037170000C6
:1097D0008320C100B3E7E7002328A4042316F40084
:1097E0000324810013010101678000008357C40036
:1097F00037F7FFFF1307F7FFB3F7E7008320C10038
:109800002316F40003248100130101016780000086
:109810008395E5006F40C021B367B50093F737002B
:109820006392070803A70500B7867F7F9386F6F744
:10983000B377D700B387D700B3E7E700B3E7D70024
:109840001306F0FF639EC706130605001308F0FF1A
:109850002320E60003A74500938545001306460034
:10986000B377D700B387D700B3E7E700B3E7D700F4
:10987000E38007FF83C7050003C7150083C62500E3
:109880002300F600638A0700A300E60063060700D2
:109890002301D6006394060067800000A301060040
:1098A000678000009307050003C705009387170032
:1098B00093851500A38FE7FEE31807FE678000007D
:1098C000130605006FF01FFB9377350013070500A3
:1098D000639C0704B7867F7F9386F6F79305F0FFB6
:1098E0000326070013074700B377D600B387D700D6
:1098F000B3E7C700B3E7D700E384B7FE8346C7FFEB
:109900000346D7FF8347E7FF3307A740638006047A
:10991000630A06023335F0003305E5001305E5FF61
:1099200067800000E38806FA8347070013071700E3
:1099300093763700E39807FE3307A7401305F7FF38
:10994000678000001305D7FF678000001305C7FF7D
:1099500067800000B3E7A50093F737001307050001
:10996000639807069307300063F4C7063703FFFECA
:10997000B78880801303F3EF93880808130E300034
:1099800083A60500B387660013C8F6FFB3F7070187
:10999000B3F71701639E07022320D7001306C6FF03
:1099A0001307470093854500E36CCEFC93851500B3
:1099B000930717006304060283C6F5FF1308F6FF3A
:1099C000A38FD7FE638E06001387070013060800D7
:1099D0009385150093071700E31006FE67800000CB
:1099E0003306C700630A080093871700A38F07FE9A
:1099F000E39CC7FE6780000067800000130101E15F
:109A00002326111E232A511D2328611D2320A11D59
:109A1000138B0500130D06002326D1002324811E7D
:109A20002322911E2320211F232E311D232C411D73
:109A30002326711D2324811D2322911D232EB11B5A
:109A4000930A0500EFD05FE983270500138507001F
:109A50002320F104EFF05FE78357CB002328010EAA
:109A6000232A010E232C010E232E010E93F7070843
:109A7000232EA1026388070083270B01639407004C
:109A80006F10C05BB767018093878719232AF100A5
:109A900083470D00930BC110B76901802322710F1A
:109AA0002326010E2324010E23280100232C01006C
:109AB00023220104232C0102232401042326010470
:109AC0002322010093880B00938949316380072288
:109AD00013040D00930650026382D73C83471400A1
:109AE00013041400E39A07FEB304A4416300A42105
:109AF0008326C10E8327810E23A0A801B38696007A
:109B00009387170023A298002326D10E2324F10E59
:109B1000930670009388880063CAF63803274100D3
:109B200083470400330797002322E1006380071C6A
:109B300083441400A303010C130414001303F0FF67
:109B4000130A000013090000130CA005930C9000E9
:109B5000930DA00213041400938704FE6364FC04B5
:109B60000327410193972700B387E70083A70700E6
:109B700067800700130A0000938704FD83440400F4
:109B800093162A00338A4601131A1A00338A4701B2
:109B9000938704FD13041400E3F2FCFE938704FE94
:109BA000E370FCFC6384041423069114A303010CEA
:109BB000130C1000930C1000130DC114930D000032
:109BC0001303000023260102232A01022328010295
:109BD000937F290063840F00130C2C00137F490826
:109BE0008327C10E63160F0033088A41E3400073D8
:109BF0008346710C638A06028326810E1306710C5C
:109C000023A0C80093871700130610009386160040
:109C100023A2C8002326F10E2324D10E13067000C0
:109C2000938888006340D660638C0F028326810E80
:109C30001306810C23A0C800938727001306200079
:109C40009386160023A2C8002326F10E2324D10EEA
:109C500013067000938888006354D6006F00107B51
:109C600093060008E302DF4E33039341E34A605A50
:109C700093760910E39E06380327810EB387970178
:109C800023A0A8011307170023A298012326F10E91
:109C90002324E10E9306700063C0E66E938888006B
:109CA0001379490063060900B3048A416346906E44
:109CB00063548A01130A0C0003274100330747014C
:109CC0002322E100E39C07602324010E63880D003A
:109CD00093850D0013850A00EFA0DFBE93880B006B
:109CE000130D040083470D00E39407DE8327C10EA4
:109CF000638407006F1090398357CB0093F70704F4
:109D0000638407006F20803F8320C11E0324811ECF
:109D1000032541008324411E0329011E8329C11DFF
:109D2000032A811D832A411D032B011D832BC11C86
:109D3000032C811C832C411C032D011C832DC11B72
:109D40001301011F6780000013850A00232E1101F3
:109D500023246100EFD05FB88327450013850700F7
:109D60002326F104EFF05FB69307050013850A0080
:109D7000938407002324F104EFD01FB683278500C6
:109D8000032381008328C101232CF1026384040092
:109D90006F10C015834404006FF0DFDB83440400C0
:109DA000136909026FF01FDB136909019377090238
:109DB0006388076C8327C1009387770093F787FF39
:109DC00003A7470083AD0700938787002326F10090
:109DD000930C07006340076E1307F0FF130C090094
:109DE000E30CE30033E79D01137CF9F7E31607006A
:109DF000E31A030013090C0013030000930C000086
:109E0000130D011B138C0C0063D46C00130C0300A6
:109E10008347710C23260102232A01022328010211
:109E2000930D0000E38607DA130C1C006FF05FDA75
:109E30001369090193770902638C07608327C100C6
:109E400013877700137787FF832D0700832C470044
:109E5000930787002326F100137CF9BF1307000046
:109E6000A303010C9306F0FF630AD366B3E69D01DA
:109E70001379FCF7E3980648E31E0312E31E07F686
:109E8000937C1C00130D011BE38E0CF6930700035B
:109E9000A307F11A130DF11A6FF0DFF6B304A44112
:109EA000E318A4C5834704006FF05FC81306410E92
:109EB00093050B0013850A00EF40507EE31E05E278
:109EC00093880B006FF09FC5937789006384070028
:109ED0006F1080078327C1001305010B232E11018A
:109EE0009387770093F787FF83A5070003A64700B2
:109EF00093878700232461002326F100EFB0C04838
:109F00008327010B8328C101032381002328F10E3D
:109F10008327410B232AF10E8327810B232CF10E7B
:109F20008327C10B232EF10E1305010F232E1101E0
:109F300023246100EFD09F932326A10C93072000D8
:109F4000032381008328C1016314F5006F10C05EF4
:109F5000930710006314F5006F109000930710062C
:109F60006394F4006F204012930710046394F4008C
:109F70006F10D04693FCF4FD9307F0FF232C91075C
:109F80006314F3006F109015930770046394FC0042
:109F90006F208017032EC10F23242107832E010F6A
:109FA000032F410F832F810F9367091063540E0015
:109FB0006F20002A232E010613890700930D00004D
:109FC000930760046394FC006F10D0219307500442
:109FD000232411036384FC006F10D029930C130019
:109FE000130C010B1308C10D93860C009307010D90
:109FF0001307C10C1306200093050C0013850A00FB
:10A00000232261022328D10B2320D103232AE10B31
:10A01000232EE101232CF10B2328F101232EC10B68
:10A020002324C101EFC04FD8032E8100832F0101EB
:10A03000032FC101832E01020323410283288102E1
:10A0400033089501130D0500930C010A93850C004C
:10A0500013050C00232E0101232811012324610084
:10A060002328D10B232AE10B232CF10B232EC10B28
:10A070002320010A2322010A2324010A2326010A9C
:10A08000EF70906A0328C101032381008328010136
:10A0900093070800630205028327C10D63FE0701D1
:10A0A0001306000393861700232ED10C2380C700CC
:10A0B0008327C10DE3E807FF0327C10CB387A7413E
:10A0C0002328F1002328E102032781079307700466
:10A0D0006314F7006F105002032781079307600491
:10A0E0006314F7006F1050278327010303278107AC
:10A0F000930510049387F7FF2326F10C93F6F40FD2
:10A10000130600006318B7009386F60093F6F60F67
:10A1100013061000230AD10C9306B00263DA07007D
:10A1200003270103930710009306D002B387E7408B
:10A13000A30AD10C9306900063C4F6006F2000239D
:10A140001308310E130508001306A000130E300685
:10A15000B3E6C70293050500138307001305F5FF57
:10A1600093860603A38FD5FEB3C7C702E3426EFEF4
:10A170009387070313F6F70FA30FC5FE9387E5FF39
:10A1800063E407016F2040339306610D6F00800088
:10A1900003C607002380C600938717009386160026
:10A1A000E39807FF9307510EB387B7401307610D7C
:10A1B000B307F7009306410DB387D7402322F1047C
:10A1C000032701018326410493071000B30CD70035
:10A1D00063C4E7006F20801C8327C103B38CFC009D
:10A1E0008327810613CCFCFF135CFC4113F9F7BFF6
:10A1F0001369091033FC8C0123260102232A010272
:10A20000232801028327C107639407006F1000769B
:10A210009307D002A303F10C13030000130C1C00DE
:10A220006FF01F9B1306410E93050B0013850A0068
:10A2300023206102232EE1012324F101EF40104687
:10A24000E318050A8327C10E03230102032FC1016E
:10A25000832F810093880B006FF01F9D0326810ED2
:10A26000032701019306100023A0A801938717007C
:10A2700093041600938C8800E3DCE632930610000A
:10A2800023A2D8002326F10E2324910E93067000FA
:10A29000E3C6963E0327C10383260104938414007A
:10A2A000B387E70023A0DC0023A2EC002326F10EF5
:10A2B0002324910E93067000938C8C00E3C2963E8B
:10A2C0008326010F138814009305010A2328D10A5D
:10A2D0008326410F1305010B232EF100232AD10AF7
:10A2E0008326810F232401012320010A232CD10A74
:10A2F0008326C10F2322010A2324010A232ED10A17
:10A300002326010AEF7050428327010103288100B0
:10A3100093888C009386F7FF130608008327C101FA
:10A32000E30C052A13071D00B387D70023A0EC0018
:10A3300023A2DC002326F10E2324010F1307700053
:10A34000E34A077713870C0113862400938C0800D7
:10A3500093080700832641041307410D23A0EC0056
:10A36000B387F60023A2DC002326F10E2324C10EBE
:10A3700013077000E356C7921306410E93050B00B6
:10A3800013850A00EF409031631405768327C10ED0
:10A3900093880B006FF0DF90930600010327810E76
:10A3A00063C496006F10D002B7660180938E46306A
:10A3B00013090001930C70006F00C000938404FF28
:10A3C000635A9904938707011307170023A0D80144
:10A3D00023A228012326F10E2324E10E938888006E
:10A3E000E3DEECFC1306410E93050B0013850A0017
:10A3F0002324D101EF40902A631C056E938404FF4F
:10A400008327C10E0327810E832E810093880B00C2
:10A41000E34A99FAB38797001307170023A0D801DE
:10A4200023A298002326F10E2324E10E9306700048
:10A43000E3D0E6881306410E93050B0013850A004E
:10A44000EF40D0256316056A8327C10E6FF05F8643
:10A450008326C1009377090113874600E39E072CEA
:10A4600093770904639407006F10C02D8327C10000
:10A47000930C00002326E10083DD07006FF0DF9DD1
:10A480008326C1009377090113874600E39C0728C0
:10A4900093770904639407006F1000278327C10096
:10A4A0002326E100839D070093DCFD4113870C0008
:10A4B000E35407923337B001B3079041B38CE740C0
:10A4C0001307D002A303E10C9306F0FFB30DB041D4
:10A4D000130C090013071000E31AD3989306100019
:10A4E000630CD710930620006302D72E130D011BB7
:10A4F0001396DC0193F67D0093DD3D009386060301
:10A50000B36DB60193DC3C00A30FDDFE33E69D0185
:10A5100093050D00130DFDFFE31C06FC93771C0053
:10A520006380072E93070003638CF62C9385E5FF69
:10A53000A30FFDFE9307011BB38CB74013090C005A
:10A54000138D05006FF01F8C8327C100A303010C3E
:10A5500003AD070093864700E3060D309307F0FF35
:10A560006314F3006F1080101306030093050000BE
:10A5700013050D00232ED100232611012324610091
:10A58000EFD09FD1032381008328C1008326C1011E
:10A59000930D0500631405006F104056B30CA541E0
:10A5A0008347710C13CCFCFF135CFC412326D100C4
:10A5B00023260102232A01022328010233FC8C01F5
:10A5C000930D000013030000E39007866FF04FE047
:10A5D0000327C100A303010C130C100083270700FD
:10A5E000130747002326E1002306F114930C100003
:10A5F000130DC1146FF08FDCE3940C4E1307900021
:10A60000E360B74F938D0D03A307B11B13090C0033
:10A61000930C1000130DF11A6FF0CFFE8344040069
:10A62000136949006FF00FD39307B002834404000D
:10A63000A303F10C6FF00FD28344040013690908DF
:10A640006FF04FD183440400930614006394B40167
:10A650006F10D061938704FD13840600130300007C
:10A6600063ECFCCE8344040093162300338366001E
:10A67000131313003303F300938704FD1304140032
:10A68000E3F2FCFE6FF04FCD8327C100834404004A
:10A6900003AA0700938747002326F100635C0ACAD8
:10A6A000330A4041136949006FF0CFCA8344040064
:10A6B000136919006FF00FCA8347710C83440400BB
:10A6C000639A07C893070002A303F10C6FF08FC8C9
:10A6D000136C090193770C02638A07768327C10004
:10A6E00013877700137787FF93078700832D070071
:10A6F000832C47002326F100130710006FF04FF65C
:10A700008327C1003787FFFF1347078383AD070007
:10A710002314E10C93874700376701802326F1005B
:10A72000930747BC930C0000136C2900232CF10005
:10A7300013072000930480076FF08FF28344040016
:10A74000136989006FF00FC1834404009307C006AA
:10A75000E386F40C136909016FF0CFBF8344040052
:10A7600093078006E384F408136909046FF08FBE31
:10A770008326C1009377090203A70600938646004B
:10A780002326D1006398077493770901E39A07623F
:10A7900093770904638407006F10C00813790920B8
:10A7A000E300096283274100130D04002300F70032
:10A7B0006FF04FD3930610006314D7006F109013FF
:10A7C00093062000130C0900E312D7D2130D011BCE
:10A7D0008327810193F6FD0093DD4D00B386D700FA
:10A7E00003C606009396CC01B3EDB60193DC4C0092
:10A7F000A30FCDFEB3E69D01130DFDFFE39A06FC0A
:10A800009307011BB38CA74113090C006FF08FDF76
:10A8100093065006E3D496A48326010F9305010AFC
:10A820001305010B2328D10A8326410F232EF100A3
:10A8300023241101232AD10A8326810F2320010A10
:10A840002322010A232CD10A8326C10F2324010AC3
:10A850002326010A232ED10AEF70006D8328810080
:10A860008327C101631C053C0327810EB766018065
:10A87000938646BF23A0D800938717009306100045
:10A880001307170023A2D8002326F10E2324E10E7C
:10A890009306700093888800E3C4E6420327C10C46
:10A8A000832601016350D762032701048326C10375
:10A8B0009388880023ACE8FE0327810EB387D70076
:10A8C00023AED8FE130717002326F10E2324E10E32
:10A8D0009306700063C4E672032701019304F7FF37
:10A8E000635090BC930600010327810EE3DA963E85
:10A8F000930C0001130D70006F00C000938404FFDF
:10A90000E3D09C3E938707011307170023A038016B
:10A9100023A298012326F10E2324E10E93888800B8
:10A92000E35EEDFC1306410E93050B0013850A0050
:10A93000EF40C056631E051A8327C10E0327810E00
:10A9400093880B006FF09FFB33088A41635E00B170
:10A95000130600018326810E635C0607130E0001B7
:10A96000930E70006F00C000130808FF63520E07BB
:10A97000938707019386160023A0380123A2C801FC
:10A980002326F10E2324D10E93888800E3DEDEFC1B
:10A990001306410E93050B0013850A00232E0101B7
:10A9A00023246100EF40804F631405140328C10184
:10A9B000130E00018327C10E130808FF8326810EA2
:10A9C0000323810093880B00930E7000E3420EFB7B
:10A9D000B38707019386160023A0380123A208013C
:10A9E0002326F10E2324D10E1306700093888800CD
:10A9F000635CD6A61306410E93050B0013850A006F
:10AA000023246100EF4080496314050E0323810075
:10AA10008327C10E93880B0033039341635A60A4CC
:10AA2000130600018326810E635866061308000191
:10AA3000130E70006F00C000130303FF635E680411
:10AA4000938707019386160023A0380123A20801EB
:10AA50002326F10E2324D10E93888800E35EDEFCCA
:10AA60001306410E93050B0013850A002324610091
:10AA7000EF40C042631E0506032381001308000156
:10AA80008327C10E130303FF8326810E93880B00D7
:10AA9000130E7000E34668FAB387670093861600CA
:10AAA00023A0380123A268002326F10E2324D10E0F
:10AAB0001306700093888800635CD69A1306410ED3
:10AAC00093050B0013850A00EF40403D6312050219
:10AAD0008327C10E93880B006FF08F991306410EE8
:10AAE00093050B0013850A00EF40403B630E059C65
:10AAF00063840DA093850D0013850A00EF909FDC01
:10AB00006FF08F9F130C09006FF05F9D3767018016
:10AB1000130600018326810E930E4730130E0001A9
:10AB200093027000634806016F004008130808FF95
:10AB3000635E0E07938707019386160023A0D80152
:10AB400023A2C8012326F10E2324D10E9388880066
:10AB5000E3DED2FC1306410E93050B0013850A00B9
:10AB60002324D1032322010323206102232EE101A8
:10AB70002324F101EF408032E31C05F60328410253
:10AB8000130E00018327C10E130808FF8326810ED0
:10AB9000832E810203230102032FC101832F810031
:10ABA00093880B0093027000E3460EF9B387070108
:10ABB0009386160023A0D80123A208012326F10EB4
:10ABC0002324D10E13067000938888006344D600B6
:10ABD0006FF00F821306410E93050B0013850A00D8
:10ABE00023206102232EE1012324F101EF40002BF9
:10ABF000E31005F08327C10E03230102032FC101D7
:10AC0000832F810093880B006FE09FFE1306410E97
:10AC100093050B0013850A00232E61002324E10114
:10AC2000EF40C027E31605EC8327C10E0323C101C3
:10AC3000032F810093880B006FF08F828325C10C56
:10AC4000635CB078032701038326010193040700A6
:10AC500063C6E632635690028326810EB38797005F
:10AC600023A0A8019386160023A298002326F10EA4
:10AC70002324D10E1306700093888800E340D63653
:10AC800093C6F4FF0327010393D6F641B3F4D4002F
:10AC9000B30497406348903E03270103937609402D
:10ACA000B304ED00639406448325C10C032701011E
:10ACB00063C6E50093761900E38606348326010413
:10ACC0000327C1031306700023A0D8008326810E3A
:10ACD000B387E70023A2E800938616002326F10E2F
:10ACE0002324D10E93888800E34CD64C832601019F
:10ACF0003307DD003386B64033079740930C0600D8
:10AD00006354C700930C0700635690030327810E1A
:10AD1000B387970123A098001307170023A2980177
:10AD20002326F10E2324E10E9306700093888800F9
:10AD3000E3CCE65E13C7FCFF1357F74133F7EC0093
:10AD4000B304E640634490006FE09FF59306000172
:10AD50000327810E63D69678930C0001130D7000C3
:10AD60006F00C000938404FF63DC9C769387070127
:10AD70001307170023A0380123A298012326F10E00
:10AD80002324E10E93888800E35EEDFC1306410E58
:10AD900093050B0013850A00EF404010E31A05D419
:10ADA0008327C10E0327810E93880B006FF09FFB52
:10ADB00093751900639405CC23A2D8002326F10EC5
:10ADC0002324910E130770006346974E1306260046
:10ADD000938808016FF00FD8635ED0D61307000187
:10ADE0006344D7006F100068130D70006F000001FE
:10ADF000938606FFE350D70C13881400938707014E
:10AE000023A03C0123A2EC002326F10E2324010FF2
:10AE100093040800938C8C00E35C0DFD1306410E37
:10AE200093050B0013850A002324D100EF4000078F
:10AE3000E31005CC8327C10E8324810E8326810075
:10AE4000938C0B00130700016FF09FFA8326C1005B
:10AE500093770C0113874600639C070A93770C04D1
:10AE6000E38407088327C100930C00002326E10038
:10AE700083DD0700130710006FE09FFE1306410EED
:10AE800093050B0013850A00EF404001E31205C64D
:10AE90008327C10E8324810E938C0B006FF08FBF2C
:10AEA0001306410E93050B0013850A00EF30107F47
:10AEB000E31005C48327C10E8324810E938C0B00FD
:10AEC0006FF00FC013771900631407006FE05FDDA8
:10AED0006FF09F9D83264100130D040093D7F64128
:10AEE0002320D7002322F7006FE0DFDF83278103D1
:10AEF00083440400639407006FE0DFC583C7070045
:10AF0000639407006FE01FC5136909406FE09FC499
:10AF10002326E10083AD0600930C00001307100008
:10AF20006FE01FF483AD06002326E10093DCFD41B2
:10AF300013870C006FE01FEA83AD0600930C00003E
:10AF40002326E1006FE05FF10327C100832707009C
:10AF5000130747002326E10083A5070003A6470047
:10AF600083A6870083A7C7002328B10E232AC10E1A
:10AF7000232CD10E232EF10E6FE01FFB93840600CD
:10AF8000E34C90CC6FF0DFCF130C09006FF08FF41F
:10AF9000B7670180938747BC232CF10093770902A0
:10AFA0006386072C8327C10013877700137787FFF9
:10AFB000832D0700832C4700930787002326F10089
:10AFC00013771900630E070033E79D01630A07003A
:10AFD000130700032304E10CA304910C1369290057
:10AFE000137CF9BF130720006FE09FE78344140030
:10AFF00013690920130414006FE0DFB51306410E36
:10B0000093050B0013850A00EF305069E31205AE7B
:10B010008327C10E93880B006FF01F8C83441400AC
:10B0200013690902130414006FE0DFB2B7670180EF
:10B03000938787BD232CF1006FF05FF69305000422
:10B0400013850A00EFC0DFA92320AB002328AB0043
:10B05000631405006F10C04393070004232AFB000C
:10B060006FE05FA293076000930C030063E86778CA
:10B0700037670180138C0C002326D100130DC7BE47
:10B080006FE0DFB3130600018326810E635A966ECC
:10B09000930C0001130870006F00C000938404FF3C
:10B0A00063D09C6E938707019386160023A0380116
:10B0B00023A298012326F10E2324D10E9388880021
:10B0C000E35ED8FC1306410E93050B0013850A00BE
:10B0D000EF30D05CE31E05A08327C10E8326810ECE
:10B0E00093880B00130870006FF05FFB03270101CA
:10B0F000130E7000130800013307ED002324E10054
:10B1000003274103630E070A0327C102631E070AD0
:10B11000032781031307F7FF232CE10203274103D1
:10B120001307F7FF232AE1028326C10403278104C2
:10B130009388880023ACD8FE8326810EB387E7006E
:10B1400023AEE8FE938616002326F10E2324D10EAB
:10B15000634EDE1203278103834607000327810025
:10B16000938C0600330697406354D600930C060078
:10B17000635890038326810EB387970123A098001C
:10B180009386160023A298012326F10E2324D10EC4
:10B19000634CDE36032781039388880083460700CB
:10B1A00013C6FCFF1356F641B3FCCC00B38C96419A
:10B1B00063449003B384D40003274103E31607F4E8
:10B1C0000327C102630007720327C1021307F7FFB9
:10B1D0002326E1026FF05FF58326810E6348980114
:10B1E0006F00C005938C0CFF635A98059387070185
:10B1F0009386160023A0380123A208012326F10E0E
:10B200002324D10E93888800E35EDEFC1306410EF2
:10B2100093050B0013850A00EF305048E31A058CA4
:10B2200013080001938C0CFF8327C10E8326810E27
:10B2300093880B00130E7000E34A98FBB3879701C5
:10B240009386160023A0380123A298012326F10E2D
:10B250002324D10E6346DE7203278103938888007E
:10B2600083460700B384D4006FF01FF58326C10026
:10B2700093770901138746006386072283AD060092
:10B28000930C00002326E1006FF09FD31306410EBC
:10B2900093050B0013850A00EF305040E31A058434
:10B2A0008327C10E93880B0013080001130E700052
:10B2B0006FF05FEA1306410E93050B0013850A0039
:10B2C000EF30D03DE31605820326810E8327C10EA1
:10B2D0009308411113061600938C0B006FF08F87B3
:10B2E00013790C4023280100130D011B6F0040034C
:10B2F0001306A0009306000013850D0093850C0033
:10B30000232E110123246100EF50403703238100D5
:10B310008328C10163880C4A930D0500938C0500B6
:10B320001306A0009306000013850D0093850C0002
:10B33000232E110123246100EF5080778327010120
:10B3400013050503A30FADFE938717002328F10013
:10B35000032381008328C101130DFDFFE30A09F8CF
:10B360000327810383460700E394D7F81307F00F00
:10B37000E380E7F863960C009307900063F2B7C987
:10B38000832781048325C104232E1101330DFD4041
:10B390001386070013050D0023246100EFE08FDB07
:10B3A000832781031306A0009306000003CE170035
:10B3B00013850D0093850C00333EC001B387C70190
:10B3C000232CF102EF50802B032381008328C1013D
:10B3D000232801006FF05FF48326810E3766018019
:10B3E000130646BF23A0C80093871700130610005A
:10B3F0009386160023A2C8002326F10E2324D10E23
:10B400001306700093888800634CD6066392051C6F
:10B410000327010193761900B3E6E6006394060062
:10B420006FE01F88832601040327C1031306700001
:10B4300023A0D8008326810EB387E70023A2E8006B
:10B44000938616002326F10E2324D10E6342D6469E
:10B4500093888800032701019386160023A0A80182
:10B46000B387E70023A2E8002326F10E2324D10EA0
:10B47000130770006344D7006FE05F826FE0DFEF77
:10B480001306410E93050B0013850A00EF301021BF
:10B49000631005E68325C10C8327C10E93880B003A
:10B4A0006FF0DFF693770904638007288327C100D4
:10B4B000930C00002326E10083DD07006FF05FB0EE
:10B4C0001306410E93050B0013850A00EF30101D83
:10B4D000631005E28327C10E93880B006FF00FBC49
:10B4E00023A0380123A29800B38797001307170001
:10B4F0002326F10E2324E10E9306700063C4E600B8
:10B500006FE0CFF96FE05FE71306410E93050B0084
:10B5100013850A00EF309018631C05DC8327810334
:10B5200093880B001308000183C60700130E7000F8
:10B530008327C10E6FF0DFC68327010F9305010A31
:10B540001305010B2328F10A8327410F232411013E
:10B550002320010A232AF10A8327810F2322010ACB
:10B560002324010A232CF10A8327C10F2326010A71
:10B57000232EF10AEF60D04283288100634C0542FC
:10B580008347710C13077004635497243767018055
:10B59000130D87BB23260102232A0102232801025F
:10B5A0001379F9F7130C3000930D0000930C300061
:10B5B00013030000638407006FE01F876FE04FE113
:10B5C00083274100130D04002320F7006FE08FF163
:10B5D000832601040327C1031306700023A0D800AB
:10B5E0008326810EB387E70023A2E8009386160026
:10B5F0002326F10E2324D10E93888800634AD62A8D
:10B60000E3DA05E4130600FFB304B040E3D6C5282F
:10B61000930C0001130870006F00C000938404FFB6
:10B62000E3DC9C26938707019386160023A038014C
:10B6300023A298012326F10E2324D10E938888009B
:10B64000E35ED8FC1306410E93050B0013850A0038
:10B65000EF30D004631E05C88327C10E8326810EF8
:10B6600093880B00130870006FF05FFB13050D004B
:10B67000232411012326D100EFE00FA58347710C8D
:10B68000134CF5FF135CFC4123260102232A01021F
:10B690002328010283288100930C0500337C850157
:10B6A000930D000013030000638407006FE0CFF7E1
:10B6B0006FE00FD21386140013878C00B387D70076
:10B6C00023A2DC0023A03C012326F10E2324C10E7B
:10B6D00093067000E3C0C6BE1306160093088700E9
:10B6E000930C07006FE01FC793770C206384071843
:10B6F0008327C100930C00002326E10083CD0700BF
:10B70000130710006FE0CFF59377092063880714C3
:10B710008327C1002326E100838D070093DCFD41D0
:10B7200013870C006FE00FEB93770920638E0710EF
:10B730008327C100930C00002326E10083CD07007E
:10B740006FF01F88937709206386070E8327C10057
:10B75000930C00002326E10083CD07006FE0CFEFBC
:10B760008327C10F63C007148347710C130770044C
:10B770006352974237670180130D07BC6FF09FE15A
:10B78000B38797009386160023A0380123A2980060
:10B790002326F10E2324D10E13067000938888000F
:10B7A000635CD6CE1306410E93050B0013850A0089
:10B7B000EF30C06E631E05B28327C10E93880B0065
:10B7C0006FF08FCD93079000E3E8B7B56FF04F832C
:10B7D00037670180130D47BB6FF0DFDB1306410EA7
:10B7E00093050B0013850A00EF30406B631205B020
:10B7F0008327C10E93880B006FF08FC8930C6000F5
:10B800006FF01F87832601013307DD003386B640C2
:10B8100033039740930C0600635EC3D0930C030080
:10B820006FF04FD183274100130D04002310F70060
:10B830006FE04FCB8327C100930C00002326E1006B
:10B8400083AD07006FE04FE18327C100930C000038
:10B850002326E10083AD07006FF08FF68327C10038
:10B860002326E10083AD070093DCFD4113870C0024
:10B870006FE04FD68327C100930C00002326E10020
:10B8800083AD0700130710006FE08FDD1306410E34
:10B8900093050B0013850A00EF3040608357CB00FF
:10B8A0006FE0CFC59307D002A303F10C6FF01FEC3C
:10B8B0001306410E93050B0013850A00EF30005E5E
:10B8C000631805A28325C10C8327C10E8326810E30
:10B8D00093880B00E3D005B86FF0DFD2130360004C
:10B8E0006FE04FEB03270101B306ED0063FE96BA4C
:10B8F000938406006FF04FBB032701039307D0FF2B
:10B900006344F700635AE3009384E4FF93F7F4FD84
:10B91000232CF1066FE04FFD83270101032701036C
:10B920006340F72883278106930C070093F71700DD
:10B93000638607008327C103B30CF70083278106C2
:10B9400093F707406386070083270103E340F0066F
:10B9500013CCFCFF135CFC4133FC8C019304700698
:10B9600023260102232A01026FE0DF898347710C3D
:10B9700013030000638407006FE00FCB6FE04FA557
:10B980001306410E93050B0013850A00EF3000519A
:10B99000631005968327810393880B001308000129
:10B9A00083C60700130E70008327C10EB384D40032
:10B9B0006FF09F809307D002A303F10C6FF09FBC40
:10B9C0001306410E93050B0013850A00EF30004D5E
:10B9D000631005928325C10C8327C10E93880B0049
:10B9E0006FF0CFB0130C010B930603001308C10DC9
:10B9F0009307010D1307C10C1306300093050C00CB
:10BA000013850A0023241103232261022328D10B6A
:10BA10002320D103232AE10B232EE101232CF10B58
:10BA20002328F101232EC10B2324C101EFA0DFB78E
:10BA3000032E8100832F0101032FC101832E0102F8
:10BA40000323410283288102130D0500930760043C
:10BA500033086D00639CFC6883460D009307000368
:10BA6000E388F614930C010A8327C10C3308F8000D
:10BA70006FE0CFDD130C010B9307010D930603005C
:10BA80001308C10D1307C10C1306200093050C0009
:10BA900013850A00232261022328D10B2320D1031E
:10BAA000232AE10B232EE101232CF10B2328F101A2
:10BAB000232EC10B2324C101EFA01FAF93077004F5
:10BAC000032E8100832F0101032FC101832E010268
:10BAD0000323410283288102130D0500E398FCF63D
:10BAE0008327810693F71700639C075E1307700492
:10BAF0008327C10D232CE1066FE00FDC8347710C17
:10BB00002326D10023260102232A01022328010231
:10BB1000130C0300930C030013030000638407005D
:10BB20006FE08FB06FE0CF8A1306410E93050B00D4
:10BB300013850A00EF308036630405006FE05FFB79
:10BB40008324C10C032701018327C10E93880B00B6
:10BB5000330697406FF00F9E83278106032701036A
:10BB600093F71700B3E76700E354E00C6398076CA2
:10BB7000832C0103930460068327810693F7074013
:10BB80006398076213CCFCFF135CFC4133FC8C010F
:10BB90006FF01FDD37670180130DC7BB6FF09F9FEC
:10BBA000832701010327C10393047006B38CE700C8
:10BBB00083270103E342F0FCB38CFC40938C1C0010
:10BBC00013CCFCFF135CFC4133FC8C016FF05FD99C
:10BBD000B7660180938E46306FE0DF8393070003E2
:10BBE0002304F10C9307800513672900A304F10CCB
:10BBF0002324E10693073006930D0000130DC114B2
:10BC000063CE6744032EC10F93FCF4FD232C9107F0
:10BC1000232E0106832E010F032F410F832F810F47
:10BC20001369291063420E3C930710066388F4627F
:10BC3000930710046384F4006FE08FB8130C010BBA
:10BC400013050C0023261103232461022328D10BA2
:10BC5000232AE10B232CF10B232EC10BEF9050155F
:10BC60001306C10CEFD05F8613860500930505000F
:10BC700013050C00EF9040719307010993850700AD
:10BC80002324F1008327010B930C010A13060108FA
:10BC90002328F1088327410B13850C002326C106B6
:10BCA000232AF1088327810B23200108232201087E
:10BCB000232CF1088327C10B23240108232EF1082C
:10BCC000B707FC3F2326F108EF6040620328010A12
:10BCD000032E410A832E810A032FC10A93850C008B
:10BCE00013050C002328010B23220103232AC10B77
:10BCF0002320C103232CD10B232ED101232EE10BB2
:10BD00002328E1012320010A2322010A2324010A16
:10BD10002326010AEF604021032F0101832EC10178
:10BD2000032E010203284102032381028328C1025A
:10BD300063160500930710002326F10CB7670180F6
:10BD4000938787BD2322F1069306F3FF93070D0027
:10BD50006F00400993850C0013050C002320C106D9
:10BD6000232EF105232C5104232A71042328F104E6
:10BD7000232A1103232861022328710A2326710232
:10BD8000232A510A23245102232CF10B2322F103ED
:10BD9000232EC10A2320C1022320010A2322010AE3
:10BDA0002324010A2326010AEF6000188326C1011B
:10BDB000032F0102832E4102032E81020328C102B8
:10BDC00003230103832841038327010583234105BE
:10BDD00083228105832FC105032601069386F6FF82
:10BDE000630E05100326810093850C00232AF102BF
:10BDF00013050C00B70703402328D104232811039F
:10BE000023266102232EF1082326E10B2320010BB8
:10BE10002322C10B2324D10B23280108232A010844
:10BE2000232C0108EF60804C832E010B032E410B65
:10BE30000328810B0326C10B13050C002324D10317
:10BE40002322C10323200103232EC100EF900024ED
:10BE5000930505002328A10013050C00EF90C03DB9
:10BE60000326C101832E8102032E4102232EC10825
:10BE70000326010B03280102832581002320C1082A
:10BE80000326410B13850C002328D1092322C10866
:10BE90000326810B232AC109232C01092324C1086D
:10BEA0000326C10B2326C1080326C106EF7080714B
:10BEB0000327410683270101832601058323010A05
:10BEC0003306F70083450600832741038322410A96
:10BED000832F810A0326C10A232AF1062380B70093
:10BEE0002328D1061307F0FF232ED1000323C1021C
:10BEF0008328010393871700E39EE6E4B706FE3F1D
:10BF000093850C0013050C002320F102232E110150
:10BF1000232461002328710A23287102232A510A4D
:10BF200023265102232CF10B2324F103232EC10AD3
:10BF30002322C1022320010A2322010A2324010A09
:10BF40002326D10AEF600011032381008328C10159
:10BF5000832701026344A00A832301038322C102D1
:10BF6000832F810203264102B706FE3F93850C0012
:10BF700013050C002328710A232A510A232CF10BE4
:10BF8000232EC10A2320010A2322010A2324010AA5
:10BF90002326D10AEF505079032381008328C10161
:10BFA0008327010263180500032701019376170018
:10BFB0006396060403270107130600039306170080
:10BFC000B386D700635407006FE00F8F9387170085
:10BFD000A38FC7FEE39CD7FE6FE00F8E23242107BB
:10BFE000930D000013890200B707008033CEC7010C
:10BFF0009307D002232EF1066FF01FC303274107DA
:10C0000093860700232EE10C0327410603C6F7FFA2
:10C010008345F7006310B60213050003A38FA6FE45
:10C020008326C10D1386F6FF232EC10C03C6F6FF2F
:10C03000E386C5FE930516001305900393F5F50FEF
:10C040006306A600A38FB6FE6FE00F8703274106A5
:10C050008345A700A38FB6FE6FE00F8693051300FC
:10C0600013850A002328110123246100EFB05FA784
:10C070000323810083280101130D05006304054299
:10C08000930D05006FF01FB8930700032304F10C14
:10C09000930780076FF05FB5B3879700938616000C
:10C0A00023A0380123A298002326F10E2324D10EC9
:10C0B00013067000635ED6B81306410E93050B009D
:10C0C00013850A00EF20905D630405006FE05FA216
:10C0D0008327C10E8326810E93880B006FF08FB7E4
:10C0E0009307700433086D00232CF106930C010AAA
:10C0F0006FD0DFF5130C09006FE0CFD09307F0FF8E
:10C100002322F1006FD05FC06314030013031000FB
:10C11000032EC10F832E010F032F410F832F810F99
:10C1200093620910E34C0EEA130C010B9306030013
:10C130001308C10D9307010D1307C10C130620004E
:10C1400093050C0013850A002326510223241103B2
:10C15000232261022328D10B2320D103232AE10BC0
:10C16000232EE101232CF10B2328F101232EC10BF7
:10C170002324C101EFA04FC38322C102232421073E
:10C18000032E8100832F0101032FC101832E0102A1
:10C190000323410283288102130D05001389020045
:10C1A000930D0000232E01066FF09F9393047006F9
:10C1B000832781039306F00F2326010283C707001C
:10C1C000232A01026388D7040327010363D4E70409
:10C1D000B307F740032781032328F10283471700A1
:10C1E000638E07000326410313071700232CE10287
:10C1F00013061600232AC1026FF0DFFC0327C102D9
:10C20000832781031307170083C707002326E10252
:10C210006FF05FFB0327C10283274103B387E70069
:10C2200003278104B387E702B38C970113CCFCFF8B
:10C23000135CFC4133FC8C016FD0DFFC8327C1030E
:10C2400093046006B30CF700B38C6C006FF0DF92C0
:10C25000930D0000138907006FF01FD9130C010B19
:10C2600013050C0023261103232461022328D10B7C
:10C27000232AE10B232CF10B232EC10BEF9040332B
:10C280001306C10CEFD04FA41386050093050500DB
:10C2900013050C00EF90400F9307010993850700E9
:10C2A0002324F1008327010B930C010A13060108D4
:10C2B0002328F1088327410B13850C002326C10690
:10C2C000232AF1088327810B232001082322010858
:10C2D000232CF1088327C10B23240108232EF10806
:10C2E000B707FC3F2326F108EF6040000328010A4E
:10C2F000032E410A832E810A032FC10A93850C0065
:10C3000013050C002328010B23220103232AC10B50
:10C310002320C103232CD10B232ED101232EE10B8B
:10C320002328E1012320010A2322010A2324010AF0
:10C330002326010AEF50503F032F0101832EC10134
:10C34000032E010203284102032381028328C10234
:10C3500063160500930710002326F10CB7670180D0
:10C36000938747BC2322F1066FF01F9E9306610D51
:10C370006318060093060003230BD10C9306710D7E
:10C380001307011B938707033386E6402380F600DB
:10C390009307D60D2322F1046FD09FE283278106F5
:10C3A00093F71700639407006FD09FE36FD0DFE22D
:10C3B000930C010A93850C0013050C00232601033E
:10C3C00023241103232261022328D10B2320D1032C
:10C3D000232AE10B232EE101232CF10B2328F10169
:10C3E000232EC10B2324C1012320010A2322010A89
:10C3F0002324010A2326010AEF501033032E810063
:10C40000832F0101032FC101832E01020323410267
:10C41000832881020328C102630805E49307100002
:10C42000B38767402326F10C3308F8006FD01FC292
:10C43000639A0700130C100093046006930C10001D
:10C440006FF00FD28327C10393046006938C17000B
:10C45000B38C6C0013CCFCFF135CFC4133FC8C01EF
:10C460006FF00FD0138708006FF04FA58327C1002E
:10C4700003A3070093874700635403001303F0FFEF
:10C48000834414002326F100138406006FD08FEC40
:10C490009307C00023A0FA009307F0FF2322F100C6
:10C4A0006FD09F868357CB0013E7070493070700DD
:10C4B0002316EB006FD09F84930720002322F10402
:10C4C0006FD01FD083A74506130101FD232861010A
:10C4D00023261102232481022322910223202103F7
:10C4E000232E3101232C4101232A510123267101DE
:10C4F0002324810113972701130B06006358070AB1
:10C5000083278600832B0600138905009309050005
:10C51000930AF0FF6388070803AC4B0003A40B00E9
:10C52000135A2C0063060A06930400006F00C00033
:10C5300013044400630C9A048325040013060900C5
:10C5400013850900EF10100293841400E31255FFC5
:10C550001305F0FF8320C1020324810223240B0072
:10C5600023220B0083244102032901028329C101F4
:10C57000032A8101832A4101032B0101832BC1007E
:10C58000032C8100130101036780000083278B00C7
:10C59000137CCCFFB38787412324FB00938B8B0054
:10C5A000E39C07F6130500006FF0DFFAEF10D00CE4
:10C5B0006FF05FFA03278600630407006FF09FF0B7
:10C5C000232206001305000067800000130101ED1F
:10C5D000232E3111232A51112320A11123261112B8
:10C5E000232481122322911223202113232C411171
:10C5F00023286111232671112324811123229111F3
:10C60000232EB10F2326D100930A0500938905003C
:10C61000130D060063060500832785036388076AF8
:10C620000397C900931707019316270193D70701B2
:10C6300063CA0602B727000083A64906B367F7005E
:10C640009397070137E7FFFF93D707411307F7FFDA
:10C6500033F7E6002396F9009397070123A2E90632
:10C6600093D7070113F787006304073E03A7090167
:10C670006300073E93F7A7011307A000638AE73E14
:10C68000B76701809304C10493874732B76B018079
:10C69000376901802320910423240104232201040B
:10C6A000138704002328010023220102232401020E
:10C6B0002326010223240100232AF100938B0B4936
:10C6C0001309094A83470D00638E072413040D00E4
:10C6D000930650026386D742834714001304140064
:10C6E000E39A07FE330AA441630EA4238326810440
:10C6F000832741042320A701B306DA00938717009C
:10C70000232247012324D1042322F10413067000BD
:10C71000130787006350F602E3840636130601040C
:10C720009385090013850A00EFF0DFD96310052017
:10C73000138704008326810083470400B3864601E3
:10C740002324D1006380071E83461400130D1400B8
:10C75000A30D0102930CF0FF13040000930D0000E1
:10C76000130AA005130C9000130BA002130D1D005B
:10C77000938706FE6364FA0403264101939727001A
:10C78000B387C70083A70700678007001304000072
:10C79000938706FD83460D0093152400338485009E
:10C7A0001314140033848700938706FD130D1D00B6
:10C7B000E372FCFE938706FEE370FAFC63840616C0
:10C7C0002306D108A30D0102130A1000130C100058
:10C7D000130BC108930C000093FF2D0063840F001E
:10C7E000130A2A008326410413FF4D08832781047E
:10C7F000138616009305060063160F0033084441A4
:10C80000E34400170345B10313068700630C0502D8
:10C810009306B1032320D7009387170093061000D7
:10C820002322D7002324F1042322B104130770002C
:10C83000E342B70C938605001307060093851500A5
:10C8400013068600638E0F049306C1032320D700CE
:10C8500093872700930620002322D7002324F10486
:10C860002322B10413077000E352B70EE3840726B6
:10C87000130601049385090013850A00232CE101A6
:10C88000EFF05FC46314050A832641048327810403
:10C89000032F8101130641059385160013870400B9
:10C8A000130500086306AF68B38C8C416342907730
:10C8B000B307FC0023206701232287012324F1040E
:10C8C0002322B104130770006352B7026382072466
:10C8D000130601049385090013850A00EFF09FBE3B
:10C8E00063160504832781041386040093FE4D001C
:10C8F00063860E00330C4441634880236354440133
:10C9000013040A0003278100330787002324E10072
:10C91000639E077A83470D002322010413870400D6
:10C92000E39607DA83278104E396076283D7C90079
:10C9300093F70704E39E07648320C1120324811246
:10C940000325810083244112032901128329C11187
:10C95000032A8111832A4111032B0111832BC1105A
:10C96000032C8110832C4110032D0110832DC10F46
:10C97000130101136780000013850A00232CE100D6
:10C98000EFA09FF583274500138507002326F102BA
:10C99000EFC09FF39307050013850A002324F102DB
:10C9A000EFA09FF303278500832781022322E10262
:10C9B00003278101E398072A83460D006FF01FDBF0
:10C9C00083460D0093ED0D026FF05FDA93ED0D01DC
:10C9D00093F70D02638A07228327C100138B770028
:10C9E000137B8BFF83264B00032C0B0093078B00DC
:10C9F0002326F1001388060063C006249306F0FF87
:10CA0000138A0D006388DC00B3660C0113FAFDF78E
:10CA1000E38E0606E318081293069000E3E48613FB
:10CA200093070C03A307F10E930D0A00130C1000DB
:10CA3000130BF10E138A0C0063D48C01130A0C0043
:10CA40008347B103B337F000330AFA006FF0DFD841
:10CA50009385090013850A00EF70CFD7E31A0552BA
:10CA600083D7C9001307A00093F7A701E39AE7C093
:10CA70008397E900E3C607C08326C10013060D00B3
:10CA80009385090013850A00EF0010562324A100A6
:10CA90006FF09FEA93ED0D0193F70D026380071489
:10CAA0008327C100138B7700137B8BFF032C0B00B4
:10CAB00003284B0093078B002326F10013FAFDBFD8
:10CAC00093060000A30D01021306F0FF638ACC1841
:10CAD00033660C01937DFAF76314066863960C3E87
:10CAE000639A067A137C1A00130B010FE3040CF40B
:10CAF00093070003A307F10E130BF10E6FF09FF3E2
:10CB0000330AA441E314A4BF834704006FF09FC31A
:10CB10002322010493FE4D0063800E72330C4441C6
:10CB2000635C8071138604001307000183264104AF
:10CB3000E3588745930C0001130B70006F008001D0
:10CB4000938526001306860093060700130C0CFF3E
:10CB500063D88C059387070113871600232076017D
:10CB6000232296012324F1042322E104E35AEBFC5F
:10CB70006388073A130601049385090013850A00A8
:10CB8000EFF05F94E31405DA83264104130C0CFFE5
:10CB9000832781041386040093851600E3CC8CFB65
:10CBA000B387870123207601232286012324F10401
:10CBB0002322B10413077000E352B7D4638E0766D3
:10CBC000130601049385090013850A00EFF09F8F77
:10CBD000E31E05D4832781046FF05FD20326C100D2
:10CBE00093F70D0193064600E390070C93F70D04AD
:10CBF000E38E07248327C100130800002326D100F9
:10CC000003DC07006FF09FEB0326C10093F70D01D3
:10CC100093064600E390070893F70D04E388072086
:10CC20008327C1002326D100039C07001358FC4131
:10CC300093060800E3D406DCB336800133080041D4
:10CC40003308D8409306D002A30DD1021306F0FF9B
:10CC5000330C8041138A0D0093061000E39ACCE652
:10CC600013061000E388C6DA130620006388C62680
:10CC7000130B010F1316D80193767C0093573C00D9
:10CC800093860603336CF60013583800A30FDBFEBF
:10CC900033660C0193050B00130BFBFFE31C06FC32
:10CCA00093771A0063860726930700036382F626AC
:10CCB0009385E5FFA30FFBFE9307010F338CB7406D
:10CCC000930D0A00138B05006FF0DFD6EF701FA7DE
:10CCD0006FF01F958327C100A30D010203AB07006E
:10CCE00093864700E3040B129307F0FFE38CFC06E6
:10CCF00013860C009305000013050B00232CD100B4
:10CD00002326E100EFB04FD90327C100832681011C
:10CD1000E30C0524330C65412326D100930C00005D
:10CD20006FF05FD18326C100A30D0102130A10002A
:10CD300083A70600938646002326D1002306F10828
:10CD4000130C1000130BC1086FF0DFA883460D0011
:10CD50009307C006E38EF60893ED0D016FF01FA157
:10CD600083460D0093078006E38CF60693ED0D04D1
:10CD70006FF0DF9F13EA0D0193770A026384075275
:10CD80008327C10093061000138B7700137B8BFF62
:10CD900093078B00032C0B0003284B002326F10084
:10CDA0006FF05FD283460D0093ED0D086FF01F9C6E
:10CDB0008327C10013EA2D00B786FFFF03AC0700ED
:10CDC000B76D01809387470093C606832326F10041
:10CDD00093874DBC231ED102130800002328F100C5
:10CDE000930620006FF01FCE0326C10093F70D02BB
:10CDF00083260600130646002326C10063920768B7
:10CE000093F70D01639E077E93F70D04E392070EDF
:10CE100093FE0D2063860E7E832781002380F6001B
:10CE20006FF05F8A8327C10083460D0003A40700CB
:10CE3000938747002326F100E35A0492330480408D
:10CE400093ED4D006FF09F9283460D0093ED1D0012
:10CE50006FF0DF918347B10383460D00E39807909D
:10CE600093070002A30DF1026FF05F9083460D005F
:10CE700093ED4D006FF09F8F9307B00283460D0036
:10CE8000A30DF1026FF09F8E83460D0093051D00E8
:10CE9000E38C6611938706FD138D0500930C00004B
:10CEA000E368FC8C83460D0013982C00330898012E
:10CEB00013181800B30CF800938706FD130D1D001E
:10CEC000E372FCFE6FF0DF8A13061000E38EC60AE1
:10CED00013062000138A0D00E39CC6D8130B010F24
:10CEE000832701019376FC00130BFBFFB386D70069
:10CEF00003C6060093574C009316C80133ECF600A6
:10CF0000135848002300CB00B3660C01E39A06FCDB
:10CF10009307010F338C6741930D0A006FF09FB1A7
:10CF20009305100093060000138604006FF01FC2E3
:10CF300033084441E35A009713050001E350050705
:10CF4000130F0001930F70006F00800113852600FE
:10CF50001307870093060600130808FF63500F07A6
:10CF60009387070113861600232027012322E70158
:10CF70002324F1042322C104E3DACFFC63840716DF
:10CF8000130601049385090013850A00232C01016F
:10CF9000EFF04FD3E31C0598032881018326410459
:10CFA000130F0001130808FF83278104138704006F
:10CFB00013851600930F7000E3440FFB130F8700D7
:10CFC000B387070123202701232207012324F1042B
:10CFD0002322A104130770006352A746638E076CD7
:10CFE000130601049385090013850A00EFF08FCD25
:10CFF000E31E059283264104B38C8C418327810470
:10D00000130641059385160013870400E352908BA5
:10D01000130500016358956913030001130F700095
:10D020006F00800193852600130787009306060092
:10D03000938C0CFF635C930593870701138616009E
:10D0400023202701232267002324F1042322C10483
:10D05000E35ACFFC63840706130601049385090095
:10D0600013850A00EFF00FC6E312058C83264104F6
:10D0700013030001938C0CFF8327810413870400A2
:10D0800093851600130F7000E34893FB9306870007
:10D09000B387970123202701232297012324F1043A
:10D0A0002322B104130770006344B71A9385150057
:10D0B00013868600138706006FF08FFF930510001C
:10D0C00093060000138704006FF09FF61306010417
:10D0D0009385090013850A00EFF0CFBEE30C0582AB
:10D0E0006FF0DF841305100093060000138704001F
:10D0F0006FF09FE6638A071E1306010493850900FB
:10D1000013850A00232EE101232CF101EFF08FBBE0
:10D11000E31E05808326410483278104032FC10178
:10D12000832F8101130641059385160013870400A0
:10D130006FF04FF19307C1032326F10493072000FA
:10D140002328F1049305100013064105938605007A
:10D150001307060093851600130687006FF04FF43F
:10D16000138A0D006FF0DFAF9305000163D60561F0
:10D1700093020001930370006F00C0011385260025
:10D180001307870093060600130808FF63D80207F9
:10D190001386160093870701232077012322570067
:10D1A0002324F1042322C104E3DAC3FC638E0706BF
:10D1B000130601049385090013850A002320010347
:10D1C000232EE101232CF101EFF0CFAF631005F620
:10D1D000032801028326410493020001130808FF7B
:10D1E00083278104032FC101832F8101138704004A
:10D1F0001385160093037000E3CC02F9B38707018F
:10D2000023207701232207012324F1042322A104F0
:10D210009306700063CAA60E1307870093051500D6
:10D22000930605006FF00FDE930600001305100053
:10D23000138704006FF05FF56354440113040A0080
:10D2400083278100B38787002324F1006FF08FECE0
:10D25000638A0734130601049385090013850A00C5
:10D26000EFF04FA6631405EC832541048327810466
:10D270001306410593851500138704006FF04FE3F3
:10D2800023220104138704006FF0CFCA639A0CF8BD
:10D29000930D0A00930C0000130C0000130B010FF8
:10D2A0006FF04FF90326C10093770A0193064600F9
:10D2B0006390071A93770A046386073C8327C100AB
:10D2C000130800002326D10003DC0700930610009A
:10D2D0006FF04FFF13064105930510009306000001
:10D2E000138704006FF0CFDB63880F1C9307C10323
:10D2F0002326F104930720002328F104930610004D
:10D30000130741056FF01FE5638E0726130601041E
:10D310009385090013850A00232EE101232CF101D6
:10D32000EFF04F9A631405E08326410483278104BC
:10D33000032FC101832F81011387040093851600F9
:10D340006FF04FCC93770A402320F102930D000039
:10D35000130B010F6F004003930508001306A00094
:10D360009306000013050C00232EE100232C01017D
:10D37000EF30C030032881010327C1016308083260
:10D38000130C050013880500930508001306A00080
:10D390009306000013050C00232EE100232C01014D
:10D3A000EF3000718327010213050503A30FABFEC5
:10D3B000032881010327C101130BFBFF938D1D007F
:10D3C000E38C07F88327410283C60700E396B6F98A
:10D3D0009307F00FE382FDF86316080093079000AF
:10D3E000E3F887B3832781028325C102232E01013D
:10D3F000330BFB401386070013050B00232CE100C1
:10D40000EFC04FD5032741020328C1011306A00036
:10D41000834517009306000013050C00B337B000D6
:10D42000B307F700930508002322F102EF3000252F
:10D4300003278101930D00006FF09FF49305150001
:10D4400013068F009306050013070F006FF0CFC57A
:10D450002326D100032C06001308000093061000B9
:10D460006FF04FE68327410283460D00638007B0CB
:10D4700083C70700638C07AE93ED0D406FF00FAFCD
:10D48000032681009357F64123A0C60023A2F6008D
:10D490006FF04FA3032C06002326D1001358FC4144
:10D4A000930608006FF04FD5032C06001308000008
:10D4B0002326D1006FF08FE093060000130641058C
:10D4C00093051000138704006FF08FBDB7670180CC
:10D4D000938787BD2328F10093F70D026384070625
:10D4E0008327C100138B7700137B8BFF032C0B006A
:10D4F00003284B0093078B002326F10013F61D0031
:10D50000630E060033660C01630A0600130600036F
:10D51000230EC102A30ED10293ED2D0013FAFDBF1D
:10D52000930620006FF00FDA138A0D006FF0DF848E
:10D53000B7670180938747BC2328F10093F70D025A
:10D54000E39007FA8325C10093F70D011386450088
:10D55000638A070603AC0500130800002326C100F8
:10D560006FF0DFF913050B00232CE1002326D10017
:10D57000EFC08FB503278101130C0500930C000049
:10D580006FF04FCB0347B10363160714E3940FBA50
:10D59000930600009305100013064105138704004D
:10D5A0006FF00FB01307100093070C0023266105DE
:10D5B00023288105232481052322E1041306410544
:10D5C0006FF0CFB293F70D046380070A8327C10081
:10D5D000130800002326C10003DC07006FF01FF2D0
:10D5E00083461D0093ED0D20130D1D006FF00F9865
:10D5F00083461D0093ED0D02130D1D006FF00F9774
:10D600008327810023A0F6006FF0CF8B9307600083
:10D61000138C0C0063EC970BB7680180130A0C00A5
:10D620002326D100138BC8BE6FF0CF9A93F70D203D
:10D63000638607108327C1002326D100038C0700CF
:10D640001358FC41930608006FF00FBB93F70D20B1
:10D65000638C070C8327C100130800002326D10028
:10D6600003CC07006FF08FC593F70D206384070A82
:10D670008327C100130800002326C10003CC070044
:10D680006FF0DFE793770A20638A07068327C100DC
:10D69000130800002326D10003CC070093061000D6
:10D6A0006FF04FC2930606006FF09F9E93079000A5
:10D6B000E3E887CD6FF0DF85130641059305100081
:10D6C00093060000138704006FF00F9E130C600098
:10D6D0006FF09FF49307B1032326F1049307100022
:10D6E0002328F10493051000130641056FF08F9471
:10D6F000832781002390F6006FE0DFFC8327C100C1
:10D70000130800002326D10003AC07009306100085
:10D710006FF04FBB8327C100130800002326C10010
:10D7200003AC07006FF09FDD8327C10013080000E2
:10D730002326D10003AC07006FF04FB88327C10048
:10D740002326D10003AC07001358FC4193060800C0
:10D750006FF08FAA130601049385090013850A0050
:10D76000EFE05FD66FF08F9C138C0C002326D10066
:10D77000930C00006FF00FAC130506006FF01FA8AC
:10D78000938516006FF0CFC1138A0D006FF04FA97B
:10D790009307F0FF2324F1006FF00F9A130F060098
:10D7A000138505006FF0DF818327C10083AC07007C
:10D7B0009387470063D40C00930CF0FF83461D0051
:10D7C0002326F100138D05006FE05FFA3787018093
:10D7D000930705000325479C930606001386050062
:10D7E000938507006FE09FDE83D7C50003AE450633
:10D7F00003D3E50083A8C50103A84502130101B8BE
:10D8000093F7D7FF13070040232C8146231AF1001A
:10D81000138405009307010793058100232A91468D
:10D8200023282147232E1146130905002326C1076B
:10D83000231B610023221103232601032324F1006B
:10D84000232CF1002328E100232EE10023200102F4
:10D85000EFE0DFD793040500635C050283574101C5
:10D8600093F70704638807008357C40093E707040E
:10D870002316F4008320C14703248147032901476D
:10D880001385040083244147130101486780000089
:10D890009305810013050900EF609FAFE30005FCCD
:10D8A0009304F0FF6FF09FFB130101FF1387050046
:10D8B0002324810023229100930506001304050010
:10D8C000B784018013860600130507002326110084
:10D8D00023AA04B0EF308F949307F0FF630CF50098
:10D8E0008320C1000324810083244100130101012E
:10D8F0006780000083A744B1E38407FE8320C10052
:10D900002320F4000324810083244100130101013A
:10D9100067800000B787018003A7479C130101FFC0
:10D920009387060013080600232611008328C700EA
:10D93000930605001387050013860700630008029D
:10D94000B76701809387074BB76501809385054CC6
:10D9500013850800EF004029EF20D01C37680180B4
:10D960009307C8AF1308C8AF6FF01FFE130101FF84
:10D97000930606001306000023261100EFF09FF91E
:10D98000B385C502130101FF232481002326110062
:10D99000EFA00F9513040500630805020326C5FFD9
:10D9A000130740021376C6FF1306C6FF6360C7065F
:10D9B000930630019307050063E2C60223A0070027
:10D9C00023A2070023A407008320C100130504003D
:10D9D000032481001301010167800000232005005A
:10D9E000232205009307B00163F0C7042324050038
:10D9F0002326050093070501E312E6FC2328050012
:10DA000093078501232A05006FF05FFB9305000053
:10DA1000EF300FEE8320C1001305040003248100C2
:10DA20001301010167800000930785006FF01FF963
:10DA3000130101FF23248100232291001304050018
:10DA4000B7840180138505002326110023AA04B0A2
:10DA5000EF20DFF99307F0FF630CF5008320C1008E
:10DA60000324810083244100130101016780000029
:10DA700083A744B1E38407FE8320C1002320F40080
:10DA80000324810083244100130101016780000009
:10DA9000130101FF2326110023248100232291007A
:10DAA00023202101638005021384050093040500EF
:10DAB0006306050083278503638C070A8317C40068
:10DAC000639207028320C100032481001309000030
:10DAD00083244100130509000329010013010101FA
:10DAE000678000009305040013850400EF608FE455
:10DAF0008327C40213090500638A07008325C40134
:10DB000013850400E7800700634C05068357C400B3
:10DB100093F70708639E070683250403638C0500BB
:10DB2000930704046386F50013850400EF609FD912
:10DB30002328040283254404638805001385040018
:10DB4000EF605FD823220404EF605FC02316040057
:10DB5000EF601FC08320C1000324810083244100A3
:10DB6000130509000329010013010101678000006A
:10DB7000EF60DFBC8317C400E38607F46FF09FF605
:10DB80008357C4001309F0FF93F70708E38607F8EB
:10DB90008325040113850400EF60DFD26FF0DFF707
:10DBA000B78701809305050003A5479C6FF05FEEE2
:10DBB000130101FC1303C1022326D10293060300C3
:10DBC000232E11002328E102232AF102232C010332
:10DBD000232E110323266100EFE05F9F8320C10104
:10DBE0001301010467800000130E050037850180D2
:10DBF000130101FC0325459C130381022324C10268
:10DC00002326D102138605009306030093050E0018
:10DC1000232E11002328E102232AF102232C0103E1
:10DC2000232E110323266100EFE05F9A8320C101B8
:10DC30001301010467800000130101FD2324810208
:10DC4000232E310123286101232611022322910270
:10DC500023202103232C4101232A5101130B05000A
:10DC60009389050013040600EF0040799307100024
:10DC70006310F5029387F9FF1307E00F636AF7005B
:10DC800013F7F90F2306E100130910006F00C0021B
:10DC90009306C405138609009305C10013050B0004
:10DCA000EF20C0539307F0FF130905006304F50A42
:10DCB000630E05080347C10093040000130AF0FF38
:10DCC000930AA0006F008002832704009386170048
:10DCD0002320D4002380E700938414009307C1001D
:10DCE000B387970063F4240703C7070083278400E2
:10DCF0009387F7FF2324F400E3D807FC83268401ED
:10DD0000930507001306040013050B0063C4D70036
:10DD1000E31C57FBEF20C032E31045FD1309F0FF71
:10DD20008320C10203248102832441028329C1018B
:10DD3000032A8101832A4101032B010113050900F4
:10DD40000329010213010103678000001389090000
:10DD50006FF01FFD8357C40093E707042316F400F8
:10DD60006FF01FFC8317C60013972701634007025B
:10DD700003274606B7260000B3E7D700B726000002
:10DD80003367D7002316F6002322E6066FF0DFEA9A
:10DD9000130101FEB7870180232C810003A4479C57
:10DDA000232E110013860500930505006306040069
:10DDB00083278403638007048317C6001397270112
:10DDC0006340070203274606B7260000B3E7D700E3
:10DDD000B72600003367D7002316F6002322E60695
:10DDE00013050400032481018320C10113010102F2
:10DDF0006FF09FE42324A100130504002326C10033
:10DE0000EF60DF930326C100832581006FF0DFFA06
:10DE1000130101FF138705002324810023229100B1
:10DE200013040500B784018093050600130507005D
:10DE30002326110023AA04B0EF20DFBB9307F0FFD5
:10DE4000630CF5008320C10003248100832441007A
:10DE5000130101016780000083A744B1E38407FE3A
:10DE60008320C1002320F400032481008324410087
:10DE7000130101016780000083278600638E07324B
:10DE800083D7C500130101FD23248102232C410106
:10DE9000232A510123261102232291022320210348
:10DEA000232E3101232861012326710123248101BE
:10DEB000232291012320A10113F78700130A0600F2
:10DEC000930A0500138405006306070803A70501EC
:10DED0006302070813F7270083240A00630C07086E
:10DEE000832744028325C401370B00809309000077
:10DEF00013090000134B0BC01386090013850A0099
:10DF0000630209049306090063742B0193060B0056
:10DF1000E78007006358A02883278A00B389A900F7
:10DF20003309A9403385A7402324AA00630A0520AA
:10DF3000832744028325C4011386090013850A0040
:10DF4000E31209FC83A9040003A94400938484001C
:10DF50006FF09FFA9305040013850A00EF608F8726
:10DF6000631C053A8357C40083240A0013F7270073
:10DF7000E31807F613F7170063140724832C8400B3
:10DF800003250400370B0080934BEBFF130C0000BC
:10DF900013090000134BFBFF630E090E13F7072054
:10DFA000630C0724138D0C006362992F13F7074845
:10DFB000630A070883294401832504011307190014
:10DFC00093961900B386360193D9F601330DB54007
:10DFD000B389D90093D919403307A70113860900E3
:10DFE00063F6E900930907001306070093F707405B
:10DFF0006384072E9305060013850A00EF905FAE39
:10E00000930C0500630205308325040113060D00FF
:10E01000EF00004F8357C40093F7F7B793E7070863
:10E020002316F4003385AC01B387A941232894015A
:10E030002320A400232A3401930C09002324F40094
:10E04000130D090013060D0093050C00EF00005D91
:10E05000032784008327040093090900B30C974128
:10E06000B387A701232494012320F400130900009F
:10E0700003268A00330C3C01B309364123243A01BC
:10E080006380090C832C8400032504008357C4009B
:10E09000E31609F003AC040003A944009384840050
:10E0A0006FF09FEF83A9440003AC040093848400C5
:10E0B000E38A09FE138609009305A00013050C00EE
:10E0C000EFA08F9D6304051213051500330B8541E6
:10E0D00093070B00938B090063F43701938B0700C0
:10E0E00003250400832704018326440163F8A70065
:10E0F00003298400338926016342790963C8DB1A46
:10E10000832744028325C40113060C0013850A00EB
:10E11000E7800700130905006356A008330B2B4165
:10E1200013051000630A0B1603268A00330C2C011A
:10E13000B38929413309264123242A01631A090896
:10E14000130500008320C1020324810283244102BD
:10E15000032901028329C101032A8101832A410184
:10E16000032B0101832BC100032C8100832C410070
:10E17000032D0100130101036780000093050C00CB
:10E1800013060900EF00804983270400930504006B
:10E1900013850A00B38727012320F400EF604F9F07
:10E1A000E30E05F68317C40093E707042316F40073
:10E1B0001305F0FF6FF01FF91305000067800000E2
:10E1C000130B000013050000130C0000930900005E
:10E1D000E38A09ECE31E05EE138609009305A0000F
:10E1E00013050C00EFA04F8BE31005EE9387190089
:10E1F000138B07006FF01FEE8327040163E2A7046F
:10E2000083274401636EF9029306090063F42B012E
:10E2100093060B00B3C6F602032744028325C4010C
:10E2200013060C0013850A00B386F602E700070008
:10E2300093090500E358A0F6330939416FF05FE315
:10E2400093890C00637499019309090013860900EE
:10E2500093050C00EF00803C832784000327040013
:10E26000B3873741330737012324F4002320E40028
:10E27000E39407FC9305040013850A00EF604F91B7
:10E28000E31205F2330939416FF09FDE930C090068
:10E29000130D09006FF01FDB9305040013850A00BE
:10E2A000EF600F8FE30205E86FF0DFEF13860B00DE
:10E2B00093050C00EF0080368327840003260400BA
:10E2C00013890B00B3877741330676012324F400CA
:10E2D0002320C4006FF09FE413850A00EF00C04CB8
:10E2E000930C0500E31005D48325040113850A006F
:10E2F000EF604FDD8317C4001307C00023A0EA00BE
:10E3000093F7F7F76FF05FEA1307C0008317C400B5
:10E3100023A0EA006FF05FE91305F0FF6FF09FE2C2
:10E32000130101FF2324810023229100130405001F
:10E33000B7840180138505002326110023AA04B0A9
:10E34000EF20CFEB9307F0FF630CF5008320C100B3
:10E350000324810083244100130101016780000030
:10E3600083A744B1E38407FE8320C1002320F40087
:10E370000324810083244100130101016780000010
:10E38000130101FF23261100232481002322910081
:10E39000630C0602B76501809385454F130506009F
:10E3A00013040600EF00D017B76401806312050262
:10E3B0001385044F8320C10003248100832441007E
:10E3C0001301010167800000B76401806FF05FFEF8
:10E3D0009385044F13050400EF009014E30A05FC35
:10E3E000B76501809385C5AF13050400EF00501396
:10E3F000E30005FC130500006FF0DFFBB787018029
:10E4000003C50796678000003787018093070500E2
:10E410000325479C13860500938507006FF05FF680
:10E42000130101FF1387050023248100232291009B
:10E430009305060013040500B784018013860600C7
:10E44000130507002326110023AA04B0EF208FDB59
:10E450009307F0FF630CF5008320C10003248100C3
:10E4600083244100130101016780000083A744B1A8
:10E47000E38407FE8320C1002320F40003248100ED
:10E48000832441001301010167800000B7870180E8
:10E4900003A3C791670003006380050263020604BB
:10E4A000638806048347060023A0F50003450600A1
:10E4B0003335A00067800000130101FF9305C10000
:10E4C00063040602638A06028347060023A0F50060
:10E4D000034506003335A0001301010167800000E9
:10E4E0001305000067800000130500006FF0DFFED9
:10E4F0001305E0FF678000001305E0FF6FF0DFFD0C
:10E50000B3C7A50093F73700B308C50063920706A9
:10E510009307300063FEC7049377350013070500A7
:10E520006398070613F6C8FF930706FE636CF708A7
:10E53000637CC702938605009307070003A80600C3
:10E54000938747009386460023AE07FFE3E8C7FEA4
:10E550009307F6FFB387E74093F7C7FF938747001A
:10E560003307F700B385F500636817016780000083
:10E5700013070500E37C15FF83C705001307170089
:10E5800093851500A30FF7FEE36817FF678000006F
:10E5900083C605001307170093773700A30FD7FE34
:10E5A00093851500E38007F883C60500130717005D
:10E5B00093773700A30FD7FE93851500E39A07FCE6
:10E5C0006FF05FF683A6450083A2050083AF850048
:10E5D00003AFC50083AE050103AE450103A385016A
:10E5E00003A8C5012322D70083A6050223205700D4
:10E5F0002324F7012326E7012328D701232AC70173
:10E60000232C6700232E07012320D702130747027C
:10E6100093854502E368F7FA6FF09FF163F6A50270
:10E62000B387C5006372F5023307C500630A060E9F
:10E6300083C6F7FF9387F7FF1307F7FF2300D70081
:10E64000E398F5FE678000009307F00063E8C702D7
:10E65000930705009306F6FF630C060C93861600DD
:10E66000B386D70003C7050093871700938515006D
:10E67000A38FE7FEE398D7FE67800000B3E7A5000D
:10E6800093F737006390070A930806FF93F808FF93
:10E6900093880801330815011387050093070500C7
:10E6A00083260700130707019387070123A8D7FED6
:10E6B000832647FF23AAD7FE832687FF23ACD7FEF6
:10E6C0008326C7FF23AED7FEE31CF8FC1377C600F2
:10E6D000B38515011378F600630E07041387050050
:10E6E00093880700130E3000032307001307470029
:10E6F000B306E84023A06800B386D500938848009D
:10E70000E364DEFE1307C8FF1377C7FF1307470054
:10E7100013763600B387E700B385E5006FF09FF30B
:10E72000678000009306F6FF930705006FF01FF364
:10E7300067800000130608006FF0DFF1130101FF8E
:10E7400013870500232481002322910093050600EE
:10E7500013040500B7840180138606001305070023
:10E760002326110023AA04B0EF204FAA9307F0FF3D
:10E77000630CF5008320C100032481008324410041
:10E78000130101016780000083A744B1E38407FE01
:10E790008320C1002320F40003248100832441004E
:10E7A0001301010167800000130101FD23202103F3
:10E7B000232611022324810223229102232E3101D8
:10E7C000232C4101232A51012328610123267101B1
:10E7D00023248101130906006384052213840500A4
:10E7E00093090500EF909FB89304B9009307600167
:10E7F00063FE970E93F484FF1387040063CE040E28
:10E8000063EC240F8327C4FF930A84FF13FAC7FF26
:10E81000338B4A01635CEA18B7760180938B064319
:10E8200003A68B0083264B00630E662313F6E6FFD8
:10E830003306CB0003264600137616006314061A2F
:10E8400093F6C6FF3306DA00635EE63293F71700ED
:10E8500063940702032C84FF338C8A4183274C0086
:10E8600093F7C7FFB386D700B38B460163DAEB3467
:10E87000B30BFA0063D2EB0C930509001385090072
:10E88000EF900FA613090500630C05048327C4FF4E
:10E89000130785FF93F7E7FFB387FA006382E7303A
:10E8A0001306CAFF9307400263E6C730130730011F
:10E8B00083260400636CC726930705001307040032
:10E8C00023A0D7008326470023A2D7000327870071
:10E8D00023A4E7009305040013850900EF509FFE71
:10E8E00013850900EF90DFA86F00C00193040001B9
:10E8F00013070001E3F824F19307C00023A0F900F7
:10E90000130900008320C1020324810283244102F1
:10E910008329C101032A8101832A4101032B0101BB
:10E92000832BC100032C8100130509000329010278
:10E9300013010103678000008327CC0003278C00AC
:10E940001306CAFF930640022326F70023A4E7001C
:10E9500013098C00330B7C0163E4C62E9305300150
:10E96000032704009307090063F2C5022324EC0087
:10E97000032744009307B0012326EC0063E2C7306D
:10E980000327840093070C011304840023A0E700ED
:10E9900003274400138A0B00930A0C0023A2E7000C
:10E9A000032784001304090023A4E70083A74A0077
:10E9B00033079A409306F00093F7170063ECE606DE
:10E9C000B367FA0023A2FA0083274B0093E71700EE
:10E9D0002322FB0013850900EF909F99130904007F
:10E9E0006FF05FF293F71700E39807E8032C84FFBA
:10E9F000338C8A4183274C0093F7C7FF6FF05FE7A2
:10EA0000032481028320C1028324410203290102DD
:10EA10008329C101032A8101832A4101032B0101BA
:10EA2000832BC100032C8100930506001301010311
:10EA30006F900F8BB3E7970023A2FA00B3859A007B
:10EA40001367170023A2E50083274B0093858500F9
:10EA50001385090093E717002322FB00EF509FE680
:10EA60006FF05FF793F6C6FF3306DA009385040173
:10EA70006350B60E93F71700E39007E0032C84FF72
:10EA8000338C8A4183274C0093F7C7FFB386D700A6
:10EA9000338B4601E34EBBDC8327CC0003278C007D
:10EAA0001306CAFF930640022326F70023A4E700BB
:10EAB00013098C0063EEC620930530010327040080
:10EAC0009307090063F2C5022324EC0003274400E6
:10EAD0009307B0012326EC0063E4C72003278400DA
:10EAE00093070C011304840023A0E70003274400CC
:10EAF00023A2E7000327840023A4E70033079C0038
:10EB0000B3079B4023A4EB0093E717002322F700F1
:10EB100083274C001385090093F71700B3E497008F
:10EB200023229C00EF90DF846FF0DFDD2320D500EF
:10EB3000832644001307B0012322D5006360C71267
:10EB40008326840013078400930785006FF05FD746
:10EB5000B38A9A00B307964023A45B0193E717009A
:10EB600023A2FA008327C4FF1385090013090400B8
:10EB700093F71700B3E49700232E94FEEF904FFF16
:10EB80006FF05FD88327CB0003278B00130A0600A2
:10EB9000338BCA002326F70023A4E7006FF01FE1A0
:10EBA0008327C5FF93F7C7FF330AFA00338B4A0167
:10EBB0006FF0DFDF93050400EFF05FA66FF09FD1E9
:10EBC0008327CB0003278B001306CAFF930640025E
:10EBD0002326F70023A4E70003278C008327CC001B
:10EBE00013098C00330B7C012326F70023A4E700D4
:10EBF00063E8C60493063001032704009307090065
:10EC0000E3F6C6D82324EC00032744009307B001A1
:10EC10002326EC0003278400E3F6C7D62328EC0064
:10EC20000327C40093074002232AEC0003270401B2
:10EC30006304F60693078C01130404016FF01FD5DB
:10EC40009305040013050900EFF05F9D130409000C
:10EC5000138A0B00930A0C006FF05FD50327840022
:10EC60002324E5000327C4002326E50083260401AE
:10EC70006302F60413070401930705016FF05FC4F4
:10EC8000832784002328FC008327C400232AFC0058
:10EC900003270401E310D6FA232CEC0003274401D8
:10ECA00093070C0213048401232EEC0003270400B5
:10ECB0006FF0DFCD2328D50083264401130784019C
:10ECC00093078501232AD500832684016FF05FBF57
:10ECD0009305040013050900EFF05F946FF01FE245
:10ECE000832784002328FC008327C400232AFC00F8
:10ECF000032704016308D60093078C011304040161
:10ED00006FF09FDE232CEC000327440193070C02D5
:10ED100013048401232EEC00032704006FF0DFDCD2
:10ED20003367B5009303F0FF1377370063100710C4
:10ED3000B7877F7F9387F7F70326050083A6050033
:10ED4000B372F6003363F600B382F200B3E26200FE
:10ED5000639272106316D6080326450083A6450009
:10ED6000B372F6003363F600B382F200B3E26200DE
:10ED7000639E720C6316D6060326850083A6850063
:10ED8000B372F6003363F600B382F200B3E26200BE
:10ED90006398720C6316D6040326C50083A6C500CB
:10EDA000B372F6003363F600B382F200B3E262009E
:10EDB0006392720C6316D6020326050183A6050131
:10EDC000B372F6003363F600B382F200B3E262007E
:10EDD000639C720A1305450193854501E30ED6F441
:10EDE0001317060193970601631EF70013570601D8
:10EDF00093D706013305F7409375F50F639005022D
:10EE0000678000001357070193D707013305F740C8
:10EE10009375F50F63940500678000001377F70F73
:10EE200093F7F70F3305F7406780000003460500AE
:10EE300083C6050013051500938515006314D600DD
:10EE4000E31606FE3305D640678000001305450033
:10EE500093854500E31CD6FC130500006780000085
:10EE60001305850093858500E312D6FC1305000089
:10EE7000678000001305C5009385C500E318D6FA26
:10EE80001305000067800000130505019385050147
:10EE9000E31ED6F813050000678000008327860074
:10EEA000130101FD232A510123261102232481028B
:10EEB0002322910223202103232E3101232C4101FF
:10EEC000232861012326710123248101930A06006E
:10EED00063880714130B05008329060003A50500AA
:10EEE00083A48500138405006F00400D8357C40080
:10EEF00013F70748630A07088326440183250401A2
:10EF00001307190093941600B386D40093D4F60126
:10EF1000330AB540B384D40093D414403307470177
:10EF20001386040063F6E400930407001306070049
:10EF300093F707406386070A9305060013050B0045
:10EF4000EF801FBA130C0500630A050A832504012C
:10EF500013060A00EFF0CFDA8357C40093F7F7B730
:10EF600093E707082316F40033054C01338A444124
:10EF7000232A940023244401232884012320A4006D
:10EF800093040900130A090013060A0093850B0075
:10EF9000EFF0CFE8032784000325040083A78A004D
:10EFA000B304974033054501232494002320A40093
:10EFB0003389274123A42A016304090603A94900D0
:10EFC00083AB0900138A040093898900E30809FED2
:10EFD000E37E99F093040900130A09006FF0DFFA49
:10EFE00013050B00EFF04FFC130C0500E31E05F6B4
:10EFF0008325040113050B00EF50DF8C9307C0003D
:10F000002320FB008357C4001305F0FF93E7070498
:10F010002316F40023A40A0023A20A006F00C000F4
:10F0200023A20A00130500008320C10203248102E9
:10F0300083244102032901028329C101032A81019A
:10F04000832A4101032B0101832BC100032C810082
:10F05000130101036780000083D7C500130101ED90
:10F06000232C4111232861112320A11123261112E1
:10F07000232481122322911223202113232E3111C4
:10F08000232A511123267111232481112322911146
:10F09000232EB10F93F707082326D100138A05000A
:10F0A000130B0500130D06006386070083A70501F7
:10F0B000E3860756B7670180930AC1049387075018
:10F0C000B76B0180B764018023205105232401041C
:10F0D0002322010413870A002328010023220102AE
:10F0E000232401022326010223240100232AF10004
:10F0F000938BCB669384C46783470D00638007209E
:10F1000013040D00930650026386D738834714001A
:10F1100013041400E39A07FE3309A4416300A41FFB
:10F1200083268104832741042320A701B386260177
:10F1300093871700232227012324D1042322F104DB
:10F14000930670001307870063CEF6348326810090
:10F1500083470400B38626012324D1006380071A65
:10F1600083461400130D1400A30D0102930CF0FF4D
:10F1700013040000930D00001309A005130C900068
:10F180009309A002130D1D00938706FE6364F90422
:10F190000326410193972700B387C70083A7070081
:10F1A0006780070013040000938706FD83460D0067
:10F1B00093152400338485001314140033848700CE
:10F1C000938706FD130D1D00E372FCFE938706FE78
:10F1D000E370F9FC638406122306D108A30D010233
:10F1E00013091000130C10009309C108930C0000C0
:10F1F00013FF2D0063040F001309290013FE4D08AF
:10F20000832781040326410463160E00B3062441BC
:10F21000E34AD0028346B103130516009305870025
:10F22000638006049306B103938717002320D70059
:10F23000930610002322D7002324F1042322A104E3
:10F2400093067000E3CEA60C930F260093060701E9
:10F25000130605001387050013850F00938506002C
:10F26000630C0F029306C1032320D7009387270066
:10F27000930620002322D7002324F1042322A10493
:10F2800013077000E34CA70C130605001387050055
:10F290001305150093858500930600086302DE6060
:10F2A000B38C8C416346906BB307FC00232037017D
:10F2B000232287012324F1042322A10413077000D1
:10F2C0006342A77493F84D0063860800330C244111
:10F2D0006348801F6354240113040900032781003D
:10F2E000330787002324E100639E077283470D00E4
:10F2F0002322010413870A00E39407E08327810493
:10F30000E392074C8357CA0093F70704E398074E2C
:10F310008320C1120324811203258100832441121A
:10F32000032901128329C111032A8111832A411162
:10F33000032B0111832BC110032C8110832C41104E
:10F34000032D0110832DC10F1301011367800000ED
:10F3500013050B00232CE100EF800FD88327450015
:10F36000138507002326F102EFA00FD693070500AF
:10F3700013050B002324F102EF800FD6032785002D
:10F38000832781022322E10203278101E3980716E4
:10F3900083460D006FF01FDF83460D0093ED0D02D5
:10F3A0006FF05FDE93ED0D0193F70D026382071E90
:10F3B0008327C1009389770093F989FF83A64900C9
:10F3C00003AC0900938789002326F100138E060001
:10F3D00063C8061E9306F0FF13890D006388DC00E6
:10F3E000B366CC0113F9FDF76384067AE31C0E00C3
:10F3F00093069000E3E8860193070C03A307F10E40
:10F40000930D0900130C10009309F10E6F00C00654
:10F4100093ED0D0193F70D02638607148327C10056
:10F420009389770093F989FF03AC090003AE490083
:10F43000938789002326F10013F9FDBF930600008E
:10F44000A30D01021306F0FF6380CC1A3366CC01D2
:10F45000937DF9F76314065E63980C3E639E067213
:10F46000137C19009309010F63080C009307000334
:10F47000A307F10E9309F10E13890C0063D48C01DC
:10F4800013090C008347B103B337F0003309F900C7
:10F490006FF01FD63309A441E314A4C983470400C5
:10F4A0006FF0DFCB1306010493050A0013050B0070
:10F4B000EFF0DF9EE31805E413870A006FF01FC921
:10F4C000930600010327410463D08607930C0001D3
:10F4D000930970006F00C000130C0CFF63D68C05FD
:10F4E000938707011307170023A0750123A2950135
:10F4F0002324F1042322E10493858500E3DEE9FC63
:10F500001306010493050A0013050B00EFF01F9981
:10F51000E31A05DE130C0CFF832781040327410443
:10F5200093850A00E3CE8CFBB3878701130717008E
:10F5300023A0750123A285012324F1042322E104E1
:10F5400093067000E3D8E6D81306010493050A0079
:10F5500013050B00EFF09F94E31605DA832781046F
:10F560006FF05FD70326C10093F70D0193064600A5
:10F570006392077E93F70D04E38C07188327C1007D
:10F58000130E00002326D10003DC07006FF0DFEA32
:10F590000326C10093F70D01930646006398077890
:10F5A00093F70D04E38607148327C1002326D100B7
:10F5B000039C0700135EFC4193060E00E3DC06E0AB
:10F5C000B3368001330EC041330EDE409306D002C5
:10F5D000A30DD1021306F0FF330C804113890D00F7
:10F5E00093061000E394CCE613061000E380C6E017
:10F5F000130620006384C6269309010F1316DE014B
:10F6000093767C0093573C0093860603336CF60098
:10F61000135E3E00A38FD9FE3366CC0193850900AB
:10F620009389F9FFE31C06FC937719006382072690
:10F6300093070003638EF6249385E5FFA38FF9FEFD
:10F640009307010F338CB740930D09009389050090
:10F650006FF09FE28327C100A30D010283A9070079
:10F6600093864700E38609049307F0FF6388FC78DC
:10F6700013860C009305000013850900232CD1008C
:10F680002326E100EF805FC10327C10083268101AB
:10F69000E3040514330C35412326D100930C0000FC
:10F6A0006FF09FDD8326C100A30D01021309100036
:10F6B00083A70600938646002326D1002306F1087F
:10F6C000130C10009309C1086FF05FB28327C100CB
:10F6D00013E92D00B786FFFF03AC0700B76D01806B
:10F6E0009387470093C606832326F10093874DBC7A
:10F6F000231ED102130E00002328F10093062000E0
:10F700006FF01FD40326C10093F70D028326060075
:10F71000130646002326C1006390076093F70D018E
:10F720006392077893F70D04E398070893F80D2088
:10F73000638A0876832781002380F6006FF0DF9BC1
:10F7400083460D0093ED0D086FF0DFA383460D0097
:10F7500093051D00E38A360B938706FD138D050084
:10F76000930C0000E362FCA283460D0093952C00ED
:10F770003383950113131300B30CF300938706FD35
:10F78000130D1D00E372FCFE6FF01FA083460D00F9
:10F7900093ED4D006FF01F9F9307B00283460D005D
:10F7A000A30DF1026FF01F9E8327C10083460D0059
:10F7B00003A40700938747002326F100E354049C29
:10F7C0003304804093ED4D006FF0DF9B83460D00C6
:10F7D00093ED1D006FF01F9B8347B10383460D001F
:10F7E000E392079A93070002A30DF1026FF09F992D
:10F7F00083460D009307C0066388F66693ED0D01FE
:10F800006FF05F9883460D00930780066386F66469
:10F8100093ED0D046FF01F9713E90D019377090223
:10F82000638407388327C10093061000938977000B
:10F8300093F989FF9387890003AC090003AE49005F
:10F840002326F1006FF0DFBF13061000638EC67829
:10F850001306200013890D00E390C6DA9309010F07
:10F86000832701019376FC009389F9FFB386D700C3
:10F8700003C6060093574C009316CE0133ECF600F6
:10F88000135E4E002380C900B366CC01E39A06FCE8
:10F890009307010F338C3741930D09006FF0DFBDE3
:10F8A000B3062441E35ED09E130E00016352DE7462
:10F8B000130F70006F00C000938606FF635EDE04C6
:10F8C0009387070113061600232097002322C70100
:10F8D0002324F1042322C10413078700E35ECFFC35
:10F8E0001306010493050A0013050B00232CD10015
:10F8F000EFF0CFDAE31805A083268101130E000193
:10F9000083278104938606FF0326410413870A0098
:10F91000130F7000E346DEFA13061600130E87007D
:10F92000B387D700232097002322D7002324F10494
:10F930002322C104130770006340C754B38C8C4169
:10F940001305160093058E0013070E00E35E9095D5
:10F9500013030001635C935F130E70006F00C0001F
:10F96000938C0CFF635A93059387070113061600C7
:10F9700023209700232267002324F1042322C104BB
:10F9800013078700E35ECEFC1306010493050A000B
:10F9900013050B00EFF08FD0E3160596130300015B
:10F9A000938C0CFF832781040326410413870A00EC
:10F9B000130E7000E34A93FB13051600130687002D
:10F9C000B387970123209700232297012324F10472
:10F9D0002322A104130770006340A7201307060029
:10F9E00013051500B307FC002320370123228701EC
:10F9F0002324F1042322A104130770009305860039
:10FA0000E352A78C1306010493050A0013050B00AB
:10FA1000EFF0CFC8E318058E8327810493850A0091
:10FA20006FF05F8A1306010493050A0013050B00AB
:10FA3000EFF0CFC6E30C058A6FF0DF8C13890D0061
:10FA40006FF09FBA9305000163D0D508930F0001B2
:10FA5000930270006F00C000938606FF63D6DF0636
:10FA60009387070113061600232077012322F7014D
:10FA70002324F1042322C10413078700E3DEC2FC20
:10FA80001306010493050A0013050B002320D1027D
:10FA9000232EC101232CE101EFF04FC0E3140586B2
:10FAA00083260102930F000183278104938606FFBA
:10FAB00003264104032EC101032F810113870A008D
:10FAC00093027000E3CEDFF8B387D7001306160069
:10FAD0002322D700232077012324F1042322C10409
:10FAE000930670001307870063D6C6F2130601045D
:10FAF00093050A0013050B00232EC101232CE101FD
:10FB0000EFF0CFB9E3100580832781040326410479
:10FB1000032EC101032F810113870A006FF08FEFBD
:10FB20001306010493050A0013050B00232EC101DF
:10FB3000232CE101EFF08FB6631605FC0326410488
:10FB400083278104032EC101032F81019305410501
:10FB50001305160013870A006FF08FF013060104D7
:10FB600093050A0013050B00232CC101EFF00FB31E
:10FB7000631A05F80326410483278104032E8101BB
:10FB8000930541051305160013870A006FF0CFF0A7
:10FB9000E3940C86930D0900930C0000130C0000F5
:10FBA0009309010F6FF05F8D0326C1009377090160
:10FBB000930646006396071893770904638807360F
:10FBC0008327C100130E00002326D10003DC0700A9
:10FBD000930610006FF0DF861306010493050A00F8
:10FBE00013050B00EFF08FAB631E05F003254104F6
:10FBF00083278104930541051305150013870A0027
:10FC00006FF08FEA937709402320F102930D0000F3
:10FC10009309010F6F00400393050E001306A00027
:10FC20009306000013050C00232EE100232CC101D4
:10FC3000EF00D024032E81010327C101630C0E3095
:10FC4000130C0500138E050093050E001306A0008B
:10FC50009306000013050C00232EE100232CC101A4
:10FC6000EF0010658327010213050503A38FA9FE8A
:10FC7000032E81010327C1019389F9FF938D1D0094
:10FC8000E38C07F88327410283C60700E396B6F9A1
:10FC90009307F00FE382FDF863160E0093079000C0
:10FCA000E3F887BF832781028325C102232EC10188
:10FCB000B389F9401386070013850900232CE1005E
:10FCC000EF905FC903274102032EC1011306A00074
:10FCD000834517009306000013050C00B337B000EE
:10FCE000B307F70093050E002322F102EF0010196D
:10FCF00003278101930D00006FF09FF483274102D9
:10FD000083460D00638007C883C70700638C07C65E
:10FD100093ED0D406FF00FC7032681009357F64116
:10FD200023A0C60023A2F6006FF00FBD032C06002F
:10FD30002326D100135EFC4193060E006FF04FE9BD
:10FD40002326D100032C0600130E0000930610009A
:10FD50006FF00FEF032C0600130E00002326D100D6
:10FD60006FF08FED13890D006FF05FABB767018007
:10FD7000938787BD2328F10093F70D026380070660
:10FD80008327C1009389770093F989FF03AC0900A9
:10FD900003AE4900938789002326F10013F61D0066
:10FDA000630E06003366CC01630A060013060003E7
:10FDB000230EC102A30ED10293ED2D0013F9FDBF56
:10FDC000930620006FF0CFE7B7670180938747BCA9
:10FDD0002328F10093F70D02E39407FA8325C1006D
:10FDE00093F70D0113864500638A070403AC0500F1
:10FDF000130E00002326C1006FF05FFA138509007F
:10FE0000232CE1002326D100EF901FAC03278101B2
:10FE1000130C0500930C00006FF00FE6930500042F
:10FE2000EF701FCC2320AA002328AA00630005201E
:10FE300093070004232AFA006FF0CFA793F70D046D
:10FE4000638A07088327C100130E00002326C10020
:10FE500003DC07006FF09FF483461D0093ED0D2037
:10FE6000130D1D006FF00FB283461D0093ED0D02C0
:10FE7000130D1D006FF00FB11306010493050A0066
:10FE800013050B00EFF08F81631E05C603264104A6
:10FE900083278104930541051305160013870A0083
:10FEA0006FF00FC08327810023A0F6006FF0CFA46E
:10FEB00093076000138C0C0063F49701130C60002F
:10FEC000B76E018013090C002326D1009389CEBEA2
:10FED0006FF0CFB193F70D206386070C8327C10025
:10FEE000130E00002326C10003CC07006FF01FEBA8
:10FEF00093F70D20638C07088327C1002326D100C8
:10FF0000038C0700135EFC4193060E006FF04FCC8C
:10FF100093F70D20638207068327C100130E0000AC
:10FF20002326D10003CC07006FF00FD1937709206F
:10FF3000638807028327C100130E00002326D10027
:10FF400003CC0700930610006FF08FCF13860500D7
:10FF50006FF01FA793079000E3E487CF6FF05F93E4
:10FF60008327C100130E00002326D10003AC070035
:10FF7000930610006FF0CFCC8327C100130E000052
:10FF80002326D10003AC07006FF00FCB8327C100FD
:10FF90002326D10003AC0700135EFC4193060E003C
:10FFA0006FF00FC38327C100130E00002326C1008A
:10FFB00003AC07006FF09FDE832781002390F600DB
:10FFC0006FF08F931306010493050A0013050B00CD
:10FFD000EFE0DFEC6FF00FB3138C0C002326D100A1
:10FFE000930C00006FF04FC913890D006FF0CFC064
:10FFF000138E0500130605006FF09F929307F0FF24
:02000004800179
:100000002324F1006FF0CFB08327C10083AC070039
:100010009387470063D40C00930CF0FF83461D00C8
:100020002326F100138D05006FF0CF959307C000D4
:100030002320FB009307F0FF2324F1006FF04FAD66
:10004000130101FE232C8100232A91002328210182
:10005000232E110023263101130905009384050086
:1000600013040600630605008327850363880714CD
:100070000317C40083268401937787002324D400C8
:100080009316070193D606016382070883270401AC
:10009000638E07061396260193F9F40F93F4F40F79
:1000A000635E06080327040083264401B307F74074
:1000B00063DED70A83268400130617002320C400BA
:1000C0009386F6FF2324D40023003701032744013D
:1000D000938717006308F70C8357C40093F7170042
:1000E000638607009307A000638EF40A8320C10192
:1000F00003248101032901018329C1001385040020
:10010000832441011301010267800000930504006C
:1001100013050900EF301FEC631E05080317C40028
:1001200093F9F40F832704019316070193D6060170
:100130001396260193F4F40FE34606F6832644064D
:10014000372600003367C70037E6FFFF1306F6FFC8
:10015000B3F6C6002316E400032704002322D406C6
:1001600083264401B307F740E3C6D7F493050400A0
:1001700013050900EF40CFA1631E05020327040009
:100180008326840093071000130617009386F6FF5A
:100190002320C4002324D400230037010327440173
:1001A000E31CF7F29305040013050900EF404F9E8E
:1001B000E30E05F29304F0FF6FF05FF3EF400FD80A
:1001C0006FF01FEB37870180930705000325479CDD
:1001D00013860500938507006FF09FE6130101FE6B
:1001E000232C8100232A9100B7870180232E110040
:1001F00083A7879113040500938406006382050298
:10020000E78007009307F0FF6306F5028320C10132
:10021000032481018324410113010102678000004E
:100220001306000093054100E78007009307F0FFE5
:10023000E31EF5FC23A004009307A0088320C1015E
:100240002320F400032481018324410113010102CE
:1002500067800000130101FEB7870180232C810015
:10026000232A9100232E110083A4479CB787018085
:1002700083A7879113040600630A0502138605000D
:10028000930604009305050013850400E78007002A
:100290009307F0FF630AF5028320C1010324810163
:1002A00083244101130101026780000093060600C8
:1002B000930541001306000013850400E780070042
:1002C0009307F0FFE31AF5FC232004008320C1010B
:1002D000032481019307A00823A0F4008324410193
:1002E0001301010267800000B787018003A3879193
:1002F00067000300638405029307F00F63E8C700FB
:100300002380C50013051000678000009307A00834
:100310002320F5001305F0FF67800000130500009F
:1003200067800000130101FF130560002326110000
:10033000EF00C02813051000EF000FE6130101FFC6
:1003400093050008232481002326110013040500CF
:10035000EF700FF9232EA42C630405029307050800
:100360002320050013054500E31CF5FE13050000DE
:100370008320C10003248100130101016780000074
:100380001305F0FF6FF0DFFE8327C52D638607009E
:1003900013050000678000006FF05FFA130101FE93
:1003A000232A9100232E1100232C81009307F001B2
:1003B0009304050063EAB702138405008325C52D65
:1003C000638405041314240033848500032504008A
:1003D0002320C4008320C10103248101832441011F
:1003E00013010102678000008320C1010324810101
:1003F000930760012320F500832441011305F0FFDA
:1004000013010102678000002326C100EFF01FF3F3
:10041000930705001305F0FFE39E07FA83A5C42D9B
:100420000326C1006FF01FFA130101FF2322910080
:1004300023261100232481009307F0019304050073
:1004400063EAB70A8327C52D138405006384070474
:1004500013972500B387E70003A70700630C070283
:1004600093061000630CD7069306F0FF6308D704C9
:100470001385050023A00700E7000700130500000F
:100480008320C10003248100832441001301010162
:100490006780000013850400EF00001E13060400AF
:1004A000032481008320C100930505001385040007
:1004B00083244100130101016F0080158320C100D6
:1004C00003248100930760012320F5008324410069
:1004D0001305100013010101678000008320C10093
:1004E000032481008324410013050000130101014E
:1004F00067800000930760012320F5001305F0FFDB
:100500006FF01FF89307F00163E6B70A8327C52D44
:10051000130101FE232C9100232E110093040500EA
:10052000638C070413972500B387E70003A7070030
:10053000630A07029306F0FF6306D70693061000CE
:100540006308D7041385050023A00700E700070010
:10055000130500008320C1018324810113010102DE
:10056000678000008320C1018324810113051000EE
:1005700013010102678000002326B100EFF01FDCA9
:100580006316050283A7C42D8325C1006FF09FF970
:100590008320C1018324810113053000130101026E
:1005A00067800000130520006FF0DFFA1305F0FFED
:1005B0006FF05FFA1305F0FF67800000B7870180D6
:1005C0009305050003A5479C6FF01FE63787018060
:1005D000930705000325479C1386050093850700B4
:1005E0006FF0DFDBB787018003A5479C8327C52D0C
:1005F0006386070013050000678000006FF01FD4BA
:10060000B78701809305050003A5479C6FF09FEF16
:10061000130101FF13870500232481002322910089
:1006200013040500B7840180930506001305070035
:100630002326110023AA04B0EF004FC39307F0FF55
:10064000630CF5008320C100032481008324410052
:10065000130101016780000083A744B1E38407FE12
:100660008320C1002320F40003248100832441005F
:1006700013010101678000006F00CFBF93080500E0
:1006800093870500130806001385060013830800EE
:1006900063940628B77601809386468463F6C50E78
:1006A000370701006378E60C1307F00F3337C700F4
:1006B000131737003355E600B386A60083C606003D
:1006C000130500023387E600B306E540630CE5003E
:1006D000B397D70033D7E8003318D600B365F700D7
:1006E0003393D80093580801B3D7150313160801A4
:1006F0001356060113570301B3F6150313850700BC
:10070000B305F6029396060133E7E600637EB70071
:10071000330707011385F7FF636807016376B700A6
:100720001385E7FF330707013307B740B377170394
:10073000131303011353030133571703939707014F
:1007400033E36700B306E60213060700637CD300B9
:10075000330368001306F7FF636603016374D30075
:100760001306E7FF131505013365C5009305000067
:100770006F00400E3705000113070001E36CA6F27D
:10078000130780016FF01FF36316060013071000B4
:100790003358C702370701006370E80C1307F00FE6
:1007A00063740701130580003357A800B386E60081
:1007B00003C70600130600023307A700B306E6408E
:1007C0006316E60AB38707419305100093580801A2
:1007D000131608011356060113570301B3F6170346
:1007E000B3D717039396060133E7E600330EF602FC
:1007F00013850700637EC701330707011385F7FFE1
:10080000636807016376C7011385E7FF33070701B4
:100810003307C741B37717031313030113530301BE
:10082000335717039397070133E36700B306E602D4
:1008300013060700637CD300330368001306F7FF39
:10084000636603016374D3001306E7FF1315050104
:100850003365C500678000003707000113050001FC
:10086000E364E8F4130580016FF01FF43318D80037
:10087000B3D5E7003393D800B397D70033D7E80058
:10088000935808013366F70033F7150393170801EF
:1008900093D7070113550601B3D5150313170701A5
:1008A0003367A700B386B70213850500637ED700C0
:1008B000330707011385F5FF636807016376D700E7
:1008C0001385E5FF33070701B306D74033F7160357
:1008D0001316060113560601B3D6160313170701A4
:1008E000B388D702B367C7001387060063FE1701FA
:1008F000B38707011387F6FF63E8070163F6170163
:100900001387E6FFB387070193150501B3871741E6
:10091000B3E5E5006FF09FEB63E6D51837070100FC
:1009200063F4E6041307F00FB335D7009395350051
:100930003777018033D5B600130747843307A70004
:1009400003470700130500023307B700B305E5406E
:100950006316E50213051000E3EEF6EE33B5C800AA
:10096000134515006FF01FEF3707000193050001D5
:10097000E3E0E6FC930580016FF09FFB3353E60054
:10098000B396B6003363D30013550301B31EB6000C
:1009900033D6E700B376A602B397B70033D7E800A3
:1009A0003368F7009317030193D707011357080122
:1009B0003356A6029396060133E7E600338FC7024B
:1009C000130E0600637EE70133076700130EF6FF80
:1009D000636867006376E701130EE6FF330767007D
:1009E0003307E741B376A7023357A7029396060170
:1009F0003386E7029317080193D70701B3E7F600A0
:100A00009306070063FEC700B38767009306F7FFEE
:100A100063E8670063F6C7009306E7FFB3876700E4
:100A200013150E01370E01003365D5009306FEFF46
:100A30003378D500B387C740B3F6DE0013560501FF
:100A400093DE0E013303D802B306D6021357030117
:100A50003308D8033308D800330707013306D60319
:100A60006374D7003306C601935607013386C60068
:100A700063E6C702E39CC7CEB70701009387F7FF81
:100A80003377F700131707013373F300B398B800F7
:100A90003307670093050000E3FEE8DA1305F5FF6E
:100AA0006FF0DFCC93050000130500006FF09FDAB4
:100AB00093080600138706009307050013880500B6
:100AC000639C0622B77601809386468463FCC50C3E
:100AD00037030100637E660A1303F00F6374C300DB
:100AE000130780003353E600B386660003CE06008A
:100AF000330EEE00130700023303C741630CC70136
:100B0000B3956500335EC501B31866003368BE0057
:100B1000B317650013D608013377C802139508018F
:100B20001355050193D607013358C802131707015F
:100B3000B366D7003308050363FA0601B3861601CE
:100B400063E6160163F40601B3861601B386064117
:100B500033F7C6029397070193D70701B3D6C602AE
:100B6000B306D50213150701B367F50063FAD70082
:100B7000B387170163E6170163F4D700B387170142
:100B8000B387D74033D56700930500006780000026
:100B90003703000113070001E36666F413078001C1
:100BA0006FF05FF46316060013061000B3581603C7
:100BB0003706010063F2C80A1306F00F63741601CA
:100BC0001307800033D6E800B386C60003CE0600C4
:100BD000330EEE00130700023303C7416318C70941
:100BE000B385154113D70801139508011355050165
:100BF00013D60701B3F6E502B3D5E50293960601D5
:100C0000B3E6C600B305B50263FAB600B3861601B3
:100C100063E6160163F4B600B3861601B385B640E9
:100C2000B3F6E5029397070193D70701B3D5E50221
:100C3000B305B50213950601B367F50063FAB70073
:100C4000B387170163E6170163F4B700B387170191
:100C5000B387B7406FF01FF3370600011307000199
:100C6000E3E2C8F6130780016FF0DFF5B398680080
:100C700033D7C501B3176500335EC50113D508012D
:100C8000B376A702B3956500336EBE009395080155
:100C900093D5050113560E013357A702939606010B
:100CA000B3E6C6003387E50263FAE600B3861601B1
:100CB00063E6160163F4E600B38616013386E64068
:100CC000B376A602131E0E01135E0E013356A60262
:100CD000939606013386C502B3E5C60163FAC500E3
:100CE000B385150163E6150163F4C500B3851501ED
:100CF000B385C5406FF01FEFE3EAD5E83707010081
:100D000063FCE604130EF00F3337DE0013173700D1
:100D1000B778018033D3E60093884884B3886800AD
:100D200003CE0800330EEE00130700023303C74161
:100D3000631EC70363E4B600636AC500B307C5401A
:100D4000B385D5403335F5003388A54013850700BA
:100D5000930508006FF09FE3B70800011307000137
:100D6000E3E816FB130780016FF09FFA3357C601C3
:100D7000B3966600336FD700B3D7C50113570F0181
:100D8000B3F8E702B39565003358C5013368B8007E
:100D900093150F0193D5050193560801331666008C
:100DA00033156500B3D7E70293980801B3E6D8007E
:100DB000B38EF5029388070063FED601B386E60181
:100DC0009388F7FF63E8E60163F6D6019388E7FFAF
:100DD000B386E601B386D641B3FEE60213180801D6
:100DE00013580801B3D6E602939E0E01B3EE0E012E
:100DF000B385D5029387060063FEBE00B38EEE0175
:100E00009387F6FF63E8EE0163F6BE009387E6FF83
:100E1000B38EEE01B385BE4093980801B70E010072
:100E2000B3E8F8009387FEFF33F8F8009356060105
:100E300093D80801B377F6003307F802B387F802B6
:100E40003308D802B388D8023308F8009356070154
:100E5000B386060163F4F600B388D801B707010032
:100E60009387F7FF13D80601B3F6F60093960601B1
:100E70003377F700B30818013387E60063E61501FE
:100E8000639E1501637CE5003306C7403337C70016
:100E90003307E701B388E840130706003307E5404E
:100EA0003335E500B3851541B385A540B397C5013A
:100EB0003357670033E5E700B3D565006FF01FCD0A
:100EC000130101FD23248102232A510123248101DE
:100ED000232611022322910223202103232E3101F4
:100EE000232C410123286101232671012322910132
:100EF00013040500130C0600938A060073292000D2
:100F000093D74501939BC5001397570193DBCB0003
:100F100013DAF501630C070213FBF77F9307F07FE9
:100F20006308FB081357D501939B3B00B36B770114
:100F3000B7078000B3EBFB0093193500130B1BC000
:100F4000930C0000930400006F008008B3E7AB002F
:100F5000638E070E63800B0413850B00EF40103384
:100F6000130755FF9307C00163CCE7029306D00136
:100F7000930985FFB386E640B39B3B01B356D4008B
:100F8000B3EB7601B31934019305D0C0338BA54080
:100F90006FF01FFBEF40902F130505026FF05FFC11
:100FA000930B85FDB31B7401930900006FF0DFFD07
:100FB00033E4AB006306040A9397CB009309050062
:100FC000130BF07F930C300093040001E3CC07F681
:100FD00013D74A011395CA009316570193070C00C3
:100FE0001354C5009375F77F93DAFA0163840608FA
:100FF0001307F07F6386E50E9357DC011315340069
:1010000033E5A700370480003364850093173C0064
:10101000138515C01307000093962C00B3E6E60075
:10102000B305AB409386F6FF1305E00033465A0143
:101030006360D51037650180939626001305057906
:10104000B386A60083A6060067800600930B000007
:1010500093090000130B0000930C10006FF09FEE3B
:10106000930B000093090000130BF07F930C2000FA
:101070006FF05FEDB36784016384070863020404C3
:1010800013050400EF40902093050500938655FF5B
:101090009307C00163CED7021307D001938785FF62
:1010A0003307D7403315F4003357EC003364A700FF
:1010B000B317FC001307D0C03305B7406FF09FF59E
:1010C00013050C00EF40901C930505026FF01FFC08
:1010D000138585FD3314AC00930700006FF09FFD6E
:1010E00033668401630806021317C4001305F07FFA
:1010F000634C070213073000930400016FF0DFF127
:1011000013040000930700001305000013071000EC
:101110006FF09FF013040000930700001305F07FA9
:10112000130720006FF05FEF130730006FF0DFEE62
:101130006366740163968B2E63E4F92E1395FB01AD
:1011400013D719009396F90193DB1B00B369E500EF
:101150001315840013D887013368A80013550501BF
:1011600033D3AB02131E0801135E0E019398870060
:1011700093D70901B3FBAB02930F030033076E0251
:10118000939B0B01B3E7770163FEE700B387070189
:10119000930FF3FF63E8070163F6E700930FE3FFA4
:1011A000B3870701B387E740B3DEA702939909012C
:1011B00093D90901B3F7A70213830E003307DE03A7
:1011C00093970701B3E7F90063FEE700B3870701D0
:1011D0001383FEFF63E8070163F6E7001383EEFF66
:1011E000B38707013387E740939F0F01B7070100DB
:1011F000B3EF6F001383F7FF33FF6F0093D20F013C
:1012000093DE080133F3680033046F02B38962028E
:10121000338FEE03B3033F01135F0401330F7F00ED
:10122000B382D20363743F01B382F200B7030100BB
:1012300093570F019383F3FFB3825700B3777F0077
:101240009397070133747400B3878700636857006E
:1012500013840F006314570463F2F604B386160177
:1012600033BF1601330F0F013307E7011384FFFF6C
:101270006366E8006314E80263E2160363665700DE
:10128000639EE20063FCF600B386160133BF1601CD
:10129000330F0F011384EFFF3307E701338FF6405D
:1012A00033075740B3B6E6013307D7409307F0FF43
:1012B0006304E812B352A70293570F013377A702D2
:1012C00093860200B30F5E021317070133E7E700AE
:1012D000637EF701330707019386F2FF6368070116
:1012E0006376F7019386E2FF330707013307F7417F
:1012F000B35FA70293170F0193D707013377A702B4
:10130000330EFE031317070133E7E70093870F003F
:10131000637EC701330707019387FFFF63680701F7
:101320006376C7019387EFFF3307070193960601A2
:10133000B3E6F6009397060193D707013307C74139
:1013400013DE0601330FF30233036E02338ECE0336
:10135000B38EFE0293570F01B38E6E00B387D70191
:1013600063F6670037050100330EAE0013D30701A3
:101370003303C301370E0100130EFEFF33F5C7011F
:1013800013150501337FCF013305E501636867005D
:101390006314673E93870600630005043307E80083
:1013A0009387F6FF63640703636667006314673C13
:1013B00063F0A8029387E6FF93961800B3B816016E
:1013C0003388080133070701938806006314670018
:1013D0006384A80093E717001388F53F635A001948
:1013E00013F77700630A070A1307200093E4140039
:1013F0006302E90A130730006308E908631E09085D
:1014000013F7F700930640006308D70813874700D7
:10141000B337F7003304F400930707006F00C007E9
:101420009385F5FF930600006FF09FD213060A0024
:1014300013840B009387090013870C009306300078
:101440006300D732930610006306D730930620005E
:10145000E314D7F86F00000113860A006FF01FFE37
:1014600093E4840013050000930700001307F07F46
:101470006F00C00537040800930700001306000042
:10148000130730006FF09FFB631806001387870077
:101490006FF01FF8E31C06FE13177400635A070071
:1014A000370700FF1307F7FF3374E4001388054084
:1014B0001307E07F634E070713D737009317D40154
:1014C000B3E7E7001355340013070800131747016B
:1014D000B706F07F1315C5003377D7001355C50045
:1014E0003365A7001316F6013367C500930507009F
:1014F000138507006384040073A014008320C102D5
:101500000324810283244102032901028329C101AA
:10151000032A8101832A4101032B0101832BC1008E
:10152000032C8100832C410013010103678000001C
:1015300093072000630AF90293073000630AF90059
:10154000631A0900930700001307F07F6F00000182
:10155000E30A06FE9307F0FF1307E07F93E45400CD
:10156000138507006FF09FF6E31E06FC6FF09FFEE9
:10157000130710006316080693F67700130704009C
:10158000638A06041307200093E414006300E9044F
:10159000130730006304E90213070400631C090207
:1015A00093F6F700130540006386A60213B7C7FF42
:1015B00013471700330787006F00C00113070400AB
:1015C000631A060013B787FF6FF09FFE130704002E
:1015D000E31A06FE13578701134717001377170006
:1015E00013051000330505419306800363CCA60E56
:1015F0009306F00163C2A6069385E54133D8A700A0
:10160000B316B400B397B700B3E60601B337F000E2
:10161000B3E7F6003355A40093F67700638006081D
:101620009306200093E414006308D9069306300063
:10163000630ED9046314090693F6F700930540007E
:10164000638EB60493864700B3B7F6003305F50002
:10165000938706006F008004930610FEB386064150
:1016600093080002B356D400130800006306150166
:101670009385E5433318B400B367F800B337F0003F
:10168000B3E7F600130500006FF01FF963180600BA
:10169000938687006FF05FFBE31C06FE93168500C0
:1016A00063DE060093E414001305000093070000B6
:1016B00063160702130710006FF05FE193D637003F
:1016C0009317D501B3E7D70013553500E30007E0C2
:1016D00013F71400E30C07DE1307000093E4240063
:1016E0006FF0DFDEB3E78700638407029307200013
:1016F00093E41400630EF902930730006302F902C9
:1017000093071000631409009307500093D7370024
:1017100093E4240013050000130700006FF01FDBA3
:1017200093079000E30406FE930710006FF01FFE7E
:1017300093079000E31C06FC6FF01FFF37050800BD
:10174000930700001307F07F1306000093040001C5
:101750006FF0DFD713050000930700006FF0DFFB89
:1017600037050800930700001307F07F13060000F9
:101770006FF0DFD593860700938706006FF09FC553
:10178000130101FD232481022328610123229101F9
:10179000232611022322910223202103232E31012B
:1017A000232C4101232A5101232671012324810185
:1017B00013040500930C0600138B06007329200008
:1017C00093D745019399C5001397570193D9C90041
:1017D00093DAF501630C070293FBF77F9307F07F21
:1017E0006388FB089357D50193993900B3E9370112
:1017F000B7078000B3E9F900131A3500938B1BC0BB
:10180000130C0000930400006F008008B3E7A900E8
:10181000638007106380090413850900EF400027E7
:10182000130755FF9307C00163CCE7029307D0016C
:10183000130A85FFB387E740B3994901B357F40012
:10184000B3E93701331A4401930BD0C0B38BAB40DB
:101850006FF01FFBEF408023130505026FF05FFC64
:10186000930985FDB3193401130A00006FF0DFFD01
:1018700033E4A9006308040A9397C900130A05001A
:10188000930BF07F130C300093040001E3CC07F6B8
:1018900013574B011314CB009316570193870C0079
:1018A0001354C4001375F77F135BFB0163860608AE
:1018B0001307F07F6306E50E93D7DC0113143400A1
:1018C00033E48700B70780003364F400130515C0C4
:1018D00093973C001307000093162C00B3E6E60034
:1018E000B38BAB009386F6FF1306E000B3C56A0125
:1018F00013851B00636AD61637660180939626000F
:101900001306C67CB386C60083A606006780060061
:1019100093090000130A0000930B0000130C100041
:101920006FF05FEE93090000130A0000930BF07F45
:10193000130C20006FF01FEDB3679401638207085A
:101940006300040413050400EF404014930655FFA0
:101950009307C00163CED7021307D001930785FF19
:101960003307D7403314F40033D7EC0033648700D7
:10197000B397FC001307D0C03305A7406FF09FF565
:1019800013850C00EF408010130505026FF01FFC5B
:10199000130485FD33948C00930700006FF09FFDC6
:1019A00033669401630806021317C4001305F07F21
:1019B000634C070213073000930400016FF0DFF15E
:1019C0001304000093070000130500001307100024
:1019D0006FF09FF013040000930700001305F07FE1
:1019E000130720006FF05FEF130730006FF0DFEE9A
:1019F00037040800930700001307F07F93050000E9
:101A00009304000113174701B706F07F1314C400B5
:101A10003377D7001354C4009395F50133648700DE
:101A20003367B4001385070093050700638404003F
:101A300073A014008320C102032481028324410285
:101A4000032901028329C101032A8101832A41015B
:101A5000032B0101832BC100032C8100832C410047
:101A60001301010367800000370601001307F6FF2A
:101A700093560A0113DE0701337AEA00B3F7E70051
:101A800033034E03B38E4703338FF6023308E3016B
:101A900013D30E0133030301B388C6036374E30158
:101AA000B388C8003378E300B3FEEE001356030199
:101AB00013180801135304013374E4003308D801E8
:101AC000330F8A02B38E8602330A43033307DA01E7
:101AD000135A0F01330AEA00B38666026376DA010D
:101AE00037070100B386E600935E0A01B38EDE007D
:101AF000B70601009382F6FF337A5A00337F5F0006
:101B000013D70901131A0A01B3F95900330AEA017C
:101B1000B302EE02B30F4601338F3703330E3E0399
:101B200013560F01B307F702330EFE003306C6014A
:101B30006374F600B382D200B70601009387F6FF04
:101B4000135E06013376F600337FFF00131606019D
:101B5000B38789023306E601330E5E003304870241
:101B6000330FE30213D70701330333033303830037
:101B70003303670063748300330FDF00370701000E
:101B80001307F7FFB376E300B3F7E7009396060178
:101B9000B388F801B386F60033BA4801B386D6019C
:101BA00033874601B388C80033B6C800B30FC701F6
:101BB000B382CF00B3B6D6013337470133E7E6002F
:101BC00033B6C2001353030133BECF01330767009E
:101BD0003366CE00939798003307C7003307E701B9
:101BE000B3E7070113179700B337F00093D87801D4
:101BF00013D47201B3E71701939292009316770002
